:020000022000DC
:1060000000000420B995020065820200BD870200ED
:1060100065820200658202006582020000000000C5
:106020000000000000000000000000006582020087
:1060300065820200000000006582020065820200A5
:106040006594020065820200B19902005D98020029
:106050006D98020065820200E585020065820200FB
:106060006582020091990200A199020089950200BF
:10607000658202006582020065820200658202007C
:10608000F19D02009995020065820200658202007E
:106090006582020065820200D598020065820200D6
:1060A000658202006582020065820200658202004C
:1060B000658202006582020000000000000000000E
:1060C0006582020065820200658202007D980200FE
:1060D000A99502006582020065820200D199020042
:1060E000C19902006595020065820200A99802002C
:0860F0000000000065820200BF
:1070000040F8044B40F8045B40F8046B40F8047B04
:1070100040F8048B40F8049B40F804AB40F804BBF4
:1070200040F804CB40F804DB6846704781F000412B
:1070300002E000BF83F0004330B54FEA41044FEA5D
:10704000430594EA050F08BF90EA020F1FBF54EAF8
:10705000000C55EA020C7FEA645C7FEA655C00F094
:10706000E2804FEA5454D4EB5555B8BF6D420CDD65
:107070002C4480EA020281EA030382EA000083EAE8
:10708000010180EA020281EA0303362D88BF30BD88
:1070900011F0004F4FEA01314FF4801C4CEA1131DE
:1070A00002D0404261EB410113F0004F4FEA03333D
:1070B0004CEA133302D0524263EB430394EA050FC8
:1070C00000F0A780A4F10104D5F1200E0DDB02FA37
:1070D0000EFC22FA05F2801841F1000103FA0EF2CB
:1070E000801843FA05F359410EE0A5F120050EF191
:1070F000200E012A03FA0EFC28BF4CF0020C43FAC2
:1071000005F3C01851EBE37101F0004507D54FF0CE
:10711000000EDCF1000C7EEB00006EEB0101B1F51E
:10712000801F1BD3B1F5001F0CD349085FEA300064
:107130004FEA3C0C04F101044FEA445212F5800F6F
:1071400080F09A80BCF1004F08BF5FEA500C50F10C
:10715000000041EB045141EA050130BD5FEA4C0CEF
:10716000404141EB0101013C28BFB1F5801FE9D24C
:1071700091F0000F04BF01460020B1FA81F308BF6F
:107180002033A3F10B03B3F120020CDA0C3208DD3B
:1071900002F1140CC2F10C0201FA0CF021FA02F116
:1071A0000CE002F11402D8BFC2F1200C01FA02F186
:1071B00020FA0CFCDCBF41EA0C019040E41AA2BFAB
:1071C00001EB0451294330BD6FEA04041F3C1CDA73
:1071D0000C340EDC04F11404C4F1200220FA04F093
:1071E00001FA02F340EA030021FA04F345EA03013D
:1071F00030BDC4F10C04C4F1200220FA02F001FAFF
:1072000004F340EA0300294630BD21FA04F0294680
:1072100030BD94F0000F83F4801306BF81F4801119
:107220000134013D4EE77FEA645C18BF7FEA655C8C
:1072300029D094EA050F08BF90EA020F05D054EA5E
:10724000000C04BF1946104630BD91EA030F1EBF63
:107250000021002030BD5FEA545C05D14000494167
:1072600028BF41F0004130BD14F580043CBF01F55A
:10727000801130BD01F0004545F0FE4141F4700140
:107280004FF0000030BD7FEA645C1ABF194610461B
:107290007FEA655C1CBF0B46024650EA013406BF1C
:1072A00052EA033591EA030F41F4002130BD00BFDB
:1072B00090F0000F04BF0021704730B54FF4806498
:1072C00004F132044FF000054FF0000150E700BF19
:1072D00090F0000F04BF0021704730B54FF4806478
:1072E00004F1320410F0004548BF40424FF0000165
:1072F0003EE700BF42004FEAE2014FEA31014FEAA8
:1073000002701FBF12F07F4393F07F4F81F06051F6
:10731000704732F07F4208BF704793F07F4F04BF41
:1073200041F40021704730B54FF4607401F000451E
:1073300021F000411CE700BF50EA010208BF70477E
:1073400030B54FF000050AE050EA010208BF70476F
:1073500030B511F0004502D5404261EB41014FF4D8
:10736000806404F132045FEA915C3FF4D8AE4FF0E0
:1073700003025FEADC0C18BF03325FEADC0C18BFC3
:10738000033202EBDC02C2F1200300FA03FC20FA14
:1073900002F001FA03FE40EA0E0021FA02F1144461
:1073A000BDE600BF4FEA4102B2F1E04324BFB3F5AE
:1073B000001CDCF1FE5C0DD901F0004C4FEAC0026C
:1073C0004CEA5070B2F1004F40EB830008BF20F050
:1073D0000100704711F0804F21D113F13872BCBF0A
:1073E00001F00040704741F480114FEA5252C2F15F
:1073F0001802C2F1200C10FA0CF320FA02F018BFA8
:1074000040F001004FEAC1234FEAD32303FA0CFCFA
:1074100040EA0C0023FA02F34FEA4303CCE77FEA89
:10742000625307D150EA01331EBF4FF0FE4040F4D3
:107430004000704701F0004040F0FE4040F4000082
:10744000704700BF80F0004002E000BF81F00041C3
:1074500042001FBF5FEA410392EA030F7FEA226CFA
:107460007FEA236C6AD04FEA1262D2EB1363C1BF8A
:10747000D218414048404140B8BF5B42192B88BFF9
:10748000704710F0004F40F4000020F07F4018BF1C
:10749000404211F0004F41F4000121F07F4118BF3C
:1074A000494292EA030F3FD0A2F1010241FA03FCE4
:1074B00010EB0C00C3F1200301FA03F100F00043CC
:1074C00002D5494260EB4000B0F5000F13D3B0F194
:1074D000807F06D340084FEA310102F10102FE2A03
:1074E00051D2B1F1004F40EBC25008BF20F0010073
:1074F00040EA03007047490040EB0000013A28BF12
:10750000B0F5000FEDD2B0FA80FCACF1080CB2EB94
:107510000C0200FA0CF0AABF00EBC2505242184312
:10752000BCBFD0401843704792F0000F81F40001B7
:1075300006BF80F400000132013BB5E74FEA41038A
:107540007FEA226C18BF7FEA236C21D092EA030FF6
:1075500004D092F0000F08BF0846704790EA010F70
:107560001CBF0020704712F07F4F04D1400028BF9D
:1075700040F00040704712F100723CBF00F500007F
:10758000704700F0004343F0FE4040F400007047B5
:107590007FEA226216BF08467FEA23630146420261
:1075A00006BF5FEA412390EA010F40F48000704774
:1075B0004FF0000304E000BF10F0004348BF40421A
:1075C0005FEA000C08BF704743F0964301464FF056
:1075D00000001CE050EA010208BF70474FF00003B2
:1075E0000AE000BF50EA010208BF704711F00043F3
:1075F00002D5404261EB41015FEA010C02BF8446C3
:107600000146002043F0B64308BFA3F18053A3F521
:107610000003BCFA8CF2083AA3EBC25310DB01FA68
:1076200002FC634400FA02FCC2F12002BCF1004FEC
:1076300020FA02F243EB020008BF20F0010070477D
:1076400002F1200201FA02FCC2F1200250EA4C00D1
:1076500021FA02F243EB020008BF20EADC70704717
:107660007BB972B90029BEBF00204FF0004106E08F
:1076700008BF00281CBF6FF000414FF0FF3000F042
:107680001DBBADF1080C6DE904CE002909DB002B10
:107690001ADB00F081F8DDF804E0DDE9022304B034
:1076A0007047404261EB4101002B1BDB00F074F896
:1076B000DDF804E0DDE9022304B0404261EB410162
:1076C000524263EB43037047524263EB430300F0C3
:1076D00063F8DDF804E0DDE9022304B0404261EB29
:1076E00041017047524263EB430300F055F8DDF867
:1076F00004E0DDE9022304B0524263EB4303704728
:1077000053B94AB9002908BF00281CBF4FF0FF3108
:107710004FF0FF3000F0D2BAADF1080C6DE904CEA5
:1077200000F03AF8DDF804E0DDE9022304B0704728
:1077300007EE900AF5EEC07AF1EE10FA01D400F0EF
:107740000BB8F1EE677A08B517EE900A00F004F86E
:10775000404261EB410108BDD0B5FFF7CBFD0C4BBA
:10776000002206460F4600F07FF900F0A9FA044611
:10777000FFF79EFD074B002200F076F902460B460C
:1077800030463946FFF756FC00F09AFA2146D0BD44
:107790000000F03D0000F0412DE9F047089D04464F
:1077A0008E46002B4DD18A42944669D9B2FA82F2B4
:1077B00052B101FA02F3C2F1200120FA01F10CFAF0
:1077C00002FC41EA030E94404FEA1C48210CBEFB28
:1077D000F8F61FFA8CF708FB16E341EA034306FBB1
:1077E00007F199420AD91CEB030306F1FF3080F040
:1077F0001F81994240F21C81023E63445B1AA4B28D
:10780000B3FBF8F008FB103344EA034400FB07F72E
:10781000A7420AD91CEB040400F1FF3380F00A816F
:10782000A74240F207816444023840EA0640E41B64
:1078300000261DB1D4400023C5E900433146BDE810
:10784000F0878B4209D9002D00F0EF800026C5E9B2
:10785000000130463146BDE8F087B3FA83F6002ECA
:107860004AD18B4202D3824200F2F980841A61EB42
:10787000030301209E46002DE0D0C5E9004EDDE760
:1078800002B9FFDEB2FA82F2002A40F09280A1EB48
:107890000C014FEA1C471FFA8CFE0126200CB1FB9D
:1078A000F7F307FB131140EA01410EFB03F0884296
:1078B00008D91CEB010103F1FF3802D2884200F223
:1078C000CB804346091AA4B2B1FBF7F007FB1011B5
:1078D00044EA01440EFB00FEA64508D91CEB040453
:1078E00000F1FF3102D2A64500F2BB800846A4EBAE
:1078F0000E0440EA03409CE7C6F12007B34022FA99
:1079000007FC4CEA030C20FA07F401FA06F31C43C7
:10791000F9404FEA1C4900FA06F3B1FBF9F8200CD4
:107920001FFA8CFE09FB181140EA014108FB0EF01A
:10793000884202FA06F20BD91CEB010108F1FF3A6A
:1079400080F08880884240F28580A8F10208614476
:10795000091AA4B2B1FBF9F009FB101144EA014184
:1079600000FB0EFE8E4508D91CEB010100F1FF342F
:107970006CD28E456AD90238614440EA0840A0FBC7
:107980000294A1EB0E01A142C846A64656D353D09D
:107990005DB1B3EB080261EB0E0101FA07F722FAC1
:1079A00006F3F1401F43C5E9007100263146BDE8EA
:1079B000F087C2F12003D8400CFA02FC21FA03F34D
:1079C000914001434FEA1C471FFA8CFEB3FBF7F0CE
:1079D00007FB10360B0C43EA064300FB0EF69E42F3
:1079E00004FA02F408D91CEB030300F1FF382FD28C
:1079F0009E422DD9023863449B1B89B2B3FBF7F634
:107A000007FB163341EA034106FB0EF38B4208D90C
:107A10001CEB010106F1FF3816D28B4214D9023E4D
:107A20006144C91A46EA004638E72E46284605E76B
:107A30000646E3E61846F8E64B45A9D2B9EB02083C
:107A400064EB0C0E0138A3E74646EAE7204694E7CC
:107A50004046D1E7D0467BE7023B614432E73046FF
:107A600009E76444023842E770B54FF0FF0C4CF46C
:107A7000E06C1CEA11541DBF1CEA135594EA0C0F6C
:107A800095EA0C0F00F0DEF82C4481EA030621EAA7
:107A90004C5123EA4C5350EA013518BF52EA0335E2
:107AA00041F4801143F4801338D0A0FB02CE4FF094
:107AB0000005E1FB02E506F00042E0FB03E54FF0C4
:107AC0000006E1FB03569CF0000F18BF4EF0010EBC
:107AD000A4F1FF04B6F5007F64F5407404D25FEAB8
:107AE0004E0E6D4146EB060642EAC62141EA55516B
:107AF0004FEAC52040EA5E504FEACE2EB4F1FD0CAD
:107B000088BFBCF5E06F1ED8BEF1004F08BF5FEA2A
:107B1000500E50F1000041EB045170BD06F00046DC
:107B200046EA010140EA020081EA0301B4EB5C0489
:107B3000C2BFD4EB0C0541EA045170BD41F4801181
:107B40004FF0000E013C00F3AB8014F1360FDEBFA6
:107B5000002001F0004170BDC4F10004203C35DA82
:107B60000C341BDC04F11404C4F1200500FA05F305
:107B700020FA04F001FA05F240EA020001F00042A6
:107B800021F0004110EBD37021FA04F642EB06011C
:107B90005EEA430E08BF20EAD37070BDC4F10C0446
:107BA000C4F1200500FA04F320FA05F001FA04F20A
:107BB00040EA020001F0004110EBD37041F10001F6
:107BC0005EEA430E08BF20EAD37070BDC4F1200501
:107BD00000FA05F24EEA020E20FA04F301FA05F269
:107BE00043EA020321FA04F001F0004121FA04F211
:107BF00020EA020000EBD3705EEA430E08BF20EAE1
:107C0000D37070BD94F0000F0FD101F0004640001A
:107C100041EB010111F4801F08BF013CF7D041EA9C
:107C2000060195F0000F18BF704703F000465200A0
:107C300043EB030313F4801F08BF013DF7D043EA71
:107C40000603704794EA0C0F0CEA135518BF95EA27
:107C50000C0F0CD050EA410618BF52EA4306D1D1AE
:107C600081EA030101F000414FF0000070BD50EACD
:107C7000410606BF1046194652EA430619D094EA57
:107C80000C0F02D150EA013613D195EA0C0F05D141
:107C900052EA03361CBF104619460AD181EA030195
:107CA00001F0004141F0FE4141F470014FF000004D
:107CB00070BD41F0FE4141F4780170BD704700BFD6
:107CC0004A0011D212F5001211D20DD56FF478735B
:107CD000B3EB62520ED44FEAC12343F0004343EAB0
:107CE000505323FA02F070474FF00000704750EAFB
:107CF000013002D14FF0FF3070474FF00000704765
:107D00002DE9F8439DF834C080F84AC00446CCF110
:107D1000080C80F84EC0002084F854006060BDF963
:107D20002800A4F85600BDF92C00A4F858009DF8CE
:107D3000380084F84F009DF83C0084F851009FED16
:107D4000307B9DF8400084F84B009DF8440084F897
:107D500052009DF84800BDF82050BDF82470BDF8D1
:107D6000306084F8530084ED027B91469846A9B1B7
:107D70008B0740D10868244B984226D0234B984269
:107D80002ED0234B984236D1224820612248606190
:107D90002248A0612248E0612248206221602249F5
:107DA0008C420DD0A4F84090A4F84280A4F846502C
:107DB000A4F8487031462046BDE8F84320F0A6BB41
:107DC0004146484654F0A4FCECE7184820611848A6
:107DD00060611848A0611848E06118482062DDE73A
:107DE00017482061174860611748A0611748E06193
:107DF00017482062D2E7174838F05CF9AFF30080EB
:107E00000000000000000000386B0900EC000900D1
:107E10008C020900B9DD030099DD030089DD030050
:107E2000E9DD0300B1DD030018090120E9EC0300DE
:107E300071A20300D1EC030019ED0300E1EC030093
:107E400085DB030059DB030029DB0300BDDB0300F6
:107E500071DB030008AD090030B5144685B019A3E5
:107E6000D3E90023FFF74CFC0546A0F16150A0F5D3
:107E7000351001A9A0F5607055F0A4FC9DF80730FD
:107E80009DF806109DF808201B0443EA41539DF815
:107E9000091043EAC2239DF80A2043EA411343EA4A
:107EA0005203BDF804200649A2F2BC7225F0010578
:107EB00043EA4263A5FB0101236005B030BD00BF6A
:107EC00000CA9A3B00CA9A3B00000000DAB32DE9D1
:107ED000F0414C1E84B00646A518102100F1F007B1
:107EE0004FF0000810290FD00A46013104AB1A44A4
:107EF00014F8013F12F8102CAC4283EA02032370FD
:107F0000F0D104B0BDE8F08138687968BA68FB68E0
:107F1000EC46ACE80F003146684600F0C9F806F5BB
:107F200080710F2211F8013DFF2B06D0324401333E
:107F300082F8F03001210022D8E7013A531C81F881
:107F40000080EFD1F6E77047182A2DE9F04FC0F80E
:107F500000215ED0202A00F08880102A7FD00023E4
:107F60001D46A0F804311A461946434EDFF80CB1FD
:107F700005EB81032FE016F804A01BF8099016F812
:107F80000E4016F80CE016F808C08AEA09088A1AAA
:107F900005EB820915F8222088EA020883F80080A0
:107FA00099F801200433544003F8034C99F8022057
:107FB0008EEA020E03F802EC99F803208CEA020C18
:107FC00003F801CC90F8042101310132B1EB820FAA
:107FD00043D290F80521B1FBF2F902FB191A13F80C
:107FE000048C13F8034C13F802EC13F801CCBAF12B
:107FF000000FC0D0D0F80071202FC8D1BAF1040F03
:10800000C5D116F80880345D16F80EE016F80CC0DD
:10801000BDE740F20C63A0F8043105460B468446E8
:1080200000241A788CF800205A788CF801209A786D
:108030008CF80220DA788CF8032090F805210134BE
:108040009442114603F104030CF1040CE9D390F8B7
:1080500004310133B2EB830F87D3BDE8F08F40F2D8
:108060000A43A0F804310546D8E740F60E03A0F80D
:1080700004310546D2E700BF207E09002CB9080074
:1080800030B500010C1D01F11405231F02EB000C9B
:1080900019781CF801EB81EA0E0103F8011BA342D9
:1080A000F6D11C1DAC4200F10400EED130BD00BF82
:1080B0002DE9F04FD1F8003187B0A3F11002102A5A
:1080C0000491824600F2C7800123934003F00133FC
:1080D00023F08073002B14BF0B46002307EE903A69
:1080E00017EE902A51460020FFF7CAFF01230293A2
:1080F0000AF104030593DFF868B10AF11003019354
:10810000D0460598C6464246002312F823101BF8B5
:10811000011002F823100133042BF6D101329042F2
:10812000F2D198F80D2098F8011098F8023098F8DC
:10813000090088F8092098F8062098F80AA088F81D
:108140000D1088F80A3098F80E1098F8033088F867
:108150000E2098F80B2098F8054098F80F9088F8B2
:108160000F2098F8072088F80730049B88F80B2028
:1081700088F8014088F8050088F802A088F8061001
:1081800088F8039093F80431029A93425AD0CDF8BC
:108190000C809EF800508AEA090785EA040C84EAFC
:1081A0000A0885EA09038CEA070600934FEADC1007
:1081B0004FEAD811FA09DB09744086EA0A0A86EA0E
:1081C0000909754000EB4000009E01EB410102EB04
:1081D000420203EB430300EBC00001EBC10102EBE1
:1081E000C20203EBC30383EA460380EA4C0081EA40
:1081F000480182EA470283EA09096840019B8EF838
:1082000000004C4082EA0A0A8EF801408EF802A073
:108210008EF803900EF1040E734506D09EF80140CF
:108220009EF802A09EF80390B3E7DDE9024817EE3E
:10823000902A20464146FFF723FF20460130C3B273
:1082400002935EE717EE902A0298414607B0BDE818
:10825000F04FFFF715BF002307EE903A40E700BF4D
:10826000207E0900FEE700BF2DE9F04F4FEAA3088A
:1082700003F00304644B03EB841943461C2B86462E
:108280006248A8BF1C2350F824A0D9F80400033387
:1082900089B023EAE37318410590D9F80800184122
:1082A0000690D9F80C00B8F11F0FC34640FA03F34B
:1082B000A8BF4FF01F0B079300205B460490C346F6
:1082C000C846D1469A460EE008AC04EB850555F841
:1082D000104C002B40EA0400B8BF6442013A41F858
:1082E000044B00F08E805EF8043B23F0004424F041
:1082F000030423F00045002CE6D023F0004424F0D2
:108300000F0454B958F82540BBF1000FBABFCAF1A9
:108310000005AC4044FA0AF4DBE723F0004424F003
:108320003F0474B93A4C103D54F825504C4685FB37
:1083300004642546AAF10304002C57DB45FA04F433
:10834000C7E76C04B4F1006FB6BF6C0500250425C7
:10835000B4F1005F009503DA009D0235A40000959A
:10836000B4F1804F03DA009D013564000095294D7A
:10837000294E2A4FAC422A4DC8BFAC46294DD8BF22
:10838000B446294ED8BF2E46284DD8BF2F46284D7B
:108390000297284FD8BF2F46274D0197274FD8BFA8
:1083A0002F460397254686FB05756544264685FBC3
:1083B00006C6039F25463E4486FB05C5019F3D44F6
:1083C00085FB0464029F1E4D3C44009F55F82750D6
:1083D00084FB0565ED004C4685FB04642546194C7D
:1083E00054F82740AAEB0404002CA7DA66426FF089
:1083F000004444FA06F7AF42FFF66BAF05FA06F405
:1084000067E709B0BDE8F08FA46F0900946E09001A
:10841000E46E09009979825A28482EB0B477F5FEA7
:10842000A4F633D3A9BDA02963218510591858FF9C
:108430008D496C23F0CEC2271BAA57598B40E946C1
:10844000C46E0900A46E09002DE9F04F9BBB12F029
:10845000010C2DD0D0F88012D0F88023D0F88041C4
:1084600049425242C0F88012C0F88023D0F88014EC
:10847000D0F880259C46D0F88036494252425B4273
:10848000C0F88014C0F88025D0F88010D0F880277C
:10849000C0F88036D0F880386442524249425B428C
:1084A000C0F88041C0F88010C0F88027C0F880383C
:1084B0006046BDE8F08F4FF00046DE4012F0010C40
:1084C00006F1FF36C3F11F0547D04FF0000C00F155
:1084D000800400F51068674654F8802C42FA05F9CC
:1084E0004FEAE27AB9EBE27F18BF86EA0A029A40C5
:1084F000BE4644F8802C82EAE27EAEEBE27ED0F803
:108500008020524242FA05FA4FEAE27BBAEBE27F60
:1085100018BF86EA0B029A40B946C0F8802082EA6A
:10852000E279A9EBE2790A684EEA090E4CEA0E0CF0
:1085300042FA05FEBEEBE27F4FEAE27918BF86EA17
:10854000090200F580709A40804541F8042B04F53B
:108550008074C1D16046BDE8F08F00F1800400F561
:10856000106E674654F8802C42FA05F94FEAE27A19
:10857000B9EBE27F18BF86EA0A029A40B84644F88F
:10858000802C82EAE278A8EBE278D0F8802042FAE8
:1085900005FA4FEAE27BBAEBE27F18BF86EA0B02EC
:1085A0009A40B946C0F8802082EAE279A9EBE279E4
:1085B0000A6848EA09084CEA080C42FA05F8B8EBE0
:1085C000E27F4FEAE27918BF86EA090200F580707F
:1085D0009A40864541F8042B04F58074C2D1604668
:1085E000BDE8F08F2DE9F04F0022164689B06C4BA4
:1085F0006C4C6D48CDE9022235460122196841B123
:10860000D4F80413114204D01D6019680191019936
:108610001643043383424FEA4202EFD1614BD3F851
:108620007C21002A6BD00022C3F87C21D3F87C3156
:1086300000934FF0A042009BD2F810255B4B0292B2
:10864000D3F810250392F3B2002B7AD100224FF019
:10865000FF33574EDFF85491CDE90622CDE90433BC
:10866000A6F15A08534C002514F9010B471C30D0D1
:10867000C0F3C20E08AB03EB0E0C00F007021CF8AF
:10868000103CD340D907C7B200F03F0021D508EB1A
:108690000003B90993F9283058F82330002B5CD037
:1086A00003295CD01F2887BF07F01F07CE46074667
:1086B0004FF0A04E1CF818CC0EEB87072CFA02F2F4
:1086C000D7F800C7D207CCF3014C3DD4BCF1030F5F
:1086D00054D0A642C8D18DB34FF0A0430299D3F82D
:1086E0001035D9F81025994202D10399914225D02D
:1086F000DDE906010293CDE903200591B2E7F3B26B
:10870000D3B12D4F01250024A30003F180432E4255
:1087100003F5C0434FEA45050BD0D3F8100557F8D1
:108720002420D3F81015C0F30520C1F3014102B194
:1087300090470134082CE7D1002E87DB09B0BDE853
:10874000F08F46F00046DCE7BCF1020FC1D10329EF
:1087500023D0002BBDD09847BBE70329B9D10DF139
:10876000180A4FF0010B1AF80EA00BFA02FB4AEAA6
:108770000B0A0DF1180B0BF80EA093E70329E8D1B3
:108780004FF4003CD7F8002722F44032013542EA8A
:108790000C02EDB2C7F80027DBE74FF4403CF1E7ED
:1087A0000061004000600040206100400003005074
:1087B000C2510120C05101206851012008B502209A
:1087C0004BF008FE2DE9F04FB7B0CDE91023409BE8
:1087D0001B68002B0C4640F3B48401F1240303937F
:1087E000A0F10C03079300920023A2F59062CDE95B
:1087F00001320493119A03999369526906922439BC
:10880000059133B1409B01995B698B42C8BF00223F
:108810000692409B409A1B690199D2680A928B424A
:1088200000F38684069B43EA0205409B9B69062B66
:1088300000F36684079A039CC3F107071346483385
:1088400000200F9319460B971BAE034694468A6887
:108850003A41D31A4A683A41181AD31A54F8042DE7
:10886000306208393A418C4546F8043D2260EED129
:108870001B9E149FDDF858C0129B1599139C721013
:10888000DDE919690892A7EB0C02A2EB09005A1066
:108890000992189A0D90C2EB630E179B9B1B0C93C9
:1088A00007EB0C02834B83FB0101179BE01A801B33
:1088B000804B83FB0080804B0E90924683FB0A8A9C
:1088C0007E484F4480FB0787A9EB0C0983FB09C94D
:1088D00080FB02C2DDF8308000F1705000F54C20C2
:1088E000C34600F2CB2080FB0BCB754B264483FBA9
:1088F00006C6179B04EB030C80FB0C4C70484346E8
:1089000080FB0343099C0D98A046189C5B0008EB74
:1089100064087C00C3EB4C0304EB4A040EEB600CD0
:108920004FEA460AAEEB000E08EB41060AEB4B0A93
:10893000CDF858E0520006EB040EC2EB4902A8EB5A
:108940004101D64404EB020BCDF848E001EB020EE6
:108950003244A3EB0A090C44A6EB0B07D21AA1EB95
:108960000B01A1EB09014F4418920E9A159117972C
:108970001F991D9FDDF878800EEB03060CEB420378
:1089800014961393219E7B1A0899239FA4EB0A0047
:1089900009901A90A1EB0609ACEB42001D991F9AB1
:1089A00019908818229A2099DF1B0C97891A1C9F0E
:1089B000404A82FB0838209EA7EB060E229EAEEBB3
:1089C000060E82FB0E3E3C4E834686FB0B3B1D9AF9
:1089D000239B3A4CD31884FB0323239A94461F9A73
:1089E000ACEB020C86FB0C2C064684FB062604F13D
:1089F000705404F54C240D968A4604F2CB2484FB73
:108A00000A2A229A2E48BA1880FB0262209E374416
:108A100084FB076780FB01610898219E0D9C00EB99
:108A20006606520060005B000C9C03EB4B0302EBFC
:108A30004A0AC0EB4C0C06EB48024900A6EB48067C
:108A4000C1EB470103EB0C00A9EB040702EB0308A1
:108A500033441F97A3EB0A0706EB0C0309EB640BE7
:108A60000B44A1EB0A09361A9444101AD044ACEB1B
:108A700001011D93A6EB090648440BEB4E03ABEB3B
:108A80004E02CDF86C80239721911E9620901C9366
:108A90002292002D40F0DE82DDF800A00949DFF8C7
:108AA0002C80059E084B099C0DF1680C2846AE46AB
:108AB000D14613E0A1EBD96E8BBE0D627E1A3A1639
:108AC000322E0E7E040A09005CEB270B1CF1080015
:108AD000DCF8207058F8043D5CF8044D83FB072750
:108AE00007EBA403326846F8043BA7EBA407544203
:108AF00051F8083CE41B84FB03B307EB830351F8F4
:108B0000047C84FB07B7C2EB87024AF82030744626
:108B1000C9F8802883EAE374A4EBE374734682EA1D
:108B2000E273A3EBE2731C43029BA9F180094B455E
:108B300045EA040501F1080100F12000C8D1039ABB
:108B4000039C019E009F0B9B059924320392029A7D
:108B5000043202923846324601360196FFF774FC21
:108B6000049B284303430493079B543318463B4616
:108B7000043300930F9B0793409B1B68B3423FF75E
:108B800039AE409B019A5B689A4280F2E98104F118
:108B900024030393109B03EB820303F5C073061DAC
:108BA000029324AB0593B046409B0199D3E903237C
:108BB0008B42C8BF00220092409B029A9B69A2F59B
:108BC000C07B039A062BA2F1240107EE901A07EE50
:108BD00010BAA8F1040000F39082C3F107040694D0
:108BE000002250F82230234140F8223058F8223039
:108BF000234148F8223051F8043B02322341122A23
:108C000041F8043CEDD1D8F83820D8F82C00D8F839
:108C10002030D8F81440D8F80850B94E871AD91B1C
:108C2000641A2B1B58F8045C891AE81A5B1A401066
:108C30005B1086FB045400EB6706B14DC01B06EBCE
:108C40004407A6EB440685FB014103EB620404EBF9
:108C500041054FEA410EAB4981FB05C5AA499A1A65
:108C6000AD0081FB0232A949A4EB0E04920081FB06
:108C70000434D8F83030D8F83C10A3EB010CD8F805
:108C80002430D8F81810A3EB0C03A1EB0309D8F893
:108C90003C10A3EB010ED8F80C30D8F8001007EB0D
:108CA000050A7D1BA3EB090317958518821AC91ABB
:108CB0001692A3EB0E0306EB8402A6EB8404491084
:108CC0005B10CDF848A01395CDE914248C4880FBA7
:108CD000092901EB6C02A1EB0C0102EB490607919B
:108CE000A2EB490980FB0E2ED8F83C50854C03EBD3
:108CF000650505EB4E074FEA4E0E84FB0727D8F8B3
:108D00003C20814C9B1ABF0084FB03237F4AA5EBC8
:108D10000E05980082FB0535D8F840E0D8F83430CD
:108D2000D8F82820D8F81C40A3EB0E03D21AF1196A
:108D3000A41AA2EB0E0AD8F81020089118910799EE
:108D4000121BF61BA446D8F804401D960E18A41A50
:108D5000091AA2EB0A020796199609EB8506A9EBF8
:108D60008505641052101C910996CDE91A65644876
:108D700080FB0C1C04EB630101EB4C05E41AA1EB36
:108D80004C0680FB0A3A02EB6E0101EB4A005D4F94
:108D90004FEA4A0A87FB00305B4FA2EB0E028000CD
:108DA00087FB02324FEA820EA1EB0A0A574A82FB86
:108DB0000A3A04EB0E01A4EB0E041F91229406EB79
:108DC0008A03059C009AA6EB8A01CDE92031291877
:108DD0002B1A0A9117EE900A2146239301F01EF8F0
:108DE00000234B490093224614A812ACCDF82C80E6
:108DF00052F8043B4FF000089B0083EAE378A8EBAD
:108E0000E378CBF80030936800279B0083EAE37790
:108E1000A7EBE377CBF88031E3681D4651F8043BBC
:108E200083FB0565536905EB8303002583EAE3753E
:108E3000A5EBE375CBF80033C3689E468B6883FBD4
:108E40000E9E136A0EEB830E00238EEAEE73A3EBE5
:108E5000EE730668CBF880E40438B6464E6986FBAC
:108E60000E9E666AB14651F8046C86FB09A9D66A63
:108E7000CE440EEB86064FF0000E86EAE67EAEEBA1
:108E8000E67ECBF8006626680434B4460E6A86FB9C
:108E90000C9C866AB1468E6886FB09A9966BCC4409
:108EA0000CEB86064FF0000C86EAE67CACEBE67C29
:108EB00048EA07073D432B4343EA0E0E009BCBF8DD
:108EC00080674EEA0C0C43EA0C030093029B0BF103
:108ED000800B5B458CD1089B0398DDF82C800A9AA7
:108EE0009B1040F8243C079B9B1040F8203C099BBA
:108EF0009B1040F81C3C0446A0F118031EA90BE08F
:108F0000A1EBD96E1D75A37B9A79825A83FB202130
:108F1000F0F4090051F8042F921043F8042B834217
:108F2000F8D1039A019D069B24320392029A0432DF
:108F3000029217EE901A2A4617EE100AFFF784FAEB
:108F4000009B03431846049B03430493409B2A461B
:108F50005B680132934208F1480801923FF724AE62
:108F6000409B019E9B68B34240F3E98024AB009490
:108F7000DDF80081049C059336AF0025D8E9032372
:108F8000DDF800B00599B342C8BF0022584600F092
:108F900045FF109B059946F3000A06F0010903EB13
:108FA0008600ABF1040E4FF0000C0A6892000260DC
:108FB000AB4682EAE27BABEBE27B4B688AEA830357
:108FC0004B441A434CEA020CC0F880302A4683EA2C
:108FD000E372A2EBE372083142EA0B028F424EF8D1
:108FE000045F44EA020400F58070DED1019AD8F8EB
:108FF0000830BCF1000F18BF32460192009A0136CA
:109000002432B3420092B9DC04941F2E0FDC109B73
:10901000002103EB8602002342F823102033B3F52E
:10902000107FF9D10136202E02F10402F3D1049B06
:10903000002B00F08280C0F2888004990023490050
:109040001A4603F10103FAD5409B0198DA6137B063
:10905000BDE8F08FDDF814900A9ADFF8FCB00DF14E
:1090600090084146484600F0D9FE069B00983849D2
:10907000099C03EBC30C374B002503EB0C1C1AAE09
:1090800044222B46AE4604E0376A5BF8041D56F8CE
:10909000044D81FB07A707EBA40149F8041BC7EBAC
:1090A000A4075CF8234087FB041458F823100C44F1
:1090B000A4005CF8021087FB01A158F802704FEA87
:1090C000C31A3944009F890047F80A407746C0F820
:1090D000801884EAE477A7EBE477744681EAE174C8
:1090E000A4EBE174043A2743202A45EA070503F17B
:1090F0000103A0F18000C7D121E50023069382E59A
:10910000079E3346483300200F9319461BAC024696
:109110008B689A1A4B680839101A8E42A3EB020228
:10912000206244F8042DF3D100230B93FFF7A0BB7A
:109130000023069D0A93FFF778BB1F2284E7019E58
:1091400063E70023049301931BE54FF0FF327BE7B5
:109150005CEB270BD0F309001CF108002DE9F04F60
:10916000D1F80031A3F11002102A85B00C468046D8
:1091700000F236810123934003F0013323F0807322
:10918000002B14BF0B46002307EE903A17EE902AEF
:1091900094F80401DFF850B24146FEF771FF94F8ED
:1091A0000431013BDBB2019308F10403039308F19E
:1091B00010030093C2469AF801009AF80D109AF82D
:1091C00009509AF805309AF802208AF805009AF8B2
:1091D00007009AF80A609AF806408AF80D508AF853
:1091E00009309AF80E509AF803308AF801108AF87C
:1091F0000A209AF80B109AF80F208AF803000398B7
:109200008AF80B208AF802608AF806508AF80E4025
:109210008AF807108AF80F3057465246002312F892
:1092200023101BF8011002F823100133042BF6D190
:1092300001329042F2D1019C17EE902A514620460D
:10924000FEF71EFF002C00F0C880CDF808A03A7889
:1092500097F80290797897F803E0D3094FEAD91686
:1092600003EB43034FEAD11C03EBC30306EB4606B3
:1092700083EA42034FEADE100CEB4C0C06EBC60609
:109280005FFA83FA86EA4906C3F3C0130CEBCC0CF1
:1092900000EB400082EA01088CEA410CC6F3C014DE
:1092A00082EA090203EB430300EBC00080EA4E00B0
:1092B000CCF3C01581EA09015FFA8CFC8EEA020248
:1092C00003EBC30304EB4404F6B283EA4A038EEAD9
:1092D00001018CEA020288EA0E0E04EBC40488EA5B
:1092E0000908C0F3C01984EA460486EA0E0E7240EB
:1092F00005EB4505C3F3C01609EB4909C0B205EB00
:10930000C5058AEA01018AEA080809EBC90906EBE2
:10931000460685EA4C0589EA400980EA0E0E8CEA89
:10932000010180EA080806EBC606D8B286EA4006C4
:10933000414080EA0E00C5F3C01E0EEB4E0EF3B2A4
:10934000EDB20EEBCE0EC4F3C0166A4085EA0808F3
:1093500006EB46068EEA45055FFA89FEC9F3C01999
:10936000E4B28EEA020206EBC60609EB4909EDB249
:10937000614060408EEA08085A4086EA440409EBDE
:10938000C909E4B283EA010C83EA080883EA000110
:1093900089EA4E0E85EA020385EA0C0C5FFA8EF22A
:1093A0006940634085EA0805534084EA0C0C61403B
:1093B0006C407B7082EA0C0C5140009B87F800C027
:1093C0006240B970FA700437BB427FF440AFDDE908
:1093D000013A581EC3B20193EDE605B0BDE8F08F27
:1093E000002307EE903AD1E65877090010B4D0F880
:1093F000C437D0F8C847D0F8BC2704FB03F302FBFE
:1094000003F3002B11DD00220239944621F802CF2C
:10941000D0F8C847D0F8C43704FB03F3D0F8BC47F2
:10942000013204FB03F39A42F0DB5DF8044B704712
:10943000012913DD821E02EB010C431EC0F1010164
:1094400001E063450AD0C81813F8012FFF2AF8D1AC
:109450005A7802F0E002E02AF3D170474FF0FF3073
:10946000704700BF10B54FF0804386B0D3F8044377
:10947000620703D5D3F80821002A62D1A30605D5D7
:109480004FF08043D3F81421002A4FD1600605D550
:109490004FF08043D3F81821002A3BD1210604D590
:1094A0004FF08043D3F81C214ABBE20504D54FF0AE
:1094B0008043D3F82021B2B9A30512D54FF08043E1
:1094C000D3F824216AB10022C3F82421D3F824213F
:1094D000214B0092009A1B68022006B0BDE81040A4
:1094E000184706B010BD0022C3F820211A4AD3F84D
:1094F0002031019301201368019A9847DCE700208E
:10950000C3F81C01144AD3F81C3102931368029A61
:109510009847CAE70022C3F81821104AD3F8183137
:10952000039301201368039A9847B7E70020C3F814
:1095300014010A4AD3F8143104931368049A984723
:10954000A4E70022C3F80821054AD3F8083105939F
:109550001368059A984791E70852012004520120A8
:1095600000520120064BD3F800213AB1054A0020F1
:109570005071C3F80001136891681847704700BF25
:1095800000900240E051012002480322002128F00F
:10959000E3BD00BF00B0004002480422012128F0D2
:1095A000DBBD00BF0010014002480422022128F068
:1095B000D3BD00BF004002409648974A904208B58C
:1095C00007D2013A121A22F00302944904322BF016
:1095D00091FE9348934A904207D2013A121A22F020
:1095E0000302043200212BF035FF4FF08053D3F8F3
:1095F0003021082A20D08C4AD2F8883043F47003F6
:10960000C2F88830BFF34F8FBFF36F8F4FF0102336
:10961000D3F80C22D20700F1DF80D3F80022002A11
:10962000C0F2B480D3F80432002BC0F2AF807F4B7D
:109630007F4A1A604FF098FC4FF080410020C1F83B
:109640000C017C4AC1F81001C1F83805D3F80414A4
:10965000C2F82015D3F80814C2F82415D3F80C1456
:10966000C2F82815D3F81014C2F82C15D3F8141426
:10967000C2F83015D3F81814C2F83415D3F81C14F6
:10968000C2F84015D3F82014C2F84415D3F82414B6
:10969000C2F84815D3F82814C2F84C15D3F82C1486
:1096A000C2F85015D3F83014C2F85415D3F8341456
:1096B000C2F86015D3F83814C2F86415D3F83C1416
:1096C000C2F86815D3F84014C2F86C15D3F83411F9
:1096D000D3F84434C2F87035032916D8564B5B5C76
:1096E0001BB1564B564AC3F88C26564B5B5C63B194
:1096F0004FF080535449D3F83021FB20C1F81805AE
:10970000082AD3F8343104D075E74FF08053D3F8EA
:109710003431032B20D94FF08053D3F83431032B4D
:109720000ED84A4AD35C5BB14FF08053484AD3F815
:1097300030314FF40071082BC2F840167FF45BAF54
:109740004FF08043D3F80024D1077FF554AF6FF07A
:109750000102C3F800244EE73E4AD35C002BDAD066
:109760004FF080524FF08040D2F85832D0F8E41ECB
:10977000D2F8304103F00F0321F00F010B43C0F882
:10978000E43E082CD2F83431C9D034E7324B012200
:10979000C3F80425D3F80024002AFBD04FF010238F
:1097A00012222D49C3F80022D1F80034002BFBD03F
:1097B0004FF010221221284BC2F80412D3F80024D3
:1097C000002AFBD000222449C3F80425D1F8003434
:1097D000002BFBD001F012F81F4B0122C3F8042527
:1097E000D3F80024002AFBD04FF010211A4AD1F8F8
:1097F0000C3223F00103C1F80C32D2F80034002BF4
:10980000FBD000231449C2F80435D1F80034002BF2
:10981000FBD0DFE70000012048050120BCFE090065
:1098200048050120CC5B012000ED00E00000012094
:109830000090D00300C0004018B80800005000405D
:109840004881030018B8080000F0004018B808006C
:109850000090024018B8080000E0014001490248A9
:1098600055F09AB9B85001200030004002494FF03D
:10987000402055F091B900BFEC500120084BD3F8BF
:10988000182102B97047002282B0C3F81821D3F81A
:1098900018310193019B034802B024F08FBD00BF33
:1098A0000030024058500120084BD3F8182102B96B
:1098B0007047002282B0C3F81821D3F81831019301
:1098C000019B034802B024F079BD00BF00F00240C4
:1098D0007C500120F0B52A4C83B00226002501A857
:1098E0004CF0CAFD05280BD0019B032B3DD02CD892
:1098F000022BF4D101A825704CF0BEFD0528F3D150
:10990000204D214F4FF40C760DF102012846ADF8A1
:1099100002604CF051FDA0B9D7F8E440002CF3D020
:1099200023462468D3E9011228469047002CF7D13A
:109930000DF102012846ADF802604CF03DFD002813
:10994000EAD00C2817D003B0F0BDA3F10902022A17
:10995000C5D80A2B0BD0092B0BD00B2B0CBF012029
:109960004FF0FF3054F09AFFB9E72670B7E70020B8
:10997000F8E70220F6E7054848F010FD03B0F0BD17
:10998000C15B0120284E01200C520120A477080061
:109990000149024828F0B8BBA050012000900040C7
:1099A0000149024828F0B0BBAC50012000A00040A3
:1099B0000149024855F01EBD205101200020004001
:1099C0000149024855F016BD445101200080024073
:1099D0002DE9F04FBA4A0023D2F8000387B002F510
:1099E00080721D4601261F4620FA03F1CC0709D5D7
:1099F000116806FA03F429B125431760BFF36F8F8E
:109A0000BFF34F8F0133192B02F10402ECD1E807A9
:109A100000F17C81AB4E290508D5A94BD3F8A836B7
:109A200001229BB286F8D720A6F8D230AA0213D51D
:109A3000A34CD4F81435DB0500F1AF81D4F8103510
:109A4000DF0540F1B28196F8D730002B40F0B681A7
:109A5000012103201CF0F2F968021FD5984BD3F8BE
:109A6000004404F4E062E105C3F8002400F18B81B6
:109A7000620510D5924B0122C3F808259A65D3F8E8
:109A8000002312F4001208BFC3F854218C4B4FF48A
:109A90000012C3F80423A30500F170812F0237D50B
:109AA000874BD3F880E4D3F88424D3F88814D3F810
:109AB0008C74D3F890445FFA81FCD3F89414D3F8F3
:109AC0009804D3F89C341EF07F0F5FFA8EF8D2B260
:109AD000FFB2E4B25FFA81F9C0B2DBB201D1052A6C
:109AE00016D08DF816008DF8173001214FF4C063A1
:109AF00003A88DF810808DF811208DF812C08DF814
:109B000013708DF814408DF8159003931CF0A6F98E
:109B10006D4B2B40002B40F0F180DFF8A8B14FF0E7
:109B200001085E46D946002412E0BEF80620A9F8D6
:109B30000420BEF8062092B21CF0C6FAB8F1090F54
:109B400041D008F1010801345FFA88F809F11809D9
:109B50005B4B04EB840203EB820204F10C0325FA55
:109B600003F304EB440706EBC7075FFA84FC13F02A
:109B7000010FBE464FF0010361464FF00000DDD0FB
:109B8000D2F808275FFA82FAD9F800205244C9F8BF
:109B90000020FA881AFA82F292B2082CFA801FFA90
:109BA0008AFAC2D0B9F808205245BED1FA88B9F86D
:109BB000047092B29742B8D9BCF1000FBED14348AD
:109BC00021F036F9BDE7424B2B40002B62D03C4BD5
:109BD000D3F86C94C3F86C94BFF36F8FBFF34F8FBF
:109BE00015F4806560D10195364FDFF8D4A00024CC
:109BF00006E0002C78D0B8F1070F29D001341837CF
:109C000004EB84030AEB830129FA04F304EB440216
:109C1000D80706EBC2025FFA84F8EAD5D1F8081635
:109C2000F868C9B20844F860538A11FA83F39BB20A
:109C30005382538A398A9BB2994240464FF00103BE
:109C400048F080014AD95AF091F8B8F1070FD5D100
:109C5000019F0024012507E0002C4CD0B8F1070F2C
:109C600018D001340BF1180B04EB440306EBC302CC
:109C700004F1100329FA03F3DB075FFA84F8EBD54C
:109C8000D388BBF804109BB2994230D8B8F1070FC3
:109C90009572E6D10F48104A0023C0E9002307B0AF
:109CA000BDE8F04F0AF0C8BCD3F88054D3F8803434
:109CB00083F08003C3F3C013C5F3C015019393E78A
:109CC00000700240581E0120FCFB1F004C70024037
:109CD0000004000130570120D5060800528A0020F8
:109CE00092B21CF0F1F986E7002D87D096E7404646
:109CF0005AF062F8B2E7002FB3D0C1E796F8D83037
:109D0000002B66D0002386F8D83006E7354B0121BA
:109D10000022C3F814151446C3F81015930003F17C
:109D2000804303F51C330132082A5C609C62F5D144
:109D30002C4B2D4E5C629C64C3F85841D3F8002430
:109D4000D3F800140A43C3F80024D3F80023C3F85F
:109D50000823264AC3F804230021DC2230462BF0D6
:109D600079FB40230121B382338103A80394CDE919
:109D700004448DF80D101CF071F84CE6012105200B
:109D80001CF05CF88AE60121C3F82C1504201CF0B5
:109D900055F862057FF57FAE6CE65AF03FF8D4F8CF
:109DA0001035DC053FF54FAE52E64FF40013C4F812
:109DB0000833012103201CF041F84DE6B6F8D2200B
:109DC0000020012392B286F8D70088211CF07CF98C
:109DD0003EE64FF0E023D3F8F03DDC077FF59DAE83
:109DE00000BE9AE600700240581E01200514C00112
:109DF00010B5084CD4F8003182B04BB1064B5B680B
:109E000098470023C4F80031D4F800310193019B36
:109E100002B010BD00000140D8510120022A2DE9F6
:109E2000F0411FD03C4B02EBC20C03EB0C1C0CF1BD
:109E3000480601F1440E0CF18C0C00F1240750F897
:109E4000043B5CF8044956F8045B1A4685FB028221
:109E500041F8042B84FB032387424EF80439EED1EA
:109E6000BDE8F08182682D4B83FB02422C4E846951
:109E700086FB045422440A602A4C426884FB025246
:109E8000294FC56987FB05C52A444A60026883FBE0
:109E90000252056A86FB05752A448A60234D0268D2
:109EA00085FB0262224E076A86FB07C73A44CA60F6
:109EB00042684FF0604C8CFB0272C7698CFB07E76D
:109EC0003A440A61826886FB0272876985FB07E76C
:109ED0003A444A61426983FB02728A61026984FBE7
:109EE0000272CA61C26883FB02420A62C36885FBD0
:109EF00003234B6203698CFB03238B62426986FB5D
:109F000002320023C1E91033C1E90E33C1E90C3339
:109F1000CA62BDE8F08100BFD0F30900D8E3CEB833
:109F2000281C310733C3BEB2CD3C410D9A615FC9D5
:109F3000669EA0F62DE9F04F90F8604095B0012C98
:109F4000069100F0D680022C45698346914600F0C8
:109F5000268190F86820436A002A40F01381C26C81
:109F6000BBF85E009BF86510C41DE410C0EBC40094
:109F700006294FEAC404C6B200F0E381C1F105012D
:109F8000C9B24FF4006088400C90402088400D908A
:109F9000012000FA01F10E91184600212BF05AFA27
:109FA00000EB860302939BF86230002B00F0D48014
:109FB000A200129209F1FF3292B2511C12B205F1C5
:109FC000180889000B929BF8667005910022CE4616
:109FD0000892C246D946002F00F0B580002299F8B9
:109FE00065300992F046D646CA46002B00F09F80A5
:109FF0009DF82420079208FB02F25200DDE90D14BF
:10A00000119200220F921092DDF830909DF82020DE
:10A010000A92019142469AF9675085EAE571A1EBEF
:10A02000E571013949B2481C6AD002980A9E85EA56
:10A03000E573A3EBE573DBB206FB031302FB03F34B
:10A04000069E07FB03F306EB8303CEB2C907049613
:10A0500002D5002DC0F28780119903EB010C07FB9C
:10A0600002F30CEB43034FF001080021002A38D023
:10A07000059D039346191FFA88F837463CF811B03E
:10A08000039B019D33F811601BEA090318BF5EF8BA
:10A09000183C1BEA050F1CBF5EF8145C2B431BEA3F
:10A0A000040F1CBF5EF8105C2B4316EA090F1CBF9F
:10A0B0005EF80C5C2B43019D2E421CBF5EF8085CD1
:10A0C0002B4326421CBF5EF8046C334350F8046BEC
:10A0D00041443343B84209B240F8043CCED19AF827
:10A0E0006670049B591E49B24B1C07D09AF9675001
:10A0F0009CE715B0BDE8F04F00F084B99AF86530E0
:10A10000019949000191109949BB052B27D90124D8
:10A110004FF400690F990298129D01310F91C9B255
:10A120002844994202901091FFF475AF9046099A25
:10A1300001320992D2B2BA42FFF457AFD146F24689
:10A1400099F86230C646089A01320892D2B2934218
:10A150000AF1180A3FF63FAF15B0BDE8F08F4FEA9D
:10A1600049096400D6E7079D791E491B02FB01F1EE
:10A1700003EB410307FB02FC0B9903EB4C0C4FF084
:10A18000FF3873E790F86A10DBF84C20C1F101004A
:10A19000B2FBF4F100FB01F103EB8103E0E690F880
:10A1A0006820436A002A40F02181C26CBBF85E003F
:10A1B0009BF86510C41DE410C0EBC40006294FEAEB
:10A1C000C404C6B200F00A81C1F10501C9B24FF45E
:10A1D000006088400890402088400990012000FAE3
:10A1E00001F10A91184600212BF034F99BF86230F6
:10A1F00000EB460C002BAFD06200109209F1FF3249
:10A2000092B213920132520005F10C0A4FF000088D
:10A2100012924A469BF86670C146D046DA46E3463B
:10A220009446002F00F0BA80002307939AF8652027
:10A23000BDF94C3005935D46CDF80490002A00F03E
:10A24000A1809DF81C300493DDE909190CFB03F390
:10A250005B000F93DDF820E0029100230B930E9337
:10A26000AB469AF9670080EAE073A3EBE073013B29
:10A270005BB25C1C6FD09DF8042003925C4680EAC0
:10A28000E0720399A2EBE072D2B201FB02320CFB46
:10A2900002F2069907FB02F201EB8202D9B2119198
:10A2A000D90702D50028C0F285800F9BD11807FB83
:10A2B0000CF201EB420201230020BCF1000F38D068
:10A2C0009BB20D93129BE3180C9331F81050029F30
:10A2D00032F8106015EA0E0318BF38F80C3C3D4206
:10A2E0001CBF38F80A7C3B4315EA090F1CBF38F83D
:10A2F000085C2B4316EA0E0F1CBF38F8065C2B4394
:10A30000029D2E421CBF38F8045C2B4316EA090F4D
:10A310001CBF38F8025C2B430D9D284434F8025BC7
:10A320002B4324F8023C0C9B9C4200B2CDD19AF8FE
:10A330006670119B013B5BB25A1C0AD09AF9670008
:10A340009DE720211027CDE90D174FF400410C9116
:10A3500022E69AF86520029B5B0002930E9B002B7D
:10A3600037D1052A35D94FF001094FF4006E0B9B08
:10A37000109901330B93DBB293428B440E93FFF49D
:10A3800070AF5D46079B01330793DBB2BB42FFF41E
:10A3900055AFDDF804909AF86230AB4609F1010937
:10A3A0005FFA89F2934208F10C083FF63AAF15B014
:10A3B000BDE8F08F049905987B1E5B1A0CFB03F334
:10A3C00002EB430207FB0CF102EB41014FF0FF33BC
:10A3D00073E74FEA4E0E4FEA4909C8E720211027DC
:10A3E000CDE909174FF400410891FBE6C26C90F8E3
:10A3F0006A10C1F10100510800FB01F103EB4103B8
:10A40000D4E600BF2DE9F04F034691B0D0F8149088
:10A4100001921A4693F8683003900491406A33B170
:10A4200092F86A30D26CC3F1010302FB0300039B74
:10A43000B3F85E2093F86510D31DDB10C2EBC302A6
:10A4400050FA82F2DB00062906920B9300F0C280DC
:10A45000C1F10503DBB24FF400629A400D92402235
:10A460009A400E92012202FA03F30F93039B93F892
:10A470006630002B00F09880019A013A12B20A92DD
:10A4800000220C92002900F088809DF8302001986D
:10A490000992DDE90E6800FB02F2520005920D9D63
:10A4A000002207920892B646039A92F96720002A82
:10A4B000B8BF5242013A52B2541C59D0069C01997D
:10A4C000049801FB02F603FB06F600EB8606D0B209
:10A4D0000290D00704D5039A92F96720002A66DB20
:10A4E000059A1644019A03FB02F706EB47074FF063
:10A4F000010C0022019999B31FFA8CFC04EB010AAC
:10A5000036F8121037F8120011EA050318BF99F84F
:10A51000003011EA0E0F1CBF99F801B043EA0B039B
:10A5200011EA080F1CBF99F802100B4328421CBF08
:10A5300099F803100B4310EA0E0F1CBF99F8041092
:10A540000B4310EA080F1CBF99F805100B4304F8E1
:10A55000013B6244544512B2D2D1039B93F866305A
:10A56000029A013A52B2511CA9D1039A92F865108D
:10A57000089A4FEA4E0E4ABB052927D94FF0010829
:10A580004FF40065079A06980B9C01320792D2B2ED
:10A5900020448A420690089286D30C9A01320C928B
:10A5A000D2B29A42FFF46EAF11B0BDE8F08F099AB3
:10A5B0005F1EBF1A01FB07F706EB470703FB01F617
:10A5C0000A9A07EB46064FF0FF3C93E76D004FEA0F
:10A5D0004808D7E720231025CDE90E354FF4004376
:10A5E0000D9343E790F8661090F865304A1E013BE2
:10A5F000DBB2D2B280F86B30012980F86C2088BFC2
:10A6000090F86C3090F8631088BF03F1FF334FF07F
:10A6100000028CBFDBB2012380F86D3070B580F88A
:10A620006E20826500293FD0944601223B4D63464F
:10A6300040F20334964614E01F2B86BF03F01F033D
:10A6400029464FF0A0410EFA03F3C1F8083590F8FF
:10A6500063100CF1010C5FFA8CF352009942D2B2F4
:10A6600022D9816C1E0101EB03131B7B1F2B86BFBC
:10A6700003F01F0329464FF0A04103F5E07341F8B2
:10A68000234090F86D301342836C33441B7BD3D14D
:10A690001F2B86BF03F01F0329464FF0A0410EFA7F
:10A6A00003F3C1F80C35D2E703681D4A934208BF93
:10A6B00008241AD01B4A934216D002F580529342C6
:10A6C00027D002F58032934225D002F58052934282
:10A6D00008BF1B2409D001224FF47A715A60DA6056
:10A6E000C3F840151A6070BD092401210022596089
:10A6F00001FA04F4C3F80425D9604FF48031C3F89B
:10A700000825C3F81025C3F80413074B1C60036821
:10A71000E1E70A24E9E71A24E7E700BF0003005055
:10A72000008000400090004000E100E030B490F86C
:10A730006E20002AFBD102F0FF030268012454605E
:10A740001464816BD2F84025026C0A6090F8622094
:10A75000B2B1234D0269D25C1F2A29468CBF02F098
:10A760001F024FF0A04104FA02F2C1F80C2590F844
:10A7700062200133DBB202EB4202B3EB420FE9DBB2
:10A78000B0F85E3023B3164C00224FF0010C90F865
:10A7900061301F2B21468CBF03F01F034FF0A041F7
:10A7A0000CFA03F3C1F8083500BF00BF90F8613020
:10A7B0001F2B21468CBF03F01F034FF0A0410CFA62
:10A7C00003F3C1F80C35B0F85E3001329A42DED3A3
:10A7D000826A036B1360C26A136030BC704700BFAB
:10A7E0000003005090F8683033B1012380F86E30D8
:10A7F00090F86E30002BFBD1704700BFBFF34F8F36
:10A800000549064BCA6802F4E0621343CB60BFF30C
:10A810004F8F00BFFDE700BF00ED00E00400FA0528
:10A8200070B510EE106A26F000450123B5F1FF4F18
:10A83000B0EE402A036020DAB5B1B5F1E45F04461A
:10A840000DDA002EBEBF4FF0FF330360B1EE400AB9
:10A850002AF056F8B1EE402AB0EE420A70BD002E42
:10A8600010DAB5F1964F65DBDFEDD17AB7EE007AFD
:10A8700087EE272AB0EE420A70BD20EE002AB0EE25
:10A88000420A70BDB5F17E5F51D0B5F1804F4ED018
:10A89000DFEDC71A730073D4C64B9D4240F3248288
:10A8A000C54B9D4240F3CE81B0EE007A37EE427A3E
:10A8B0009FEDBF0ADFEDC16A9FEDC16A9FEDC15AEE
:10A8C000DFEDC15A9FEDC12A67EE077AA7EEA66AAF
:10A8D000E7EE855ADFEDBE6A9FEDBE5AE6EE276AC7
:10A8E000A5EEA75A9FEDBC6ADFEDBC5AA6EEA76A9B
:10A8F000E5EE275ADFEDBA6AE6EE276A9FEDB96A00
:10A90000A5EEA76AA6EEA72ADFEDB76AE6EE276AEC
:10A9100022EE072AF6EE005AA6EEA72AA7EE652A2F
:10A9200032EE002A002E97DA31EEC22A94E79FED2C
:10A93000A02A91E7B5F17A5FC0F2E481B1EE407AE6
:10A94000B0EE470A24F0DEF9B4EE407AF1EE10FAE8
:10A9500040F0E880DFEDA57A77EEC27A17EE903A04
:10A9600003F0010307EE903AF8EEE77A9B00062B1E
:10A9700000F22782DFE803F0588B8B54549A9A0038
:10A98000B5F1824F80F2E180BDEEC27ADFED986AC8
:10A990009FED986A9FED985ADFED985AF8EEC77AC6
:10A9A00017EE103A72EE677A033BA7EEA66AE7EE5F
:10A9B000855ADFED936A9FED935AE6EE276AA5EE7E
:10A9C000A75A9FED916ADFED915AA6EEA76AE5EED0
:10A9D000275ADFED8F6A9FED8F5AE6EE276AA5EEC4
:10A9E000A75A9FED8D6ADFED8D5AA6EEA76AE5EEB8
:10A9F000275ADFED8B6AE6EE276AB7EE006AA5EE0E
:10AA0000A76A66EEA76AB6EE005A86EE862AA7EE19
:10AA1000852A042B86D8DFE803F06B587D6E800012
:10AA2000B7EE007A77EE677A9FED7E0ADFED600A77
:10AA300027EE800A002000F021FEF1EE401AF5EE2C
:10AA4000401AF1EE10FA3FF40FAF62EE217A9FED5B
:10AA5000750AF0EEE77A80EE270A29F051FFF5EE4D
:10AA6000C01AF1EE10FA4CBF4FF0FF330123B5F1DD
:10AA70007E5F2360F0EE401A00F05981B5F1804FFF
:10AA8000B1EE422A7FF406AF9FED492A4CE7B6EEBD
:10AA9000007A77EE677A9FED630ADFED450A27EECD
:10AAA000800A00F009FBF1EE401AC8E7B7EE087A19
:10AAB00077EEC77A9FED5B0ADFED3D0A27EE800A4D
:10AAC00000F0FAFAF0EE401AB9E7B7EE007AB0EE0D
:10AAD000080A37EE800A20EE070AB0EE007A77EE19
:10AAE000877A27EE800A29F00BFF32EE002A19E759
:10AAF000B7EE000AF1E7B7EE000AB1EE047A37EEDE
:10AB0000877A27EE000AB1EE007A37EE877A27EED1
:10AB1000007ADCE7B7EE000AF5E7B1EE080A37EE97
:10AB2000800AEAE7F6EE007A27EE277AB0EE470AC7
:10AB300024F0E8F837EE400A70EE007AB0EE677A5B
:10AB4000BEEECF7A17EE103A11E7B5F1B94FB0EE7D
:10AB5000420A80F2E38029F0D3FEF7EE007A87EE16
:10AB6000826A30EE670A9FED303ADFED303A9FEDB2
:10AB7000304ADFED304A9FED305ADFED305A9FED1D
:10AB8000307A66EE067AF6EE006AE7EE833A72EE07
:10AB9000666AA3EEA74AE4EE274AA4EEA75AE5EEBA
:10ABA000275AA5EE867AB0EE472AA6EE802AB9E6A5
:10ABB000000000006666663F17A6DD3FA283D3371C
:10ABC00067976739752C3C384584E2383F239E3DB2
:10ABD000A1549C3A34B6053A7E02F23BC66E3D3B28
:10ABE00001F0893D1599A83C661AA53E0000004B6E
:10ABF00067FF0538B435F13ABDD7F536D6EE4B3A96
:10AC0000E440DA3C54BF983CE6DC153E6E0F303E23
:10AC10007ACCA63EC5D0383F5A245C3E3B2DB23F8D
:10AC20003F239EBDDB0F4940E8C4D5BAD23D5B3A15
:10AC30005C061CBAFD0C503A610B36BBABAAAA3DB0
:10AC40001D7FD63E614B9D4274DDDFED617A9FED45
:10AC5000610A32EE672A22EE024ADFED5F5A9FED6B
:10AC60005F7A9FED5F6ADFED5F6A9FED5F5ADFED10
:10AC70005F4A64EE027AA7EEA56AE7EE876ADFED27
:10AC80005C5A9FED5C7AE6EE275AA6EEA77A9FED16
:10AC90005A6ADFED5A6AA5EEA76AE7EE276AE7EE81
:10ACA000854A9FED577A9FED575ADFED575AA6EE2A
:10ACB000277AE6EEA75AA4EEA75A9FED546ADFED75
:10ACC000546AA5EE827AA5EE276A9FED522ADFED3F
:10ACD000525AE6EE276AA7EE672A94EE262A32EE4B
:10ACE000652A32EE002A1DE6B0EE420A29F008FE7F
:10ACF0004A4B9D42B1EE400A5BDDB7EE007A37EE7B
:10AD0000427AD7E59FED460ADFED320A22EE000ACD
:10AD1000002000F0B3FCF0EE401A90E629F0F0FDC0
:10AD2000F7EE007A30EE670A20EE022AFAE5B0EE7E
:10AD3000402A91E5F7EE007A32EE672A9FED250A68
:10AD4000DFED386ADFED387A9FED387A9FED386AAB
:10AD5000E2EE267AA2EE076ADFED366A9FED367ADA
:10AD6000E7EE826AA6EE027ADFED347A9FED346A6E
:10AD7000E6EE827AA7EE026ADFED326A9FED327A62
:10AD8000E7EE826AA6EE027ADFED307AE6EE827AAC
:10AD9000F7EE006AE7EE026A67EE827ABEEE006ABC
:10ADA00087EEA67AF0EE477AE2EE067A37EE802A50
:10ADB000B8E5274B9D42C3DDDFED267A32EE672AE8
:10ADC00049E7B0EE007A77EEC77A2DE61FA69D3FE1
:10ADD000C316BB3F0000000027F9A3B9F7E9AF395C
:10ADE00067F8663A85300DBA6B7BA53976F4B7BA49
:10ADF000FE7771BB9916143B3D37933CFEFC28BC93
:10AE00003C2117BE07E7C73B155A843D474D06BD99
:10AE10005EB9F73E521CE631CDCDF83D1F4A3B3FAF
:10AE2000DB0F49405E3C5B3C78756A3EDBD5523BAC
:10AE3000AF72D53DB24B7A3FDFEF443FE73ABA3FBE
:10AE40002D390840F400223FBE2E1D403F239EBDF9
:10AE500007336D3E0C5BEC3E30B510EE103A894A7C
:10AE600023F0004C944585B0044664DD864A944541
:10AE700010EE105A22DC002BDFED847A844A2CF08D
:10AE80000F0CB0EE407A40F3E380944570EE677AA1
:10AE900009BFDFED806A9FED807A9FED807A77EEC3
:10AEA000E67A012077EEC76A77EEE67AC4ED006AAB
:10AEB00077EEC77AC4ED017A05B030BD784A944583
:10AEC00040DCDFED786ADFED715AF0EEC07AB6EE65
:10AED000007AA7EEA67ADFED706ABDEEC77A17EEAC
:10AEE000100AB8EEC76A1F28E6EE657A26EE267AC3
:10AEF000F1EE465A68DC6C4A411E23F0004352F8DA
:10AF0000212023F0FF0393425ED077EEC76AC4EDA1
:10AF1000006A77EEE67A002D77EEC77AC4ED017A03
:10AF2000CADAF1EE666AF1EE677AC4ED006AC4ED42
:10AF3000017A4042C0E7002284ED000A426000200E
:10AF400005B030BDBCF1FF4F73DA4FEAEC52863AE0
:10AF5000ACEBC25307EE903ABDEEE77ADFED536AF1
:10AF6000B8EEC77A77EEC77A8DED017A67EEA67AEA
:10AF7000BDEEE77AB8EEC77A77EEC77A8DED027A42
:10AF800067EEA67AF5EE407AF1EE10FACDED037A8F
:10AF90005CD1B5EE407AF1EE10FA14BF0223012322
:10AFA000214601A800F00AF9002D85DA94ED007A17
:10AFB000D4ED017AB1EE477AF1EE677A84ED007A4A
:10AFC000C4ED017A404277E777EEC76A4FEAEC5268
:10AFD00016EE903AC3F3C753C3EBDC5CBCF1080F29
:10AFE00095DD9FED2C7ADFED2D6AB0EE675AA5EE68
:10AFF000875A77EEC57AE5EE877AD6EE267A75EE31
:10B00000676AB0EE677A16EE903AC3F3C753D21A66
:10B01000192A16DDDFED266ADFED264AF0EE457AC5
:10B02000E5EEA67A35EE677AA5EEA67A96EE247A54
:10B030006BE770EE407A0020C4ED017AC4ED007A2F
:10B040003AE7F0EE457AC4ED006A62E70323A7E72A
:10B05000944570EE277A09BFDFED0E6A9FED0E7AF8
:10B060009FED0E7A77EEA67A4FF0FF3077EE876A83
:10B0700077EEE67AC4ED006A77EE877AC4ED017A5E
:10B080001AE700BFD80F493FE3CB1640800FC93FF6
:10B09000D00FC93F004435374344353708A3852EC8
:10B0A000800F494384F9223F9066090000008043E5
:10B0B00000A3852E32318D2410EE103A23F0004388
:10B0C000B3F1485F2CDAFDEEC07A17EE903A002B10
:10B0D00060D020EE007ADFED317A9FED315ADFED5E
:10B0E000315A9FED316ADFED316AA7EE275ADFED65
:10B0F000307AE7EE055AA7EE256AE7EE067AE7EE24
:10B10000276A67EE266A60EEC00AF6EE007AE7EE7E
:10B11000260AB7EE000AD7EE270A30EE600A70471B
:10B1200020EE007ADFED1D7A9FED1D5ADFED1D5AEE
:10B130009FED1D6ADFED1D6A1E4AA7EE275A934256
:10B14000DFED1B7AE5EE075AA5EE876AE6EE077A91
:10B15000E7EE876A66EE876AD5DD174A934214DC0C
:10B1600003F17F4307EE903AB7EE006A36EE676A66
:10B1700060EEC00AF6EE005AD7EE257AE7EE260A10
:10B1800077EEE00A36EE600A7047B6EE076AF5EE33
:10B19000027AEDE7B7EE000A704700BF4ED747AD21
:10B1A000F6740F317CF293B4010DD037ABAA2A3D6F
:10B1B000610BB6BA9999993E0000483F2DE9F04FCE
:10B1C000D61E48BF161DD5B0F61006F1010B02922F
:10B1D00001914FEACB0182460391581E02999FEDDF
:10B1E000B47AB44F321A03F10905A1EBCB0B541911
:10B1F00018A9002AA4BF12F807C007EE90CA02F1EE
:10B200000102ACBFF8EE677AF0EE477AA242E1ECB9
:10B21000017AEED118AA0DF5807C02EB83070AEBC8
:10B220008304DFEDA37A39465246F2EC016A31ED30
:10B23000017A9442E6EE877AF7D101308542ECEC50
:10B24000017A07F10407ECD16FF040473B44DFED92
:10B250009A5A9FED9A6A0093B4EE004AF2EE004AC1
:10B26000F7EE003A4FF0090909EB070854AB03EB7E
:10B2700089034FEA880813ED140A08F1040240AB71
:10B280001A4404A94D4660EE257AB0EE407AFDEEF0
:10B29000E77A72ED016AF8EEE77A013DA7EEC67A29
:10B2A00037EEA60ABDEEC77AA1EC017AEBD158467B
:10B2B0004AF010FEB0EE407A20EE040A23F022FDA0
:10B2C000A0EE647ABBF1000FBDEEC75AF8EEC57A66
:10B2D00037EE677A69DD09F1FF3C04ABCBF1080179
:10B2E00053F82C0040FA01FE04AA0EFA01F1411AAB
:10B2F00042F82C1015EE102ACBF10703724405EE2C
:10B30000102A41FA03F2002A59DCB5EE407AF1EE38
:10B3100010FA40F09080B9F1090F09F1FF3100F007
:10B32000538104AB98440DF1300C002358F8040904
:10B33000C44543EA0003F9D1002B40F051810C9B36
:10B34000002B40F049810BAA012352F80419013364
:10B350000029FAD009F101009944564B06EB000C84
:10B360009C44009B191818AB03EB810140AB03EB25
:10B37000800E1CF8013B9FED4E7A07EE903AF8EEF6
:10B38000677A0A46C1ED007A5346043101E072ED56
:10B39000017AF3EC016AA342A6EEA77AF7D1013055
:10B3A0004845AEEC017AE4DD5EE740F0FF8009F14C
:10B3B000FF3304AA52F823201212002AA5DD15EE4D
:10B3C000103A013305EE103A049B002B40F0F78051
:10B3D00004A8012350F8041F002940F0CE80013357
:10B3E0009945F7D1BBF1000F10DDBBF1010F00F063
:10B3F0001B81BBF1020F09D109F1FF3004AB04AD91
:10B4000053F8203003F03F0345F82030022A7FF440
:10B410007CAF33EEC77A00293FF477AFB7EE000A6E
:10B4200058464AF057FD37EE407AB5EE407AF1EED5
:10B4300010FA3FF470AFDDE90213B0EE470A581A74
:10B440004AF048FD9FED1D7AB4EEC70AF1EE10FAFE
:10B45000C0F2F780DFED187A60EE277A04A8FDEEDF
:10B46000E77A09F10101F8EEE77A0BF1080BA7EE94
:10B47000C70AFDEEE77ABDEEC00A17EE904A10EE5D
:10B48000103A40F8293040F821405846B7EE000AFB
:10B490004AF020FD40AB4FEA810E03EB8106AEF18E
:10B4A000040504AB1D449FED047A301D0B4609E0F2
:10B4B00000000000C88F09000000803B00008043AE
:10B4C00055F8044907EE904AF8EEE77A013B67EE3B
:10B4D000807A5C1C20EE070A60ED017AF0D10DF154
:10B4E000B00C0F460025634CDFED637A3046002335
:10B4F000AB4203F1010307DCF4EC016AB0EC017A22
:10B500000A2BE6EE877AF3D1013F7B1CECEC017A43
:10B5100005F10105A6F10406E5D12CAB0EF10400FE
:10B52000DFED557A18440B4630ED017A013B5C1C87
:10B5300077EE877AF8D19DED2C7A002A40F08F8043
:10B54000019B0029C3ED007A77EE677A0BDD2DA809
:10B550000123B0EC017A01338B4277EE877AF8DD74
:10B560000AB1F1EE677A019BC3ED017A15EE103A4C
:10B5700003F0070055B0BDE8F08F04A8C1F5807155
:10B5800040F82310013399450EDD04A904A851F8B1
:10B59000231000EB830000E001680133C1F1FF01DB
:10B5A000994540F8041BF7DC01211BE7F6EE007A11
:10B5B000B4EEE77AF1EE10FA41DA2A46A5E6C3F5D1
:10B5C000807304930123E0E70C9B002B3FF4BBAE98
:10B5D0004FF00A094846C0E609F101094846BCE6B1
:10B5E00004ABABF1080B53F82140002C7FF44DAFB6
:10B5F00009F18043023B04A800EB830353F804499C
:10B600000139ABF1080B002CF8D05846B7EE000A10
:10B610004AF060FC0029BFF63DAFDFED177A9DEDE3
:10B620002C7A002A8CD01AE009F1FF3004AB04AD6B
:10B6300053F8203003F07F0345F82030E6E602227D
:10B64000BDE6FDEEC07A04AB17EE904A584643F8CB
:10B650002940B7EE000A49464AF03CFC1AE7019B34
:10B66000F1EE676A002977EE677AC3ED006A3FF76B
:10B670006EAF76E700B908000000000010EE103A47
:10B6800023F00043B3F1485F04DAFDEEC07A17EE11
:10B69000903A5BB360EE007A9FED157ADFED155AB4
:10B6A0009FED156ADFED156AE7EE875A9FED147A74
:10B6B000A5EEA76A20EE275AE6EE276AA6EEA77A3D
:10B6C00030B9DFED106AE7EE876AA6EE850A7047AB
:10B6D00027EE457AF6EE006AA0EEA67ADFED0A6A5A
:10B6E000D7EE270AE5EE260A30EE600A704700BF63
:10B6F000D3C92E2F342FD7B21BEF3836010D50B9D6
:10B700008988083CABAA2ABEABAA2A3E10EE103AA2
:10B7100023F00042B2F1465F10DAFDEEC07A17EE78
:10B72000901A01BB431C134300F0A280012800F0D3
:10B73000A880BFEE007AC7EE007A76E052498A42CE
:10B7400011DBDFED527A9FED527A002BBCBFF1EE98
:10B75000600AB1EE400A37EEC00A77EE607ADFED9C
:10B760004D0A37EE800A20EE007A9FED4B5A9FED8E
:10B770004B6ADFED4B5ADFED4B6A434967EE077AC0
:10B780008A42A7EE856AE7EEA56A9FED475ADFED8C
:10B79000475AA6EE275AE6EEA75A9FED456ADFED17
:10B7A000456AA5EE276AE5EEA76A9FED435ADFEDED
:10B7B000435AA6EE275AE6EEA75ADFED416A9FEDFF
:10B7C000416AE5EE276AA5EEA76AF0EE667AE6EE34
:10B7D000077A60EE075AF0EE606AE7EEA56A9FED21
:10B7E0003A5AE6EE870AE5EE850A70EE207A1FDA0D
:10B7F00001281AD0BFEE007AC7EE276A334B17EE46
:10B80000902A1A4006EE102A16EE902A134007EEF0
:10B81000903AB7EE007AA6EE277A36EE400A70EE3E
:10B82000C00AA0EEA77AE7EE267AB0EE670A704764
:10B8300007EE100AB8EEC77A67EEA75A77EE877A56
:10B840009B17C5EEA76A03F00203C3F10103B0EE34
:10B85000006A76EEE00A07EE903A30EE600AF8EE03
:10B86000E77AA0EE467A67EE877AB0EE670A70470D
:10B87000B0EEC00AB7EE007AC7EE007AB0EE670A03
:10B880007047F0EE407AD0E740A12C3FDA0F493FF5
:10B8900068212233000000005FAE9BB745F4A33857
:10B8A0008453D9377AC09538C8261A3AB9378139BE
:10B8B00016696B3B48DEBE3AA427B33C1F37113CE8
:10B8C0008988083ED10D5D3DABAAAA3E00F0FFFF7E
:10B8D00070B504464FF491600D4634F0DDFA50B176
:10B8E000D0E9013228469568984704F108012B46B3
:10B8F000BDE87040184729462046BDE8704000F07A
:10B9000001B800BF70B50E460546264930462FF0F7
:10B910001DFC08B390F85030D9063CD443F0100316
:10B9200080F8503005F108011FF054F995F82A30DD
:10B9300090F8512003F00C03002B14BF01230023C7
:10B9400063F3410280F8512005D190F8503043F064
:10B95000020380F8503070BD134930462FF0F6FBDB
:10B960000446D8B190F82A309A0714D443F0020361
:10B9700005F1080180F82A301EF092FB95F82A3074
:10B9800013F00C0F204618BF0121BDE8704008BF1E
:10B9900000211EF03BBB054834F08CFB044834F01A
:10B9A00089FB00BF280609000002090058B60900FB
:10B9B00044B60900F0B50C4685B0002307466A4638
:10B9C00001A92046019331F0AFFC019B022B54D911
:10B9D0003A89B2EB430F4FEA43012FD33981002458
:10B9E0002246009B53F822506B68022B4FEA8206D6
:10B9F0003ED1A86803A930F05BFB00282ED0E86890
:10BA000002A930F055FB48B3039A02F50043B3F5A1
:10BA1000803F23D2029B03F50043B3F5803F1DD244
:10BA20007B689A537B680299334401345980019BA7
:10BA3000A4B29C422246D4D305B0F0BD786810B1C0
:10BA400024F012FD019B9800002124F011F9019BC4
:10BA500078605A003A81002BC1D1EDE7786824F074
:10BA600003FD002306487B6040F2764134F02AFB58
:10BA7000044840F2764134F025FB034834F006FBDD
:10BA8000CCA40900D8C10900DCB209002DE9F04FAF
:10BA90002DED028B93468DB0C268BDF86490DDF841
:10BAA0006880BDF86C701D9E04468A461D46B0EE47
:10BAB000408A2AB143689A4200F0B6800FF06CFFCA
:10BAC000B9F11F0F5BD9BAF1000F00F08380002697
:10BAD0004FF0060ABBF1000F74D040F201230DF1C4
:10BAE000180BADF818306B1CADF81A30584600230F
:10BAF00007934AF087FC00283CD19FED4F0ADFED09
:10BB00004F6A189B029328EE000A4D4B0690C0EE38
:10BB1000267A03FB05F54B4BCBF81400002FA3FB53
:10BB20000535CBE90100CBE9030008BF4FF0000861
:10BB30000796B6EE007A77EE877A6D0BFCEEE77A21
:10BB40000126ADF80C90ADF81470CDF810808DF88A
:10BB500018A0CDED087AADF824508DF82D6002F0D4
:10BB60006DF938B9384D5A4602A928464AF02AFCE0
:10BB700000283FD00DB0BDEC028BBDE8F08F1F2F29
:10BB8000A1D8BAF1000F2DD0002E4AD0F0EE0C7AD9
:10BB9000B4EEE78AF1EE10FA304669460AD807EEAD
:10BBA000905A9FED2A7AF8EE677AF4EEC77AF1EEB2
:10BBB00010FA3BD900F07AFC6E464FF0030ABBF155
:10BBC000000F8AD1CDE906BB0DF1180B58464AF09B
:10BBD00019FC90E7002F564614BF4FF0080A4FF0AB
:10BBE0000A0A77E7002F564614BF4FF0040A4FF0B9
:10BBF000050A6FE71649224604F1280009F002FF02
:10BC00001C9B29785AB230464AF006FC0028B1D174
:10BC1000287831464AF0D8FB0028ABD1189BE36066
:10BC2000A8E74FF0010A55E71120A3E700F03EFC1A
:10BC30006E464FF0020A4DE70024744900401C4450
:10BC400040420F005917B7D1450501206666A63F4F
:10BC5000B5E502002DE9F8434160044648680A9DB5
:10BC6000807984F82800A5848E7DDDF82C809946A3
:10BC700006F0300706F00605002831D14FF6FF73B5
:10BC80006384E7B1089BA361099B84F82900C4E998
:10BC90000229C4E9040084F826002084E361B8F195
:10BCA000000F18D030492246404609F0ABFE25B1BE
:10BCB00073073DD4022384F82730BDE8F883089B3E
:10BCC000A361099B84F8297084F826702784E361B6
:10BCD000B8F1000FE6D12448214609F075FEE6E7E9
:10BCE0004B68D8680AF064FD608435BB089BA3618B
:10BCF000099B84F8295084F826502584E361B8F123
:10BD0000000F2BD019494046224609F07BFE5DB159
:10BD100015F0040118BF012160681ABF84F82710CC
:10BD2000002201220FF0CCFF002FC6D0B206C1D4F2
:10BD3000012384F82730BDE8F883089BA361099BA1
:10BD4000E3610023C4E90229C4E9043384F82930FB
:10BD500084F826302384B8F1000FD3D1034821465C
:10BD600009F032FED3E700BF3DF30600C9F206003A
:10BD700030B504464FF6FF70A080002083B0A1606C
:10BD8000E2712361A071E060824288888B79ADF80E
:10BD9000040004F1040201A90CBF012002208DF867
:10BDA00006304AF051FB054610B1284603B030BDBD
:10BDB000A188084600F054FC284603B030BD00BFFF
:10BDC0002DE9F04F89B016469DF84820002B4AD047
:10BDD0005FFA81F84168DFF8A8A0002A0A790968AB
:10BDE00081464FF0340000FB02A24FF00600C1F87C
:10BDF00000054FF002011D4682F82D1014BF0023EC
:10BE000020234FF6FF7B00275D452C4628BF5C466C
:10BE1000CDE90447D9F804200696079710798DF8E4
:10BE20000C708DF80D801168019300EB400200EB5F
:10BE300082000AEB800003AA52F070FF0F4B984279
:10BE4000264402D12D1B019BDED1D9F8043001908C
:10BE5000197918683FF094FE019A104609B0BDE8C0
:10BE6000F04F52F07BBEC9B210F034FC002814BF72
:10BE70000020132009B0BDE8F08F00BF0000AD0B1B
:10BE8000B85001202DE9F04F85B007460C460292CC
:10BE9000002A40F0198201F10C053B78D4F800A08B
:10BEA0003846002B76D00AF102024FF00008AA189B
:10BEB00003925646CDF80480292B5AD05E2B00F20F
:10BEC000C381232B3FD9243B3A2B3CD8DFE813F026
:10BED000A6013B003B003B005E013B00B00091002F
:10BEE0003B003B0007013B003B003B003B003B00AD
:10BEF0003B003B003B003B003B003B003B003B006A
:10BF00003B003B003B00E4003B003B003B003B00B0
:10BF10003B003B003B003B003B003B003B003B0049
:10BF20003B003B003B003B003B003B003B003B0039
:10BF30003B003B003B003B003B003B003B00100153
:10BF40006F003B0065002668002D00F05282731CD4
:10BF500023604FF00103AB5523685A1C22603A78E6
:10BF6000EA5439466368013363604B784F1C002BF9
:10BF7000A2D10199384649B123685B1A013B5AB2F4
:10BF80009A4218BF48F0010805B16B54B8F1000F90
:10BF900040F0928105B0BDE8F08F002D00F0908157
:10BFA00023685022591C2160EA542668D9E77B781F
:10BFB000791C002B00F0808143F02002642A26685F
:10BFC00000F0358123F0040343F02003732B00F0CD
:10BFD0002E81002D00F0B381731C23604FF001030C
:10BFE000AB55787827687B1C236053F0F7FAE85547
:10BFF000B8E72268B24200F05F817B783F2B00F007
:10C00000F381002D00F00F8239466223AB54236880
:10C01000F61A0133023EEE5472B2B24218BF48F033
:10C02000010822686368961C0133266063609CE700
:10C030002268B24200F04081002D00F06781B01C00
:10C04000921BA919284429F085F92368023360223C
:10C050002360EA542368F21A2B44023A5A70236888
:10C06000023323607B7851B2914218BF48F0010837
:10C070003F2B00F0CB8139466123AB552368721CFE
:10C080009E1B023E73B2AE54B34218BF48F0010883
:10C090005FFA88F826680BE12268B24200F00C8152
:10C0A000002D00F02381B01C921B2844A91929F00F
:10C0B00051F92368023323607B783F2B00F0DD8148
:10C0C00039466123AB552368721C9E1B023EAE5459
:10C0D00073B2B34218BF48F00108266842E72668E9
:10C0E000731C2360002D3FF43CAF0223AB5538E7AF
:10C0F0007B7826685E2B07F1010100F05781002D47
:10C1000000F08781731C23600323AB552368013340
:10C1100023606368013363607B785D2B00F0588196
:10C120004FF00009002B00F0C7805C2B00F00A8163
:10C130002368002D00F032815A1C22600A78EA54EC
:10C140000F467B782D2B00F00F810B785C2B00F0D5
:10C150001481002D00F01D8123685A1C22600A788A
:10C16000EA540F467B785D2B07F1010109F10109C3
:10C17000D8D14FFA89F34B4518BF48F00108002D7C
:10C180003FF4F3AEAB1983F80190EEE67B782668B6
:10C190003F2B00F02081A36803F10109C4F8089047
:10C1A000002D00F02981731C23607E23AB554FEADC
:10C1B0004903226859B2994218BF48F00108511C3E
:10C1C0002160AB546368013363604FF0010B21467B
:10C1D000029A781CFFF756FE014600286CD00278C0
:10C1E000292A69D1BBF1000F3FF4BFAE002D00F04A
:10C1F000478123687E22581C4FEA4909206009F1D3
:10C200000109EA544FFA89F34B4518BF48F0010879
:10C2100023685A1C226005F80390A3E6002D4FD036
:10C2200023685122591C2160EA54266899E6002DA2
:10C2300000F08580731C23600523AB5523685A1CCE
:10C2400022607A78EA548DE67C2B7FF47CAE0198EC
:10C2500000283BD02268131A013B59B2994218BFFB
:10C2600048F00108002D34D02B542268039805EBC8
:10C270000A063146A2EB0A0229F06CF82368EA1894
:10C280006021033323609170236801931A460132C1
:10C290006123226005F80A302368A3EB0A03023BFE
:10C2A00073705AB226689A4218BF48F0010839469E
:10C2B00063680233636058E6002005B0BDE8F08F84
:10C2C0002668013626604CE60025E6E5002DCCD137
:10C2D0002268161DD31C0193A6EB0A03023B5AB237
:10C2E00026609A4218BF48F00108E0E70232226057
:10C2F0007B783F2B00F0D080931B023B16465AB24E
:10C3000039469A4218BF48F001082BE6131D2360F6
:10C31000B21A043A797850B2904218BF48F0010836
:10C320003F2900F09E809A1B023A1E4653B2934268
:10C3300018BF48F0010839465FFA88F8B8E7B31C1F
:10C3400023600FE648784F1C0028B5D055B3D4F8C9
:10C3500000B00BF10103236053F040F905F80B0026
:10C360007B782D2B7FF4F1AEBB785D2B3FF4EDAEE7
:10C370005C2B07F102017FF4ECAE48784F1C0028DB
:10C380009AD03DB121684B1C236053F027F96854C3
:10C39000E8E60F46236801332360E3E601332360B8
:10C3A0000F46CEE6236801332360CAE6002D43D052
:10C3B000731C23600423AB55236801332360636837
:10C3C00001336360BB785D2B07F102017FF4A8AEF7
:10C3D0004FF00009D6E6BB783A2B7FF4DCAE4FF085
:10C3E000000B0237D946F2E6002D31D0791C6123CB
:10C3F0000CE6B31C2360B4E54FEA4903B21C22608B
:10C400005AB29A4218BF48F00108DBE6791C622351
:10C4100033E6636801336360B31C23607B785D2B74
:10C420007FF47EAEA1E5B31A023B58B2394698427A
:10C4300018BF48F00108F5E5636801336360B31C79
:10C440002360BB785D2B07F102017FF469AE8CE5B8
:10C45000B31A023B58B2791C984218BF48F0010841
:10C46000E0E59A1B023A1E4653B2934218BF48F0C9
:10C470000108791C5FFA88F81AE7791C622321E623
:10C4800022684FEA49030133023222605AB29A42CB
:10C4900018BF48F0010865E5931B023B16465AB2E7
:10C4A000791C9A4218BF48F001085BE530B5027963
:10C4B0000B780D4662F3470305F8013B85B00C4647
:10C4C0008068012201A92DF017FB019B1A68C4F8AE
:10C4D00001209B88AB8005B030BD00BF154B98890B
:10C4E000D98993F900C0421A92B2402A28BF40224B
:10C4F000BCF1000F05DB884218D00F49002055F031
:10C500002FB888420ED000B583B099680A480192CE
:10C5100028F0F0FE0849019A802003B05DF804EB92
:10C5200055F01EB88020002155F01AB800200146B1
:10C5300055F016B8441E0120B44401202DE9F04FF7
:10C54000DFB000AF0A460D4607F10801804659F0FA
:10C5500053FD334A13685268391D5B1A9A4257D902
:10C560000446002841D107F1580107F1080059F0AD
:10C5700030FE04466E462846A246002C46D197F867
:10C580007240002C42D04EF021FD044607F17200AB
:10C590004EF01CFD04EB000B0BF1080222F0070229
:10C5A000ADEB020D814622462946684628F0A2FEE0
:10C5B0004FF02F030DF8043001344A460DEB040010
:10C5C00007F1720128F096FE97F864300BF1010B29
:10C5D000DB060DF80BA0EA4611D45146404659F04F
:10C5E0009BFF0446B5460028BDD007F1080059F06E
:10C5F0000AFA204607F5BE77BD46BDE8F08F6946CA
:10C600004046FFF79BFF04460028E6D0B546ECE71E
:10C610000224204607F5BE77BD46BDE8F08F00BF77
:10C620000C5201200C4B187E01280DD002280ED090
:10C630000A4B1B68D9070BD4DA030BD413F4801F01
:10C640000CBF0020042070475B7EFF2BF0D07047AA
:10C650000520704701207047D05B01204455012020
:10C660002DE9F041DFF8288006460D4600244FF6FC
:10C67000FF7738F81400B84204F144042A463146E2
:10C6800001D049F0E3FEB4F5AA7FF2D1BDE8F08114
:10C69000A8050120034B53F8203013B19A680132EA
:10C6A0009A607047841D0120244B53F82030002BE2
:10C6B00042D010B4197993F805C09879204C1F29FD
:10C6C0008ABF204A4FF0A04201F01F01D2F8102586
:10C6D000BCF11F0F22FA01F28ABF1A494FF0A041A4
:10C6E0000CF01F0CD1F81015520021FA0CF101F0DA
:10C6F000010102F002020A4342EA8000D97914F8EB
:10C7000000C093F908009A71614449B28142D9711D
:10C710000ADA4042814204DCDA680021013ADA6038
:10C72000D9715DF8044B7047DA6800210132DA6094
:10C73000D9715DF8044B7047704700BF7C3501200C
:10C74000848F0900000300502DE9F04F0446ABB080
:10C750008B4640F28A40214633F09EFB002800F0D1
:10C760000183012120462DF00FFA4268CDE90D42E8
:10C7700000230F938DF864300DAD082109A856F001
:10C78000D9FD002328469946CDE9073352F004FF2E
:10C79000DFF814A6C8464F469DF86440002C00F010
:10C7A0002981284652F0F8FEA4F10903742B00F207
:10C7B000298201A252F823F099C7020099C702000A
:10C7C00005CC020005CC020099C7020005CC02008E
:10C7D00005CC020005CC020005CC020005CC02000D
:10C7E00005CC020005CC020005CC020005CC0200FD
:10C7F00005CC020005CC020005CC020005CC0200ED
:10C8000005CC020005CC020005CC020005CC0200DC
:10C8100005CC020099C7020005CC020027CB02001C
:10C8200005CC020005CC020005CC020005CC0200BC
:10C8300005CC020005CC020005CC020005CC0200AC
:10C8400005CC020099C702008DC9020005CC020088
:10C8500005CC02008DC902008DC902008DC90200FD
:10C860008DC902008DC902008DC902008DC9020068
:10C870008DC902008DC902008DC9020099C702004E
:10C8800005CC020005CC020005CC020005CC02005C
:10C8900005CC020005CC020005CC020005CC02004C
:10C8A00005CC020005CC020005CC020005CC02003C
:10C8B00005CC020005CC020005CC020005CC02002C
:10C8C00005CC020005CC020005CC020005CC02001C
:10C8D00005CC020005CC020005CC020005CC02000C
:10C8E00005CC020005CC020005CC020005CC0200FC
:10C8F00005CC020005CC020005CC020005CC0200EC
:10C9000019CA020005CC0200CBC9020005CC020006
:10C9100005CC020005CC020005CC020005CC0200CB
:10C9200005CC020005CC020005CC0200A3CA02001F
:10C9300005CC020005CC020005CC020005CC0200AB
:10C9400005CC020005CC020005CC020057CA02004B
:10C9500005CC020005CC020005CC020005CC02008B
:10C9600005CC02000FCC020005CC020005CC020071
:10C9700005CC020005CC020005CC020005CC02006B
:10C98000FBCA020005CC0200CBC9020000260A96B1
:10C990000DE02B2C08D02D2C06D0204652F018FF8D
:10C9A0000346002800F05581284652F0F5FD214647
:10C9B00009A856F0D5FB9DF864402E2C03D004F056
:10C9C000DF03452BE5D10126EEE7002F00F01A81A9
:10C9D000079B002B00F0DD81013B089A079352F87A
:10C9E000237038462FF0A0FB9DF864408046002C51
:10C9F0007FF4D7AEBBF1000F00F08D81002F00F067
:10CA00000181079B002B40F0FD8009A856F032FC05
:10CA100038462BB0BDE8F08F002027F0F3FA04462B
:10CA2000A7B1D04571D0B9F1000F00F0EB804946B5
:10CA3000224638462EF0A8FD089B4FF00009002B37
:10CA40006AD0394605A830F02FFC20462FF06CFB49
:10CA500027468046A0E69DF86430752B40F0D280D2
:10CA6000284652F099FD6C2840F0CC80284652F0C0
:10CA700093FD6C2840F0C680284652F08DFD002FB3
:10CA800000F03B81D04500F06381B9F1000F00F068
:10CA9000268149460E2238462EF076FD4FF00009D9
:10CAA0007AE69DF86430612B40F0AC80284652F065
:10CAB00073FD6C2840F0A680284652F06DFD732867
:10CAC00040F0A080284652F067FD652840F09A802B
:10CAD000284652F061FD002F00F02B81D04500F078
:10CAE0003C81B9F1000F00F0008149461E22384612
:10CAF0002EF04AFD4FF000094EE6002030F0FCFC1D
:10CB00000446002FA2D0D0458DD12146384630F0C2
:10CB1000CBFB089B002B94D1012105A830F012FC1F
:10CB2000089B1F6091E79DF8641000230A9351B998
:10CB300068E009A856F014FB284652F02DFD9DF838
:10CB4000641000295ED0222900F099805C29F0D180
:10CB5000284652F021FDA0F162030146132BE8D8CC
:10CB600001A252F823F000BF0BCC020033CB02002D
:10CB700033CB020033CB0200C5CB020033CB020023
:10CB800033CB020033CB020033CB020033CB0200A5
:10CB900033CB020033CB0200C1CB020033CB020007
:10CBA00033CB020033CB0200BDCB020033CB0200FB
:10CBB000B9CB0200C9CB02000921BAE70D21B8E7C1
:10CBC0000A21B6E70C21B4E704240026284652F0D7
:10CBD000E3FC40F02000C3B2A3F13002D2B2092A34
:10CBE00084BF573BDAB2013C42EA0616EED1314629
:10CBF00009A856F0C1FA284652F0CEFC9DF8641000
:10CC00000029A0D1654833F055FA082191E79DF835
:10CC10006430722BF6D1284652F0BEFC7528F1D153
:10CC2000284652F0B9FC6528ECD1284652F0B4FCF5
:10CC3000002F00F08380D04500F08580B9F1000F0F
:10CC400050D049463E2238462EF09EFC4FF0000957
:10CC5000A2E55EB3009002460390DDE90A1032F0CF
:10CC600035FC039BAFB3D04542D0B9F1000F1BD0C8
:10CC700049460246384699462EF086FC8CE5284601
:10CC800052F08AFCDDE90A1030F03AFE0FB3D045CD
:10CC90002ED0B9F1000F07D04946024638462EF093
:10CCA00073FC4FF0000977E5814675E5DDE90A1070
:10CCB00033460A2232F09AFD5FB1D04518D0B9F15F
:10CCC000000FF1D0494602463846B1462EF05CFCD2
:10CCD00062E50746BBF1000F7FF490AE1BE04FF01A
:10CCE0000E0959E54FF03E0956E54FF01E0953E590
:10CCF0000146384630F0D8FA4EE50E27BBF1000F5A
:10CD00007FF47FAE9DF86420104652F075FD48B167
:10CD1000284652F041FC9DF86420104652F06CFD0C
:10CD20000028F5D1002A7FF46DAF002F7FF469AEA3
:10CD300068E71E27BBF1000FE4D062E63E27BBF197
:10CD4000000FDFD05DE63E21384630F0ADFA23E536
:10CD50000E21384630F0A8FA1EE51E21384630F084
:10CD6000A3FA19E5034610AA7E212046CDE9173320
:10CD70002DF066FC0A4A0B4B139201214022CDE9AB
:10CD800014120DAD1AA913AACDE90D5316911292E2
:10CD9000F3E4BBF1000F7FF438AEBCE718BB090029
:10CDA000005A09004DF507009C5F090038B503885B
:10CDB000112B0C460AD0362B06D119B182888B89EB
:10CDC0009A420AD0012038BD002038BD4FF6FF72CC
:10CDD00001238A810B74002038BDC388CB81C589AB
:10CDE0004A68954228BF154600F110012A4620687E
:10CDF00028F080FA0120A560207438BDC2070346E0
:10CE000021D400B510F0030283B00BD1114A0168A0
:10CE100091421BD018462FF087F95E22C1880E4838
:10CE200033F03CF9022AF5D10C4A0240062AF1D02F
:10CE30002FF0CAF8FCEEC07ACDED017A9DF804001F
:10CE400003B05DF804FBC0F3470070472FF05AF9B8
:10CE5000C0B2F5E7245F0900ECA80900070080FFD5
:10CE60002DE9F041044682B09846A37C099D089EB6
:10CE70005B422B70CB07084617460FD52FF042F9BF
:10CE800003143B70031288F800303070A37C13B990
:10CE9000227B042A31D002B0BDE8F08111F00303F7
:10CEA00026D0022B3AD001AA69462FF051F8009AF9
:10CEB000D31E012B3DD8019B1868FFF79FFF019BF4
:10CEC00038705868FFF79AFF019B88F8000098684F
:10CED000FFF794FF009B3070032BD7D9019BD868D4
:10CEE00000F00303022B28D02FF00CF92870D2E7B2
:10CEF0001A4B0A689A42D6D1C0E7627C002ACAD08F
:10CF0000397898F800208A42C5D131789142C2D14F
:10CF100029703B7088F800303370BCE7104B0B4031
:10CF2000062BC0D02FF050F8FDEEC07A17EE900A15
:10CF3000A6E7217B0B4833F0C5F8094B0340062BCD
:10CF4000D2D02FF041F8DFED087A20EE270AFCEE70
:10CF5000C07A17EE903A2B709DE700BF245F09005E
:10CF6000070080FFA0B9090000007F4330B585B0FD
:10CF700003AC0DF10D0301940D46009311460DF124
:10CF80000E030DF10F020446FFF76AFF9DF80C1027
:10CF90009DF80D209DF80E30CDE9002120469DF82A
:10CFA0000F20294600F002F805B030BD70B50589A4
:10CFB0009DF810E09DF81460042D34D0446A01FB04
:10CFC00005FC002C3AD004EB0C01046A6444042DE7
:10CFD00004BF057C4E55457B4A55857B4B55C57B2B
:10CFE00001F805E0A4B10189042912D0418901FBAF
:10CFF00002F2417B121262544289817B02FB03F3ED
:10D000001A1262544389C27B0EFB03F31B12A35412
:10D0100070BD817C21B9418901FB06F6C6F3072664
:10D02000017C6654E2E7847C002CC7D0446AF60891
:10D0300046F0E00601FB05FC002CC4D1016A614406
:10D04000C5E700BF38B500F110050446284651F089
:10D0500029FA3F2800D838BDE07854F04BF9002871
:10D06000F9D0284651F01EFA3F28E07806D904F698
:10D0700038014022BDE8384054F072BABDE838406B
:10D0800054F018BA38B500F110050446284651F09E
:10D0900009FA3F2800D838BDA07854F02BF90028B1
:10D0A000F9D0284651F0FEF93F28A07806D904F5BA
:10D0B0009C714022BDE8384054F052BABDE8384077
:10D0C00054F0F8B970B5294E7388CCB031220124E0
:10D0D000B3F57F7F8DF80C208DF80D4039D20546D1
:10D0E000022103A800F0DAFE38BB73881A1DAA4299
:10D0F00024D81F4AD2F8EC20946833444434187181
:10D1000004AA311D204659F05FF900BB9DF81C3080
:10D11000DB0616D42046174959F0FEF9044654F0B0
:10D12000D5F8B0B900900346022203A912480FF0C7
:10D1300031F811480EF06CFF00E0002420464CB09E
:10D1400070BD311D2046FFF7F9F90028E2D054F0F8
:10D15000BDF800230222009303A907488DF80D2093
:10D160001C460FF017F820464CB070BD2047012038
:10D170000C520120244701205C4401202DE9F04F8E
:10D180000446E1B06E480EF05BFFB0F1000BC0F258
:10D19000AC806C4F7B88B3F57F7F80F0B2801A1D26
:10D1A000A24200F2A880684AD2F8EC20391D9068AB
:10D1B0005A1E44308C5C2F2C00F0AE803B44002281
:10D1C0001A71624A04A958F017FF002340F2511265
:10D1D000C7E90023C7E902330390002840F09F808D
:10D1E00018A904A858F0F5FF002840F0A280DDF847
:10D1F0000CA004E058F0EDFF0AF1010A28B99DF8EF
:10D200007A3018A904A8002BF4D1002104A858F002
:10D21000E0FFC7F808A0BAF1000F52D0DFF8208174
:10D220004FF0000918A904A858F0D3FFBDF86A30E0
:10D23000BDF86810C7F8049003F01F025200019275
:10D24000480AC3F344120092DB0A01F01F0200F205
:10D25000BC70C1F3431150F005FA3D4B3D49C01875
:10D26000A0FB01034FF00002386142F1000001FB16
:10D2700000309DF86C30786113F0100331D0012339
:10D28000BA61FB600DF17A004DF0A0FE0546788092
:10D29000584649F045FC85B1002426462A1B042A3D
:10D2A00028BF04220DF17A031919009614440023B3
:10D2B00040460EF06FFFA542F0D809F10109D145B3
:10D2C000B0D104A858F09FFB0023BA687B80584671
:10D2D0007A60FB60BB6149F023FC039861B0BDE854
:10D2E000F08FFB60189BBB61CCE70023039303988E
:10D2F00061B0BDE8F08F01230393039861B0BDE8EE
:10D30000F08F40F251233B800023039349F008FC47
:10D31000039861B0BDE8F08F00238B5451E70322DE
:10D3200058467A70039349F0FBFB039861B0BDE85F
:10D33000F08F039C04A8214658F04BFFBC60C0E767
:10D340005C440120204701200C5201202447012089
:10D3500080436D3800CA9A3B30B52E4B2E4A1B686D
:10D3600014681A68012151641B682C4AD3F844558B
:10D3700002F1200C52F8043F13B11979814202D016
:10D380006245F7D130BDDA7932BB5A699969A21A80
:10D39000691AC2EB02420A44D989188A80B210FA8B
:10D3A00081F198894FF6FF7C4FF6FE7E724588BF6B
:10D3B0006246B1FBF0FC00FB1C11986820F81120BC
:10D3C000198A988989B2814219D21A8A013292B295
:10D3D0001A825C619D6130BD1F288ABF104A4FF0E0
:10D3E000A04200F01F01D2F8102522FA01F15A796B
:10D3F00001F001018A42ECD00022DA71E9E7DA8912
:10D4000092B20132B2FBF0F100FB112292B2DA814A
:10D41000DFE700BFE45601201055012058350120F8
:10D42000000300502DE9F04F2DED048B00F1080BA7
:10D4300093B0064608AF58461BF0F8F828B92C37C9
:10D44000BD46BDEC048BBDE8F08F96F86210002954
:10D4500040F05D81F068002800F0E6801CF0D2FA10
:10D460003860002800F0E080396807F11002584663
:10D470001AF094FE6B4609EE903A002800F0CB803B
:10D48000B7F91210B7F91630B7F910A0B7F9145060
:10D49000F9605A1A1FFA82F950462A461AF0F4F92E
:10D4A00096F8A330F96882B2002B00F0D0804FEAE2
:10D4B000D90078604FF4007008EE100A0820F86078
:10D4C00052090132900018EE102A073222F00702AA
:10D4D000ADEB020DC21D22F007020DF12008ADEBED
:10D4E000020D08AA09EE102A7A6808EE900A002AAE
:10D4F00000F091800024BC609C4678E02044084401
:10D5000000B27884FA6896F89A10A9EB020996F8A6
:10D510009B20CDF80CA0CDE90435CDE9060C002305
:10D52000029396F89F3001934FF48073009358460E
:10D530001AF092FE96F85250B7F92230B7F920202F
:10D54000B7F91E10B7F91C00072D1FFA89F974D915
:10D550001AF09AF9ED0815FB00FA1FFA8AFA18EE8C
:10D56000902A002119EE100A27F074FF18EE102AF5
:10D570000021404627F06EFF584619EE102A434618
:10D5800007F11C011AF04CFE58461AF0FFFD002866
:10D5900041D0316AB0681AF0F7FD96F89F1031B9A2
:10D5A0000122B0680092756A06F19C03A847BB6827
:10D5B000B0680133BB60CDF800A0434600220121D2
:10D5C000756AA847B16AB0681AF028FE52F0A0FB4D
:10D5D000FA683B8914447A689A42A4B21BD9B7F915
:10D5E00010A0B7F91210B7F9145096F8A3C0F86854
:10D5F000A7F81CA089B200230A197B62814513B2E7
:10D600003D84FB831FFA82FEBFF478AF0EEB090264
:10D6100010B2788476E73B6819EE902A9B683B60ED
:10D620009546002B7FF420AF58461AF007FE2C37A2
:10D63000BD46BDEC048BBDE8F08F1AF025F9082338
:10D64000B3FBF5F5B0FBF5F51FFA85FA87E796F819
:10D6500052C02024B4FBFCF4B0EBC41F4FEAC41E3C
:10D6600019D852090132920008EE902A0732ADF51E
:10D67000007D22F007020DF12008ADEB020D08AA93
:10D6800009EE102A01227A604FF4007208EE102A87
:10D69000C7F80C902EE7A5EB0A021FFA82F8BEFB32
:10D6A000F8FE7246012A38BF0122BCF1070FFA606A
:10D6B0000DD896F8590050B90820B0FBFCFCB2FB1D
:10D6C000FCFE0CFB1E2CA2EB0C0082B2FA60F86888
:10D6D000B9FBF0FC00FB1C901FFA8CF280B27A6060
:10D6E00018B11046013082B27A60FA6812FB08F273
:10D6F00092B2B2FBF4F004FB10241FFA80FC14B1C8
:10D700000CF1010080B2800008EE100AD8E6002378
:10D71000736406F13C033B60A6E600BF2DE9F04FC1
:10D720002DED088B8FB0C36E00AF054600F170047D
:10D730005B6878612146806E98472B6FA3B12B46BA
:10D740000833184608EE903A1AF070FF95F8621008
:10D7500081B97B69D86818B11CF054F9786078B940
:10D7600018EE900A1AF06AFD3C37BD46BDEC088BF6
:10D77000BDE8F08F7A690023536402F13C037B60BB
:10D780007D69B5F84A2007326B46D2100BEE103A8D
:10D79000D31D6946DB08A1EBC3039D460021684603
:10D7A00027F058FEEB6EA86E5B6821469847E94665
:10D7B0004FF0010A796818EE900A07F120021AF07A
:10D7C000EDFC6B460AEE903A002800F027817B6959
:10D7D00093F85250072D00F238817B6993F8593045
:10D7E000002B00F03281B7F92460B7F920400823FC
:10D7F000B3FBF5F31E449AB294FBF3F4013E96FB9F
:10D80000F3F604FB03F316FB02F636B21CB2BE8439
:10D810003C84B7F92630B7F92280A3EB080189B21E
:10D820003246F961204641461AF02EF82023B3FB18
:10D83000F5F2B0EB421F4FEA421100F2A180C0F3B3
:10D840004A1301339B0009EE103A0733A0B023F0CE
:10D8500007036A46ADEB030D6B4609EE903AFB6990
:10D86000BB610123BB60802308EE102A0AEE103A48
:10D8700000223A6141460023B869FD697B6389B2A1
:10D880008B189BB2A842BC853E86FB8571D8831855
:10D890001944FB607986D7E906239B1A9BB219EEDF
:10D8A000102A002119EE900AFB6127F0D3FD1AEE31
:10D8B000102A002118EE100A27F0CCFD18EE103ABD
:10D8C00019EE902A18EE900A07F12C011AF0A8FC24
:10D8D0007B69B7F92C0093F85210B7F93020B3F8F0
:10D8E0009660B7F92E40B3F89450121A11FB00F36A
:10D8F00001FB02F2002B796906FB0455B8BF073320
:10D9000005EBE3030D6F1D44B7F93230002AA4B2D2
:10D91000B8BF0732A342C8BF18EE108A4FEAE20B25
:10D9200016DDE20804F0070319F802100AFA03F3FF
:10D930000B4309F80230414628465A4627F0DAFCE4
:10D940000134B7F93230A4B29C42D8443544E8DB04
:10D950003C6901343C6152F0DBF9B968BA89A3B281
:10D9600099425BD9B7F92040B7F92210B7F9246082
:10D9700081E7F9690B447B86BB691344FB608AE746
:10D98000331B9BB2B1FBF3F1012938BF0121072DF5
:10D990000846B9610DD8796991F8591049B908213B
:10D9A000B1FBF5F5B0FBF5FC05FB1C01411A89B292
:10D9B000B961F969BD69B1FBF5F005FB101189B2D8
:10D9C00080B2B86019B10146013189B2B960B96954
:10D9D00011FB03F39BB2B3FBF2F102FB113289B2EC
:10D9E0000AB1013189B25B098A0001339900D31D64
:10D9F00023F00703ADEB030DCB1D0AEE102ADB0865
:10DA00006A46A2EBC30309EE903A9D46BB6809EE55
:10DA1000101A08EE102A002B7FF42AAF7B681AEE4A
:10DA2000902A9B687B609546002B7FF4C3AE7A6991
:10DA3000D36E906E9B68494698471BEE103A18EEDD
:10DA4000900A9D461AF0FAFB8EE6B7F92040B7F926
:10DA50002460DEE6F0B54368DB6853F8216085B0EA
:10DA600004460F464FF49160314632F015FA0546F0
:10DA700090B16B6830469847AB6801A95B68064671
:10DA80009847AB6802469B68304600211546984788
:10DA90006368DB6853F82760234930462DF056FB56
:10DAA0000346C8B1B0F93C20B0F93810914239D0E2
:10DAB000816B0191C18FADF80820ADF80A100125E6
:10DAC00093F850206FF3041283F8502000229A62DA
:10DAD0006368DB6853F82760144930462DF036FB45
:10DAE000064638B101A91BF01BFF00210546304650
:10DAF0001CF0D6FA7DB194F82A30DB070DD504F17D
:10DB0000180201A9104619F0C7FE94F82A3043F014
:10DB1000010384F82A3005B0F0BDDDE90123C4E932
:10DB20000623F2E70025CBE72806090000020900DA
:10DB3000F8B51C4B1C4E4FF0FF0C002714461F7607
:10DB400083F819C00D4600F0D7FF00220023C6E974
:10DB500000231DB3BC463946201F144F634602E024
:10DB600001339D420DD050F8042F9407F8D114686A
:10DB7000BC42F5D199B901339D4294464FF0010161
:10DB8000F1D159B19CED017ADFED097A67EE277A80
:10DB900017EE900AF9F7CCFDC6E90001F8BD05487B
:10DBA00032F088FAD05B0120E009012050BD080066
:10DBB00000007A4490B309002DE9F84F0546C78963
:10DBC0002B7A008A8A46BFB280B2002B43D1391A21
:10DBD0008742AB8889B253D35E1AB6B2964228BF49
:10DBE0001646A6EB0308B5F806901FFA88F89F4280
:10DBF0003C4603D3E41AA4B29C42FBD21B1B286808
:10DC00009BB29E4209FB040012D809FB06F2514662
:10DC100027F070FBF3199BB29F4202D8AA899A425F
:10DC200002D26A8913449BB2EB813046BDE8F88F7B
:10DC300013FB09F31FFA83FB5A46514627F05AFBA0
:10DC400008EB040212FB09F228680AEB0B0192B2FE
:10DC500027F050FBDEE7AB889A4209D3B5F806906F
:10DC6000D61A09FB061A07461E464FF00008BEE703
:10DC7000A2EB0308B5F806901FFA88F81646B6E737
:10DC80006889091A89B2A7E72DE9F84343689A68B9
:10DC900062B3DFF87090DFF87080074600250BE074
:10DCA00063689847A36807F108019B6898477B68F9
:10DCB0009A680135954219D2DB6853F825604FF414
:10DCC0009160314632F0E8F804463046002CE7D146
:10DCD00049462DF03BFA414650B107F108011CF0CE
:10DCE00079FF7B689A6801359542E5D3BDE8F883F2
:10DCF00030462DF02BFA0028D9D007F108011CF08E
:10DD0000CFF9D4E7280609000002090090F9503045
:10DD1000234910B5002B836AB4BF428A028AB0F946
:10DD20000CE0002B08BF0B46997BD9B193F9054055
:10DD3000B3F802C004FB0ECC0FFA8CFCA0F846C06E
:10DD40000EEB020193F905205C8812FB01F32344DA
:10DD50001BB29C45D2BFA0F84A30A0F84AC0A0F838
:10DD6000463010BD93F90440B3F800C004FB0ECC5C
:10DD70000FFA8CFCA0F844C00EEB020193F90420CA
:10DD8000B3F800E012FB01F373441BB29C45D2BF11
:10DD9000A0F84830A0F848C0A0F8443010BD00BF3B
:10DDA0003003012090F95030234910B5002B836ACD
:10DDB000B4BF028A428AB0F90EE0002B08BF0B46BE
:10DDC000997BD9B193F90440B3F800C004FB0ECCA1
:10DDD0000FFA8CFCA0F844C00EEB020193F904206A
:10DDE0001C8812FB01F323441BB29C45D2BFA0F850
:10DDF0004830A0F848C0A0F8443010BD93F9054061
:10DE0000B3F802C004FB0ECC0FFA8CFCA0F846C09D
:10DE10000EEB020193F90520B3F802E012FB01F3C7
:10DE200073441BB29C45D2BFA0F84A30A0F84AC048
:10DE3000A0F8463010BD00BF3003012010B500210E
:10DE4000044688B0084601E0082919D03DF05CF886
:10DE5000F8B14378013BDBB2FD2BF5D8037803F032
:10DE60000103A342F0D1C38808AA502B02EB810220
:10DE70000FD1013100F14003082942F8203CE5D1DF
:10DE8000CAB26846002148F0ADFA0146084608B01B
:10DE900010BD0029F4D1084608B010BD10B50E4BD6
:10DEA0001C7882B014B9204602B010BD0B4B1B7811
:10DEB00043B10B4A13782BB91C460121204611703F
:10DEC00002B010BD0023052242700A4600930146AD
:10DED00004480EF05FF9E6E7C25B01205C02012016
:10DEE000AB5B01205C44012010EE102A22F00043BD
:10DEF000B3F17E5F09D344D1DFED4C7A9FED4C0A3C
:10DF0000002AA8BFB0EE670A7047B3F17C5F05D264
:10DF1000B3F14A5F3CD89FED470A7047002A5ADBAD
:10DF2000B7EE007A37EE400AF6EE007A20EE270AC6
:10DF3000DFED415A9FED416ADFED417AF1EEC06AB3
:10DF4000A0EE256ADFED3F5AE0EE067AA0EE257AD4
:10DF500016EE903A60EE277A23F47F6323F00F03E6
:10DF600087EE876A07EE903AA7EEE70A76EEA75AA1
:10DF700080EE257AA6EE867A37EE870A30EE000A22
:10DF8000704770EE407A9FED297A87EE270A704736
:10DF900020EE007ADFED286ADFED287ADFED285ADF
:10DFA000E7EE267ADFED276AE7EE275AB7EE006A3A
:10DFB000A7EE266A27EE257ADFED236ADFED1D7ACC
:10DFC000C7EE065AB0EE667AA0EE657A30EE470AE2
:10DFD00037EEC00A7047F7EE007A30EE270AB6EE49
:10DFE000007A20EE070A9FED156A9FED137ADFEDA8
:10DFF000145A9FED145AA0EE076AE0EE057AE0EE9F
:10E00000065AB1EEC07A20EE250AF0EE676AC0EE3D
:10E01000265A9FED0E6ADFED077AA7EE256A37EEE6
:10E02000060A37EEC00A30EE000A70470000000012
:10E03000DA0F4940DA0FC93F6BD30DBCBA132FBDBD
:10E0400075AA2A3EAEE534BF6821A2336821A2B387
:10E0500008B510EE103A5A00F0EE407A1FD523F0C2
:10E060000042B2F18B4F06D326F04AFCDFED147A62
:10E0700030EE270A08BDFFEE006AE0EE006ABDE858
:10E080000840B1EEE67AF7EE005A37EE007AB0EECD
:10E09000006A85EE870A97EE860A26F031BCB7EE55
:10E0A000000A77EEC07ABDE8084037EEA77AA7EEFF
:10E0B000A77AB1EEC70A37EE800A26F069BB00BF27
:10E0C0001872313F70B588B00D460C2000211646FD
:10E0D000039326F0E1FC0F4B036005AB01930E4B5D
:10E0E000039A0093044603233146284628F04EF84D
:10E0F0009DF81830059A626023729DF81C3013B9A0
:10E10000204608B070BD20460BF0CEFE204608B079
:10E1100070BD00BF38BA080080CD080010B50446B5
:10E1200040680BF0A3FE204610BD00BF08B50B6889
:10E1300058680BF0F9FE0E2008BD00BF10B58EB078
:10E1400003AB51F8044B0193184B009301380323A0
:10E1500027F0B2FF606806AA40F2A5412CF070FAE1
:10E16000227A049B03980599520042F0010208921A
:10E1700040F62612CDE909025B006FF0004243F041
:10E18000010391420B930ED0490041F0010140F28E
:10E19000E643CDE90C31022106AA022029F074FBE6
:10E1A0000E200EB010BD0121F6E700BF58BF0800D9
:10E1B00010B58EB003AB51F8044B0193184B00938C
:10E1C0000138032327F078FF606806AA40F2C151A6
:10E1D0002CF036FA227A049B03980599520042F0FB
:10E1E0000102089240F62612CDE909025B006FF0A9
:10E1F000004243F0010391420B930ED0490041F0DD
:10E20000010140F2E643CDE90C31022106AA0220C9
:10E2100029F03AFB0E200EB010BD0121F6E700BF39
:10E2200088CF080030B597B003AB51F8044B019389
:10E23000314B00930138062327F03EFF606809AA9E
:10E2400040F2C2512CF0FCF9227A0398059B069902
:10E25000520042F001020B92049A5B00CDE90C02DD
:10E260006FF0004243F0010344F266509142CDE961
:10E270000E0338D0490041F0010144F2465209230F
:10E28000CDE910214FF00B0E4FF00A0C1C46032174
:10E2900016AA02EB8300079B02EB8C0C5B0043F099
:10E2A0000103089A43F6964540F8345C4CF8343C38
:10E2B0006FF000439A420FD016AB03EB8E0E03EBC8
:10E2C0008404520042F00102013143F676434EF8D5
:10E2D000343CC9B244F8282C09AA032029F0D4FA06
:10E2E0000E2017B030BD07234FF0090E4FF0080C79
:10E2F0001C460221CCE700BF48CE080070B58CB0A8
:10E300000D46182000211646039326F0C5FB164B38
:10E31000036005AB0193154B039A00930446072352
:10E320002846314627F032FF9DF82430089A059D93
:10E330009DF828009DF82C1023739DF81C30A260D6
:10E34000069A656060730698A1732261237528B1EF
:10E35000002201210EF0AAFE022802D020460CB0B5
:10E3600070BD034831F060FEF8BA080070BF0800C5
:10E3700004B3090010B58AB004466A46406840F20A
:10E380007B512CF05DF901E02BF03EFD00216A4647
:10E39000084629F079FA2EF021FF03460120002BD0
:10E3A000F2D060686A464FF43F712CF049F9A268D8
:10E3B000217B637B520042F0010242F606304900A5
:10E3C000CDE9020241F0010144F286705B00CDE923
:10E3D000040143F0010344F2B661CDE9061342F6AD
:10E3E000A6301123CDE908036A460421002029F054
:10E3F0004BFA23691BB1217D58680EF025FE606839
:10E400000AB010BDF0B50D682B6989B02BB1297D1C
:10E41000586881F001010EF017FEAB7B73B905AAB5
:10E420006868019240F292512CF00AF90021019A99
:10E43000084629F029FA0E2009B0F0BD01202FF07E
:10E440001DF8022202A906462BF056FB029BFF2272
:10E450001A70AB7B6868073305AADF10A42101920C
:10E46000DC082CF0EDF8019A0796002FD8D0002197
:10E470000120019229F008FA631E13F0FF04019AAB
:10E48000F5D1CDE72DE9F041054682B001F1340028
:10E490000E4606F0D1F82B88102B31D0112B2BD142
:10E4A0000022A888364F134637F81210814202F135
:10E4B000440203D00133052BF6D1042303EB0313ED
:10E4C00007EBC3042F4821464FEAC30807F0B4FA0C
:10E4D000E36D4FF6FF7227F808200E2B4FF0000275
:10E4E00084F85A2002D05A602A7A1A720023012036
:10E4F000B36102B0BDE8F081002002B0BDE8F08158
:10E5000000231F4F1A464FF6FF7037F81310814251
:10E5100003F1440303D00132052AF6D1042202EBB1
:10E520000212D400AB883B5307EBC2020E234FF01C
:10E53000000804F16000D365384482F85A80A2F8DC
:10E540007680104907F05EFAC6F818802869696974
:10E550006C34274403C7684647F050FFBDF80030CD
:10E560002A8A9A4202D86A8A9A4203D2A8886946BD
:10E5700047F032FF00230120F36002B0BDE8F081D4
:10E58000A80501202D4D040070B50E46C18A044631
:10E59000013189000069154626F0B2FAE38A20614C
:10E5A000591CE18200EB8302002120F823109670B1
:10E5B000D57070BD10B50388102B0C4606D0262BE5
:10E5C0000CD108460DF0E8F9012010BD8188002229
:10E5D000032047F021FF20460DF0DEF9002010BD9A
:10E5E0002DE9F04383078BB0054670D13A4B1446B2
:10E5F00002689A426BD10846012203A92BF07CFAEB
:10E600002046022269462BF077FA049C019A2146A3
:10E61000284653F001FB03990098224626F06AFE33
:10E6200095F80C31022BDDE9000607D0062B45D00A
:10E63000012B3CD00E200BB0BDE8F08305F104089F
:10E64000002EF7D06FF00E0705F1F30900F10F046B
:10E650003F1AF43554F80F0C54F80B1C54F8033CD3
:10E6600054F8072C0DF1180CACE80F004146A4F14A
:10E670000F00FAF773FDA4F11003494613F8012FB8
:10E6800011F8010F9C4282EA00021A70F6D10DF1D6
:10E69000180CBCE80F001034696039198E422860EC
:10E6A000AA60EB60D6D80E200BB0BDE8F083291D20
:10E6B000FAF754FD0E200BB0BDE8F0830146324658
:10E6C000281DF9F703FC0E200BB0BDE8F0830348CA
:10E6D000F72131F0E3FC00BF50BB0800C4B90900CA
:10E6E0002DE9F047830786B0044670D13A4B1546B2
:10E6F00002689A426BD10846012203A92BF0FCF96B
:10E700002846022269462BF0F7F9049D019A294612
:10E71000204653F081FA2A460399009826F0EAFD34
:10E7200094F80C31022BDDE9000507D0062B43D00D
:10E73000012B3AD00E2006B0BDE8F08704F10408A2
:10E7400004F1F407002D40D06FF00E06361A00F1E8
:10E750000F09BA46D446A9F11003A9F10F0A0CF12A
:10E76000FF3C13F8012F1CF8011F994582EA0102B2
:10E770001A70F6D14146504609F11009F9F798FC94
:10E7800006EB09039D42E5D8DAF80000DAF8041038
:10E79000DAF80820DAF80C30C4F8F4000E207960BA
:10E7A000BA60FB6006B0BDE8F087211DF9F780FC78
:10E7B0000E2006B0BDE8F08701462A46201DF9F775
:10E7C00085FB0E2006B0BDE8F087BA46DCE70348BB
:10E7D000F72131F063FC00BF50BB0800C4B9090049
:10E7E00008B5830709D1074B02689A4205D190F812
:10E7F0000C01400040F0010008BD0348F72131F052
:10E800004DFC00BF50BB0800C4B90900F0B58BB087
:10E81000264C009405AD0846019511461A4605237D
:10E8200027F0B4FC00214FF48A7026F035F9204B14
:10E83000036004460122059802A92BF049F970B340
:10E84000039E26F00803102B01D0202E24D1069D14
:10E85000029F022D0DDD062D0DD1079870B102A982
:10E8600001222BF035F948B1039B102B1AD1029BE2
:10E8700005E0002DF1DC0F4831F008FC002384F89E
:10E880000C51089DC4F810512046324639460BF011
:10E890006BFC20460BB0F0BD074831F0F7FB074892
:10E8A00031F0F4FB0648102131F0F8FBD8BF080026
:10E8B00050BB080004B2090074B6090000B5090095
:10E8C00034B809002DE9F0410C4684B0012201A9B9
:10E8D00005466068D4F800802BF00EF9DDE901767A
:10E8E0000FB326F00803102B01D0202E18D1022DD3
:10E8F00009D800234046324639460BF035FC0E203D
:10E9000004B0BDE8F0810122A06801A92BF0F4F861
:10E91000DDE90132102AEDD00448102131F0BEFBB0
:10E92000034831F0B3FB034831F0C4FB34B80900AD
:10E9300074B6090000B50900830710B5044613D169
:10E940000B4B02689A420FD108462DF093FB022828
:10E9500005DD062805D184F80C010E2010BD002825
:10E96000F9DC044831F092FB0348F72131F096FBC3
:10E9700050BB080004B20900C4B9090000B583B057
:10E980000446019153F04CFA21460120019AFFF709
:10E99000CFF80248002131F0D9FB00BF34550900FF
:10E9A00070B510B90E25284670BD0E46044653F0CA
:10E9B00037FA324621460020FFF7BAF800F086FA0F
:10E9C00000231A464EF024F91F4B5D6A3DB10E2517
:10E9D00000F02EF9284648F017FD284670BDFDF7D7
:10E9E00021FE431EDBB2022BF1D8012814D00228ED
:10E9F0000DD11648311F2A4651F8045FAE0702F1C7
:10EA0000010202D12B68834202D09442F4D10E2538
:10EA1000284648F0F9FCDBE70D4B0E4893F819C087
:10EA20002A46331F01E09442F1D053F8045FA9074E
:10EA300002F10102F7D129688142F4D169680979AC
:10EA40006145F0D1E4E700BF0C52012050BD080041
:10EA5000D05B01207CBC080070B588B00D460C204E
:10EA600000211646039326F017F8134B036004ABFE
:10EA70000193124B039A009331460423044628461F
:10EA800027F084FB049853F091F99DF818309DF815
:10EA900014109DF81C2043B903792F2B08D860600F
:10EAA00020462172627208B070BD054831F002FB49
:10EAB000044831F0FFFA00BF7CBC080000C0080029
:10EAC00000BC0900ECB609004068002808BF0E2011
:10EAD000704700BF037A002B14BF3E201E207047F2
:10EAE00010B5044C237803B110BD16F069F801236A
:10EAF000237010BDBC5B01202DE9F04F89B0079059
:10EB000000296BD0444BDFF8249118685B680293AE
:10EB1000D9E90087414B424D0190043A002602EBAF
:10EB2000810C19685B6803910493B34605964FF016
:10EB3000FF314FF0010E0696009701E0944530D06A
:10EB400052F8043F9807F9D11868A842F6D15968DD
:10EB50001E7A0979A1F12000C1F12004002E40D0D5
:10EB6000009F05962EFA04FA0EFA00F646EA0A0607
:10EB700037430EFA01F6009746EA08085B7A0EFA68
:10EB800000F0002BDAD006932EFA04F4049B204305
:10EB90000343039804930EFA01F31843944503903A
:10EBA000CED1059B069E009F0BB1C9E90087BBF142
:10EBB000000F04D0184B019A1A60029A5A6026B1CD
:10EBC000164B039A1A60049A5A60013106D0079BCB
:10EBD000E3B11449144A00230B60137009B0BDE877
:10EBE000F08FA1F12000C1F12004029F0EFA00F67F
:10EBF0002EFA04FA46EA0A0637430297019F0EFAF4
:10EC000001F6374301974FF0010BB7E709B0BDE8B4
:10EC1000F04F15F0D5BF00BFC8090120D809012069
:10EC20007CBC080044550120BC5B0120B8090120D0
:10EC30002DE9F0433D4C3E4DA36A23F47F0323F4BA
:10EC40007F43AB4283B022D04FF48072002104F1A5
:10EC50002C0026F0FFFB4FF080434FF440320021A0
:10EC60004FF47C10A562C3F804292176C3F8142957
:10EC70006176C3F82429C3F83429C3F84429C3F8BA
:10EC80005429C3F86429C3F87429C3F88409DFF848
:10EC9000B480284FD8E900653B681E437B68002498
:10ECA0001D434FF00109A4F12003C4F1200229FA09
:10ECB00002F209FA03F3134309FA04F232402B403B
:10ECC0001343E0B207D045F09BFB20463CF0E8FA46
:10ECD00020463CF017FC0134402CE4D116490022B8
:10ECE0000023C8E90023C7E90023C1E90023134B2F
:10ECF0004FF40032C3F84823D3F80413890304D532
:10ED0000C3F80823D3F844213AB90D4B0020002161
:10ED1000C3E9000103B0BDE8F0830022C3F8442139
:10ED2000D3F844310193019BEFE700BFD05B012092
:10ED3000AF0000ADC8090120D80901200040024001
:10ED4000E0090120B809012070B5144686B0002AF8
:10ED50006ED011F0030503468C464FF0000603D138
:10ED6000474A086890422AD01868624600234FF448
:10ED700080712AF0CBFE042C054613D020462DF0DE
:10ED800079F9FF2803466FD86A1CB2F5807F02D953
:10ED90003C4831F067F93C4A15440E2085F82C3088
:10EDA00006B070BD431CB3F5807F03D836480544D8
:10EDB00095F82C60700040F0010006B070BD6A4606
:10EDC0004FF4807031F014FC002850D0042C34D063
:10EDD000DDE90035ED1AA3072CD123682B4A9342B5
:10EDE00008D02B4A934205D02A4A934202D02A4A9D
:10EDF00093421FD1012203A920462AF07DFE049BE5
:10EE0000AB423AD19DF81410039C0022402027F019
:10EE100011FA01282ED1009BEA18B2F5807FB7D8ED
:10EE20001E482A462146184426F064FA0E20B7E709
:10EE30001046B5E71A4831F0F7F8DDE90034E41A76
:10EE40002946204625F028FE009B1A19B2F5807F3E
:10EE5000054604D811492246194426F04BFA2946A2
:10EE600020462EF0FBFA9BE70E4831F023F90E48BE
:10EE700031F0DAF80D4831F01DF90D4831F01AF98A
:10EE800084620900C8AD0900D05B012080580900E8
:10EE9000005A0900146009003C5A0900FC5B01207B
:10EEA0005CAA090074BD0900709C090034BF090008
:10EEB00098B10900042806D0052840F2012314BFA8
:10EEC0000020184670473E20704700BF38B5084BF9
:10EED000D3E9004554EA050305D04DF017FD201A8B
:10EEE00065EB010138BD4FF0FF30014638BD00BF72
:10EEF000E009012070B52DED028B8AB00D46082087
:10EF000000211646039325F0C7FD314B036005AB86
:10EF10000193304B039A009304460223284631465E
:10EF200027F034F9DDE90505B0F10E0218BF012222
:10EF3000B5F10E0318BF01239A4242D00E283DD0EE
:10EF40002DF042F8B0EE408A4DF0E0FCF8F742FBBD
:10EF5000DFED217A07EE100A0E2DC7EE278A21D0A9
:10EF600006982DF033FF054646F08EF907A94CF0C0
:10EF700035F99DF822109DF821209DF82030BDF82C
:10EF80001C00CDE900219DF81F209DF81E104EF0B9
:10EF9000E7FB124B281A034407EE903AB8EEE78AD3
:10EFA00038EE288AB4EEE88AF1EE10FA0CD4204646
:10EFB00084ED018A0AB0BDEC028B70BD9FED088A1A
:10EFC000C2E7084831F076F8074831F073F800BF1F
:10EFD00050BD080020C0080000007A4480BC92C7E1
:10EFE0000000000028B1090020AF0900406820F0AF
:10EFF000030040F00200A0F1FF40704700B587B069
:10F000000C46082000211546039325F045FD094BC9
:10F010000360094E039A009605AB294620460193EA
:10F02000012327F0B3F8059852F0C0FE002030F01D
:10F03000FBFF00BFC4BD080030C008004068704737
:10F0400008B5054B1B6813B1044A934201D102482D
:10F0500008BD034831F006F850080120A056090009
:10F06000FCAE090008B5064BD3F8C03013B1054A11
:10F07000934201D1024808BD034830F0F3FF00BFBE
:10F0800050080120A0560900F4AE090010B500F0A8
:10F0900009F8044628B1002000F0BEF808B1083491
:10F0A000046010BD2DE9F843364F3D680446002D3D
:10F0B0005ED06B6805F1080823F003039844DFF87D
:10F0C000D0903148D9F80060002E14BFB64686466D
:10F0D000601C04BFAEEB0804083C3CB3A30725D179
:10F0E000002914BF3046284618B344F0010C01E053
:10F0F0000068F0B143686345FAD144608AB9BDE85D
:10F10000F8839AB1214DD5F88C317BB1012160464D
:10F1100025F0E6FC50B1D5F8DC300360C5F8DC0022
:10F12000446044F002044460BDE8F8830020BDE878
:10F13000F88304F1080CAEEB080363450FDA0029ED
:10F1400008BF3546002DDCD044F00101284602E01E
:10F1500000680028D5D043689942F9D1CDE751B174
:10F160002CF00300AEEB0000C9F800000660C4E715
:10F17000DFF82080A3E7C8F800504046C7F80080B9
:10F18000BBE700BF244E0120000004200C520120E8
:10F19000184E0120005D0120002211464FF0FF3083
:10F1A000FFF774BF30B58BB0154D164C6846F7F7B6
:10F1B00027FF2A68241A02F5806C012100220CEB3B
:10F1C0000400FFF763FF78B10F4B2A681A600368E9
:10F1D0000E4C53F8042C0E480E49236022F0030213
:10F1E000026019600BB030BD0246012104F5C84031
:10F1F000FFF74CFF044B4FF4C0421A60E7E700BF33
:10F20000F802012000000420284B0120885501202D
:10F2100084550120EF29780100B50E4B1968B9B16A
:10F220000D4B002808BF19460B1F01F1380CC1F126
:10F23000040101EB030E53F8042F824204D063450E
:10F24000F7D100205DF804FB034870445DF804FB2F
:10F250000149E9E70C5501200046012008B508687E
:10F260000AF0EAFF0E2008BD08B50AF0E5FF0E20FF
:10F2700008BD00BF38B51C46084611464FF00212C3
:10F2800026F0EEFE206852F091FD00210446082091
:10F2900025F002FC0D4B036063799BB123791F2B92
:10F2A00086BF03F01F030A494FF0A04103F5E07346
:10F2B000022241F82320054620790AF009FA6C6001
:10F2C000284638BD034830F0F5FE00BF34D30800AF
:10F2D000000300500CB3090008B5406809F070FF46
:10F2E000004808BD3233D3C010B5044684B040682E
:10F2F00009F066FF304B002201210320C3F8F0051E
:10F30000C3F8F425C3F800151146130103F1804337
:10F3100003F5E0430132082AC3F81415C3F81015A9
:10F32000F3D1254B4FF49052C3F8182561680122A0
:10F330004979C3F814150DF10200C3F81015C3F88C
:10F340002C06C3F830261A60D3F80021002AFBD01F
:10F350000022C3F80021D3F8002101921649019838
:10F3600001225A60D1F80431002BFBD00023C1F8F0
:10F370000431D1F8043102930F4A029801238B60C3
:10F38000D2F81431002BFBD00023C2F81431D2F88C
:10F39000141103910399C2F80035BDF90230002B16
:10F3A00006DB980080B2400040F0010004B010BDC0
:10F3B000012004B010BD00BF007000400E20704757
:10F3C0000E2070471C4608B5084611464FF0021241
:10F3D00026F046FE206852F0E9FC0021042025F0CA
:10F3E0005BFB0346024A03481A6030F03BFE00BF55
:10F3F000ACD308005CBF090008B543F03BFD00BF7B
:10F4000010B50B685C1C19D01F2B4FF001028ABF8E
:10F410003A4C4FF0A04403F01F0302FA03F3C4F880
:10F4200008350B681F2B86BF03F01F03334A4FF0CC
:10F43000A04203F5E073032442F823404B685A1CB2
:10F440000BD01F2B86BF03F01F032C4A4FF0A042A6
:10F4500003F5E073002442F8234003684A69C3F8C7
:10F4600024258B7E91F81BE091F819C0026843EACD
:10F470000E0343EA0C03C2F86C35D1E9004203687D
:10F48000C3F80C45C3F814254B7E012B00D010BDEA
:10F490008B685C1C0BD01F2B86BF03F01F03174A21
:10F4A0004FF0A04203F5E073002442F82340CB68FC
:10F4B0005A1C1BD01F2B4FF001028ABF0F4C4FF07C
:10F4C000A04403F01F0302FA03F3C4F80835CB6825
:10F4D0001F2B88BF03F01F0303F5E0738CBF074A9F
:10F4E0004FF0A042032442F82340CB6802688968A9
:10F4F000C2F80835C2F8101510BD00BF0003005057
:10F5000001B97047F0B511F0030683B01D4603D171
:10F510004F68FBB2934204D02B4603B0BDE8F040E5
:10F5200018473F0A08D00C1D019054F8041F0136FB
:10F53000A847B7420198F7D103B0F0BD2DE9F04FCD
:10F540002DED048B8DB007AB784C0193009405230F
:10F5500026F0B2FD0021079838F02CFF00218346E9
:10F56000089838F027FF81460021099838F022FFDB
:10F5700099F807200290012A40F0D480C279012A2C
:10F5800040F0D080D9F80810012940F2CB80826881
:10F59000012A40F2C780914240F0C4806621DBF826
:10F5A00008003AF0F1FDD9F81C4099F804100490D5
:10F5B000204638F0F3FFD9F80820D9F81800013AAE
:10F5C00000FB0240B0EE408A38F0E8FF0A98029B48
:10F5D0000E28DC69B0EE409A00F08E802CF0F4FC2E
:10F5E0000B980E28F0EE408A00F090802CF0ECFC96
:10F5F000F0EE406A029BDBF80820DB690393049B72
:10F60000D9F81C10DBF81C70DE696AB3CDF81490D1
:10F610004FF00008894609E0C6ED008ADBF80820B3
:10F6200008F10108424506F104061DD938469BF849
:10F63000041038F0B3FFDBF81820B4EEC08AF1EE06
:10F6400010FAF0EE407A1744E6DCB4EEC09AF1EE20
:10F6500010FA0FD5C6ED006ADBF8082008F10108A2
:10F66000424506F10406E1D804980DB0BDEC048BC8
:10F67000BDE8F08F059B9D68D3F818A01979013D6E
:10F6800000240CE004EB520202FB0A9038F086FFE3
:10F69000F4EEC07AF1EE10FA8CBF144615462A1B20
:10F6A000012AEFD80AFB049038F078FF05FB0A9096
:10F6B000F0EE405A38F072FF029B03999A6902FB00
:10F6C00004101979B0EE407A38F068FF039B05FB0F
:10F6D0000230B0EE406A38F061FF77EEE57A30EE46
:10F6E000460A37EE657A67EE807A87EE870A30EE53
:10F6F000066A86ED006A91E72046197938F04EFFD8
:10F700000B980E28F0EE408A7FF470AF029B986849
:10F710009A691979013802FB004038F03FFFF0EE9A
:10F72000406A67E7024830F0C5FC00BFE0CC080043
:10F7300058A109002DE9F04F2DED048B87B003ABE4
:10F74000594C01930094032326F0B6FC0398002142
:10F7500038F030FE8368012B70D9C579012D06463B
:10F7600040F09E80007938F0B7FE049BF7690E2BBD
:10F77000814669D00021184638F01CFEC579012D5C
:10F78000834640F08A80B26883689A4240F0858060
:10F790000079DFED468A38F09FFE82463846DBF876
:10F7A0001C40C847B36920461F44B0EE409AD0477A
:10F7B000DBF8183004EB0308B468012CF0EE409A33
:10F7C00028D93846C847B3694046B0EE498A1F4435
:10F7D000B0EE409AD047B0EE697A39EE088A30EE42
:10F7E000477AB0EE686A07EE905A97EE086AB468F6
:10F7F000DBF81830F8EE676A0135C6EE267AAC42BF
:10F800009844F0EE409A78EEA78ADAD8F6EE007ABD
:10F8100068EEA78A013C07EE904AF8EE677A67EE39
:10F82000A87A17EE900A20F0030040F00200A0F141
:10F83000FF4007B0BDEC048BBDE8F08F1C4807B05B
:10F84000BDEC048BBDE8F08F05982CF0BDFB38466D
:10F85000F0EE408AC847B468012C1BD9F7693179AA
:10F860009FED127A2A463846F0EE407A38F052FE82
:10F8700006EE902A70EE277AB8EE666A77EEC77ABF
:10F880000132C7EE866AA24237EE267AEBD168EEE5
:10F89000878ABBE79FED057AF9E7064830F00AFC56
:10F8A000054830F007FC00BF58C908000000000000
:10F8B000020080805CAF0900B8AE09001E280ED09F
:10F8C0003E280CD010F001030AD1820708D103684A
:10F8D000044A9B1AB3FA83F35B0918467047012365
:10F8E00018467047245F090008B50146FFF7E6FF98
:10F8F00018B901F00303022B00D008BD02480840EC
:10F90000063818BF012008BD070080FF70B54268A7
:10F9100032F0FF0582B004460B460ED0D4E9022136
:10F92000207927F0AFF8D4E901320E200132A3F597
:10F930008073C4E9013202B070BD2A460191017999
:10F94000402026F077FCA16862680831064600FB7B
:10F9500001F1082060F31F226260E06825F0D0F812
:10F960006268E0602946C2F31722A568013A06FBE7
:10F9700002F205FB0666304425F06CFD019BCDE7E5
:10F980002DE9F04106468CB00C461546242820D8B7
:10F99000DFE800F024242424241F1F1F1F1F1F1F23
:10F9A0001F1F891F131F1F1F1F1F1F1F1F1F1F5DCB
:10F9B0001F131F1F1F1F1F1F950012F0010040F093
:10F9C0008F8012F0030104D1814B12689A4200F03B
:10F9D0008780002420460CB0BDE8F081012209A9EF
:10F9E000204600F0B5F9012206A928462AF070F851
:10F9F000002870D00B9A012A00F0C1805A2A40F3E7
:10FA0000AA800021089B012B00F0BC805A2B00F338
:10FA1000BB802033934240F0948023F00203642B98
:10FA200000F08F80022E02D0002800F08A80DDE9ED
:10FA30000630DDE909120090304630F02BFD002839
:10FA40000CBF1E243E2420460CB0BDE8F08109A95D
:10FA50000122204600F07CF906A9284601222AF05E
:10FA60004BF89DF82C100022402026F0E3FBA16803
:10FA7000079E05469DF82C00B6FBF5F6314400F0D4
:10FA8000DFF90446DDE90912C06825F033FCE068BF
:10FA90000A9B069906FB05F2184425F02BFC20462C
:10FAA0000CB0BDE8F0814B4B0A689A4291D02946D0
:10FAB000204600F015F920460CB0BDE8F081012287
:10FAC00003A928462AF004F890B3A20703D1424BB9
:10FAD00022689A4242D01E2420460CB0BDE8F08134
:10FAE00028462CF0C7FA012209A90746204600F053
:10FAF0002FF9102EDDF8288048D0A1689DF82C0041
:10FB000007FB01F100F09CF9C5680446B8F1000F4D
:10FB10003FF460AF7E1E002F3FF45CAF099928468A
:10FB20004246013E25F0E6FB711C4544F6D151E703
:10FB3000EB0706D415F0030306D1254B2A689A4239
:10FB4000C9D1002030F070FA022BC4D1234B2B40D6
:10FB5000062BF6D1BFE72032014653E7012209A95F
:10FB60002046012400F0F4F8DDE90323DDE9090172
:10FB700000941EF003FA0028ADD03E242AE762224A
:10FB800001463FE7622345E7084643E72179002223
:10FB9000402026F04FFBA36807FB03F300FB03F1B3
:10FBA000E06824F0ADFFA36807FB03F3C4E902306B
:10FBB00063686FF31F2305466360002F3FF40AAFAD
:10FBC000013F4544B8F1000F3FF404AFA2E700BF86
:10FBD000245F090014600900005A0900070080FF33
:10FBE0002DE9F041012884B080460C4633D08B07C4
:10FBF0002AD020462DF030FB00284CD04510294655
:10FC0000404600F01DF900210646204629F0DAFFA3
:10FC10000024074638462AF0B1F948B165B90146D3
:10FC20003046FFF773FE38462AF0A8F90028F5D1D0
:10FC3000304604B0BDE8F08122460346F1684046F4
:10FC400026F020FF0134E5E70B68154A934202D005
:10FC5000144A9342CDD1012201A9204629F038FF50
:10FC60000028C6D041460022402026F0E3FA029B3D
:10FC7000B3FBF0F100FB01F4A3420ED1404600F0CB
:10FC8000DFF8019906462246C06825F033FB30466E
:10FC900004B0BDE8F0810546B1E7034830F00AFA48
:10FCA0003C5A0900005A090044A9090000B501287E
:10FCB00083B00B4608D084460022614607482EF0E8
:10FCC0000BFD03B05DF804FB0A6840F61623CDE98E
:10FCD00000234FF0020C6B46EEE700BFBC62090048
:10FCE00070B5044684B00846012201A929F004FF3A
:10FCF00000222179402026F09DFA6368029DB5FB21
:10FD0000F0F5B5EB132F0646C3F3172212D8521B9A
:10FD100062F31F23E0686360A368019903FB060098
:10FD200005FB06F225F0E6FAA3680E202B44A3603B
:10FD300004B070BDD4E90210294406FB01F124F09F
:10FD4000DFFE6368E0606FF31F236360E4E700BFDA
:10FD5000F8B5037904460D46164603F07F010022EC
:10FD6000402026F067FAE7682F60A1680E4A00FB82
:10FD700001F16960217901F07F01A9602168914258
:10FD800001D00020F8BD94F90420002A034603DBCB
:10FD9000B20701D50120F8BD6268C2F3172203FB48
:10FDA00002732B600020F8BD1460090010B4426893
:10FDB000C46891688C420CD20346D16810799A6865
:10FDC00022440134DC605DF8044B00F07F0026F033
:10FDD00047BB00205DF8044B704700BF084A002372
:10FDE000C1E90233C1E90020064B02689A4201D002
:10FDF000084670474368C3F317238B600846704773
:10FE0000BC5809001460090038B50C461D4611465F
:10FE100020460A4A26F024F928682EF031FC012CED
:10FE200005D069680078BDE83840FFF7D9BEBDE865
:10FE300038400078002100F003B800BF0400020041
:10FE40007828F8B520D005460E460022014640200D
:10FE500026F0F0F900210746102024F01DFE04468C
:10FE60000571866062680A4B6FF31F226260094A5F
:10FE7000012D18BF134606FB07F00021236024F074
:10FE80000BFEE0602046F8BD034830F013F900BFD8
:10FE9000005A090080580900C8A90900F8B50A7974
:10FEA000012A0C46064631D01F492FF0E7FFA36810
:10FEB0002BB930461D49BDE8F8402FF073BF1C49EF
:10FEC00030462FF06FFFA368B3B11A4F00252A46C2
:10FED000E168207926F0C4FA0122014630462DF06F
:10FEE00043FEA3680135AB4206D9002DEFD0394659
:10FEF00030462FF057FFEAE70F4930462FF052FF08
:10FF000030460A49BDE8F8402FF04CBF0B492FF0AE
:10FF100049FFD4E90221304630F0B4FF30460349AE
:10FF2000BDE8F8402FF03EBF0476080024730800B7
:10FF3000107608000073080014730800F8750800B4
:10FF40002DE9F04387B0002A37D011F003060446AC
:10FF50008C46154603D1874B0A689A4232D0A16875
:10FF600020680023624629F0D1FD834B2168994225
:10FF700002460ED0042D11D094F804C0E1682B463F
:10FF80000CF07F0026F07EFD0E24204607B0BDE871
:10FF9000F0836368042D00EB132208D12079E16817
:10FFA00000F07F0007B0BDE8F04326F059BA94F99D
:10FFB000043094F804C0002BE0DB0024204607B096
:10FFC000BDE8F08380686A4630F012FB002800F03C
:10FFD000CA802179042D324601F07F014FF04000A4
:10FFE0006ED026F027F915F00302064602D06348CA
:10FFF00030F01AF829688B881B0604D5604B886A94
:020000023000CC
:10000000984200F09B805F4B9942F0D1012E40F066
:10001000AD80324603A9284629F06EFDDDE903983C
:10002000554A2368E768DDE900019342A1EB00052A
:10003000A8EB050524D0002D2DDD6368B5EB132F4B
:1000400058D8A36840442B441A1A06FB017106FBDA
:1000500002F206FB007025F07DF9009806FB08F21D
:10006000494600FB067025F075F96368C5EB13225D
:1000700062F31F23A26863602A44A2600E2484E70F
:1000800094F90430002B98DA002D6FD16368C3F324
:10009000172306FB0377494606FB08F206FB0070B0
:1000A00025F058F90199A2680098521A404406FBBD
:1000B00002F206FB017106FB007025F04BF9D4E754
:1000C00026F0B8F82C4B22689A42054622D0DDE98A
:1000D00000312079C91AFFF7B3FEDDE90013E668A5
:1000E0005B1A044605FB03F205FB0161C06825F0BD
:1000F00001F94AE7A1682944384606FB01F124F0DA
:10010000FFFC6368E06065F31F2363600746DDE979
:10011000000196E73146102024F0BEFC054694E825
:100120000F0085E80F00009A02EB112060F31F21F9
:100130006960019B9B1A2C46AB6026E72979402019
:1001400001F07F0126F076F8B0420FD10A4A2B6801
:100150009342D5E902897FF464AF6B68C3F3172338
:1001600006FB03995DE708482FF05EFF07482FF074
:10017000A1FF00BF84620900146009005CAA0900A5
:1001800041FF02003C5A0900709C0900E89F0900E9
:10019000042808D0052804D18868400040F00100F8
:1001A0007047002070478B68002B14BF3E201E2034
:1001B000704700BF10EE102A22F00043B3F17E5FBB
:1001C00009D315D070EE407ADFED356A86EEA77A56
:1001D000B0EE470A7047B3F17C5F2FD2A3F500035E
:1001E000B3F1645F0DD2B0EE407AB0EE470A7047CB
:1001F000DFED2C7A9FED2C7AA0EE277AB0EE470A3D
:10020000704760EE007A9FED297A9FED296ADFED55
:10021000296ADFED295AA7EE876AB7EE007AE7EE82
:10022000866AA7EEA57A67EEA67AC7EE876AB0EE71
:10023000407AA0EE267AB0EE470A7047B7EE007A11
:10024000F0EEC07A77EE677AB6EE000A67EE807A53
:10025000DFED166A9FED166ADFED165A9FED165A0E
:100260009FED100AA7EEA66A002AA7EE857AE7EEB0
:10027000865AF1EEE76A67EEA57A9FED106AC7EE3F
:10028000875AB0EE005AE6EEA56AB0EE467AA6EEC0
:10029000857A30EE477A9BDAB1EE477A98E700BF6D
:1002A00000000000DA0FC93F000080036BD30DBCD3
:1002B000BA132FBD75AA2A3EAEE534BF6821A2B39A
:1002C00010B584B08DED010A019B23F00042B2F11C
:1002D0008B4F00EE102A4FEAD37425D25B000ED468
:1002E000B2F1665F27D2DFED1C7A70EE277ACDED92
:1002F000037A039B0CB1B1EE400A04B010BDB7EE17
:10030000007AF0EE476AE0EE006AB0EE006AF1EEC5
:10031000E67A77EE807AC7EE276AE0EE066AB0EEFC
:10032000660A24F0EDFAE5E724F0EAFADFED0B7A4D
:1003300030EE270ADEE720EE007AF7EE006A37EEAD
:10034000266AF1EEC67A77EEA67AC7EE276A36EE0F
:10035000800A24F01DFACDE70000807B1872313F3F
:1003600050B110B50E2884B0044603D000790EF0C9
:100370005BFA10B104B010BD7047204601A94FF4DC
:10038000FE7403AB02AA039420F000FE0399014817
:100390002FF098FE50C20900F4EE400AF1EE10FA78
:1003A000F0EE407A53D610EE902AB2F17E5F10EE56
:1003B000103A47D010B5940F04F0020444EAD37405
:1003C00033F0004308D1022C3ED09FED380A032CB5
:1003D00018BFB0EE670A10BD32F0004228D0B2F16B
:1003E000FF4F1BD002F15061994221D3B3F1FF4F6F
:1003F0001ED0A1072ED503F15063934243D29FED47
:100400002C0A022C46D0002CE5D09FED2A7ADFED95
:100410002A7A30EE070A30EE670A10BDB3F1FF4FBB
:1004200004F1FF3427D0022C1FD99FED210A10BD03
:10043000DFED227A9FED220A14F0010F18BFB0EE13
:10044000670A10BD00F044B89FED1B0A10BD30EEE6
:10045000800A704787EEA00AB0EEC00A00F038F8B4
:10046000012CCED1B1EE400A10BD164B03EB840433
:1004700094ED000A10BD022C15D8134B03EB840435
:1004800094ED000A10BD87EEA00AB0EEC00A00F09D
:100490001FF8B6E79FED077ADFED077A30EE070A1F
:1004A00037EEC00A10BD9FED090A10BDDB0F49C031
:1004B000000000002EBDBB33DB0F4940DB0FC9BF7E
:1004C000DB0FC93F1CB808000CB80800DB0F493F20
:1004D00010EE102A22F00043B3F1994F4FEAD27187
:1004E0000DD3B4EE400AF1EE10FA11D6DFED4B7ADF
:1004F0009FED4B0A002908BFB0EE670A70474948D4
:10050000834206D8B3F1665F39D212F0FF4F7DD037
:100510007047454A9342B0EEC00A4BD9434A9342D2
:100520006BD8F7EE087AB7EE006AA0EE276A70EE95
:10053000677A9FED3F7A9FED3F0AC7EE866A66EEC7
:10054000A65A9FED3D6ADFED3D4A9FED3D4A9FED86
:100550003D5A65EEA57AE7EE864AA7EE845A9FEDEE
:100560003A6AA7EEA46A67EE857AE5EE867A97EE98
:10057000A67A77EE667A30EE670A71BB704760EE56
:10058000006A9FED2D7ADFED2D5A9FED2D5A9FEDDC
:100590002D6A66EEA67AE7EE875AA7EE856A9FED8A
:1005A0002A7AA7EEA57A67EE867AE6EE877AA7EE34
:1005B000C00A7047A2F5D002934211D8F0EE007A3B
:1005C000BFEE006AA0EE276A70EE277A9FED1F7AD1
:1005D0009FED1F0AC6EE276AB1E7B1EE400A7047E9
:1005E000F7EE007A30EE676A70EE277A9FED197A9F
:1005F0009FED190AC6EE276AA1E7FFEE007AC7EE63
:10060000806A9FED167A9FED050A98E760EE007A02
:1006100082B0CDED017A019B02B07047DA0FC93F7D
:10062000DA0FC9BFFFFFDF3EFFFF973FFFFF1B4011
:10063000B40F14335E987B3F25AC7C3D0DF5113E25
:100640004712DABD98CA4CBEA9AAAA3E6937AC3196
:100650003863ED3E68212233DA0F493F6821A23327
:1006600000B585B08DED010A019B23F00042B2F187
:100670007C5F00EE102A4FEAD37023D2B2F13E5FC6
:100680000DD213F0FF4F04D160EE007ACDED037A66
:10069000039B08B1B1EE400A05B05DF804FB30EEF3
:1006A000007AF7EE007A77EEC07A67EE006A86EE9F
:1006B000A70A30EE070A24F06BF8F6EE007A20EE77
:1006C000270AE6E7F7EE007A77EEC07A80EE277A1F
:1006D00037EE070A24F05CF8F6EE007A20EE270ADF
:1006E000D7E700BF10B584460C46BCF1010F134696
:1006F000086888BF221D0CF1FF3198BF002246F028
:10070000BDFE206810BD00BF0C4B196899B130B414
:100710000B4B1B6800240E2503EB01119A688242E3
:1007200004BFC3E90044C3E9025410338B42F5D13E
:100730000E2030BC70470E20704700BF4C46012091
:100740004446012008B590F82330FF2B01D009F072
:1007500091FD0E2008BD00BF2DE9F04387B002AD2A
:100760002A4C01950846009411461A46042325F0A8
:100770000DFD029851F01AFB0746039851F016FB45
:100780000646049851F012FB00210546282024F06B
:10079000ABF91F4B03601F4B9DF81490D3F80080FA
:1007A000B8F1000F2FD104461860387908F090FF97
:1007B000307908F08DFF287908F08AFF164B3A79D6
:1007C00084F82120C3F86425327984F82220C3F804
:1007D00068252A7984F82320C3F870250122C3F8FC
:1007E0000485C3F80885C3F80C25C3F81025C3F8A1
:1007F0001C25C3F82085C3F824954BF085FC2046C2
:1008000007B0BDE8F08305482FF02CFC38C0080085
:10081000F8D508001C4E0120005002403CBA0900E7
:1008200008B5086890F82330FF2B01D009F022FDAD
:100830000E2008BD10B5044690F8230008F0E6FC31
:1008400094F8263013F0080F14BF3E201E2010BD70
:1008500010B5044690F8230008F0D8FC0A4BD3F8F2
:10086000082142B194F8262000216FF3410284F858
:100870002620C3F8081194F8263013F0020F14BF95
:100880003E201E2010BD00BF0050024010B504469F
:1008900090F8230008F0BAFC0C4BD3F8082142B1C1
:1008A00094F8262000216FF3410284F82620C3F833
:1008B000081194F826309A0705D543F0080384F808
:1008C00026300E2010BD00F003F800BF005002409B
:1008D00008B501482FF0C6FB30B409002DE9F04FF0
:1008E0002DED028B0C4689B054F8045B039206464A
:1008F00095F8230008F08AFC06AB01937F4B039A1E
:10090000009321460223701E25F0D6FB7C4B069CEB
:10091000D3F808119DF81C2041B195F826106FF30B
:10092000410185F826100021C3F8081195F82630FA
:100930009B070BD5724901234B6095F8263043F095
:10094000040385F826302023C1F8083395F82630B3
:100950006C6062F3041385F82630204603F00CFE29
:100960000346204608EE103A03F0B2FD05F12403D9
:10097000C00805AA85F825000121CDE900232046FD
:100980000DF113030DF1120203F0D2FD9DF81330A7
:100990009DF8120095F8261095F82520DFF8609153
:1009A000DFF86881DFF868A15B0143EA8013013A50
:1009B00003F0600321F0600143EA010318BF012244
:1009C00085F82630C9F81C2595F82430A3F10103D9
:1009D000B3FA83F34FF0000E5B09C9F82835B7EE80
:1009E000006A76467746F4460AE008EBCC034FEA05
:1009F000CC029B7953B90CF1010CBCF1090F32D038
:100A0000D9F81C35012BF0D04FEACC023D4B58F8F9
:100A10003C404244F8EE486A03F15800B2F9041031
:100A20009AFBF1F15A6891FBF2F207EE902AF8EE88
:100A3000E77AD3F800B076EEE77A0833F0EEE77A9B
:100A400087EEA67AB4EEC67AF1EE10FA04D5B0EECF
:100A5000476A96465E4627469842E3D10CF1010C60
:100A6000BCF1090FCCD1264CC4F81875C4F8146534
:100A700095F8243095F82500A5F81AE010FB03F04E
:100A800018EE103A03FB00F01F4B0001A3FB0030EF
:100A90008009033020F0030080B20021288323F076
:100AA000FBFF03460021AB60288B23F0F5FFE860D5
:100AB000686803F053FD95F8263023F00E030022FA
:100AC00043F002032846C5E9042285F8202085F872
:100AD000263020F03BFE2B8B01229B082021C4F8FE
:100AE0005035C4F80413C4F80025226020F00AFE33
:100AF0000E2009B0BDEC028BBDE8F08F98CD080048
:100B000000500240B41A0900D34D6210207409004D
:100B10000048E80110B5044690F8230008F076FB81
:100B200094F826301A0744BF6FF3C30384F82630C5
:100B30000E2010BD10B5044690F8230008F066FBA7
:100B4000064A0123536094F82630202143F0040321
:100B500084F82630C2F808130E2010BD0050024061
:100B600038B5084B1B6800220446C3F80025FF2552
:100B7000007943F045FC6079257143F041FC6571D3
:100B80000E2038BDFC0201202DE9F0438BB003ADEF
:100B9000404C01950846009411461A46072325F05B
:100BA000F5FA039851F002F90746049851F0FEF85F
:100BB00000210646082023F06FFF374B03609DF8A5
:100BC0001850DDF814806A075DD1089B5B0754D18B
:100BD000044609989DF81C90002848D02BF0F4F9A1
:100BE000B5EEC00AF1EE10FA44D4F7EE007AB4EE96
:100BF000E70AF1EE10FA3DDC387908F069FD30794A
:100C000008F066FD84F806903A79227133796371B1
:100C1000B8F57A5F34D1102D38D1204BDFED207A32
:100C20001B6820EE270AC3F840256579C3F84455B0
:100C30004FF00460C3F80405FCEEC07A0020C3F84E
:100C40002005012228211748C3F81815C3F81C15E0
:100C5000C3F80025C3F8600517EE900AC3F86425B1
:100C60001A6028F0FDFF20460BB0BDE8F0839FED31
:100C70000E0AC1E70D482FF01DFA0D482FF01AFAA1
:100C80000C482FF017FA0C482FF014FA0B482FF0ED
:100C900011FA00BF58C00800B0D60800FC020120BD
:100CA00000007A443C4B0120AE47E13DF0B509001D
:100CB00064B30900889C09007CBE0900989C090067
:100CC00038B5084B0C681B680022C3F80025207952
:100CD000FF2543F095FB6079257143F091FB657129
:100CE0000E2038BDFC02012008B50379FF2B02D08D
:100CF00047F6015008BD42F0BDF800BFF0B50379DA
:100D0000FF2B85B05CD0D40762D5551060D48B071B
:100D10000646084603D1314B0A689A4255D0022252
:100D200001A928F0D5FE10B90E2005B0F0BD9DF840
:100D30000C10029C0022402025F07CFAB4FBF0F05D
:100D4000A84248D3039B482B02D025482FF0B2F984
:100D5000244F019C3B680122C3F80825C3F8604575
:100D6000C3F86455204B4FF4485043F001039847B3
:100D70003B681E4A0021C3F80811C3F86025012210
:100D8000C3F86425D3F8083133B903F075FC3B6828
:100D9000D3F80831002BF8D04DB1A31E03EB450169
:100DA00033F8022FA2F5004299421A80F8D1B379A4
:100DB00043B925F00300400040F0010005B0F0BD4C
:100DC00042F058F825F00100F5E709482FF02CF91A
:100DD00008482FF05BF908482FF06CF9E46309002C
:100DE0000CA60900FC02012090F808003C4B0120F1
:100DF00078BC0900FCA5090044BA0900002343603F
:100E00000E20704710B4019CA4468468CCF80040C2
:100E100089B1817BB2FBF1FC01FB1C2290F80CC074
:100E200041685DF8044B4FEADC00D2B202FB0012CD
:100E30001A600020704742685DF8044B1A60002079
:100E4000704700BF4FF0010C82F800C0427B1A705F
:100E5000009A83681360019B09B190F80EC083F873
:100E600000C0704730B589B01E4C009405AD0846EF
:100E7000019511461A46032325F088F90021142014
:100E800023F00AFE184B036004460122059802A9CC
:100E900028F032FE049B622B1ED023F02002A3F127
:100EA0006801B1FA81F1482A4FEA511112D0422B60
:100EB00001D0012B13D108230398617302999DF887
:100EC00018202373079BA273C4E9011020462361F5
:100ED00009B030BD1023EFE708230121ECE70348F8
:100EE0002FF0E8F890C008007CD7080000C4090083
:100EF0000B6800220E205A60704700BF08B5436897
:100F000023B10069400040F0010008BD41F0B2FF8C
:100F100010B5436833B1044608462BF0ABF82061A6
:100F20000E2010BD41F0A6FF704700BF00234360B4
:100F3000C3600E20704700BF2DE9F04383B0044624
:100F40000A9E9846002970D1856B0F46226A636B12
:100F5000C2B9AB426FD0A28B01351544ED1AEB0735
:100F60004FD4E368C8F8003023693360002F4FD1B5
:100F7000A36B0133A363206A003818BF012003B0BC
:100F8000BDE8F083AB42E6D1E36A9A4228BF1A4635
:100F9000A38BD8074CBFE1686168C8F80010206BCC
:100FA00001AB0830914655F064F800284AD1019B06
:100FB000994547D1226AD21A22628AB913F00300F6
:100FC0000ED0A17E0344082901933FD0102907D1F8
:100FD000D8F8001023F00103194421F8022C019BDA
:100FE0003360A28BD1074CBF2361A3600132636BD6
:100FF00092B2013501331544ED1A6363EB07A28306
:10100000AFD56368C8F80030A3683360002FAFD055
:10101000012FB0D1E26BA17E0132E263D8F800303B
:1010200003EBD103C8F80030A5E7012A856B08BFA0
:10103000C56B17468AE71046C8F80020326003B037
:10104000BDE8F083022003B0BDE8F0834FF0800ECE
:10105000D8F800106FEA020C0B44013203F80CE0E0
:101060009042019BF4D1BBE74FF0000C82F800C026
:10107000827E082A94BF002201221A70009A4FF43F
:1010800000731360019B19B190F824201A70704707
:1010900001221A70704700BF70B50D4684B011462A
:1010A00028461D4A1E4624F0DBFF0021402023F085
:1010B000F3FC1A4A0260316811F0030220D1184B88
:1010C0000446086898421BD1012D06D820461346D5
:1010D00009F0FEF8204604B070BD022201A9706834
:1010E00028F00AFDDDE90123A3F10801B1F57E7FB7
:1010F00009D82046316809F0EBF8204604B070BDED
:1011000008482EF0C3FF08484FF48063082240F2DD
:10111000CA212EF0D7FF00BF0400020078D80800D3
:10112000E4630900E8A409002CC209000B6800224E
:101130000E205A60DA60704710B50446406808F027
:101140006BF8A07E400040F0010010BD10B50446D1
:10115000406808F061F894F82400400040F0010075
:1011600010BD00BF10B50446406808F055F8A06AED
:10117000400040F0010010BD38B50D4604464068FF
:1011800008F04AF828462AF075FFA0620E2038BD04
:1011900038B5044609B1012A0BD0206B636923627C
:1011A0000025228B08302B4654F036FCC4E90D553F
:1011B000E56338BD0023C0E901330E20704700BF4E
:1011C0002DE9F04F2DED028B89B0CDE90423149C5D
:1011D000C3690646C9B9F2682260B26904919A42AD
:1011E0001CD0737C002B00F0DD80059AB36813607F
:1011F000049B002B40F0C380F3690133F3610120AD
:1012000009B0BDEC028BBDE8F08F049A012AF268A8
:1012100008BF036A2260B2699A42E2D17368727CA5
:101220001946B368002A08BF1946059A069111604D
:10123000737C96F8242083F001037374F3689B0891
:101240000393002A00F0A381002306F128010193F3
:1012500002914FF0802B9A46029B53F8044F029361
:10126000A368002B64D0039B002B5FD02346069F0E
:1012700053F8140F039D08EE103AD8B9637B33B9C5
:10128000237B002B00F07481A06803F067F9A0684D
:10129000002800F0B48018EE102A04F1100103F0C9
:1012A00033F9A0F10100B0FA80F040096073606981
:1012B00080086061854229462369B4F818E096F8F1
:1012C00010C028BF0146BAF1000F6FD1BCF1100F5A
:1012D00040F0978096F812C0BCF1000F00F02A8110
:1012E000C9B14FEA0E42043BA7F1040ED44653F8AD
:1012F000040F32FB00F832FB10F028F3CF3820F354
:10130000CF30C8EA00400CF1010C61454EF8040FE3
:10131000EDD1D4E9043003EB8103401A6D1A236147
:10132000606107EB8107A8D196F824204FF0010AED
:10133000019B01339A4201938EDCBAF1000F00F059
:101340002681B37CA3B9337C102B039B00F02E8144
:1013500073B1069B039903EB8102043A043B4FF0FF
:10136000803053F8041F81FA40F193421960F8D19C
:10137000B3690133B361049B002B3FF43DAF049B81
:10138000012B7FF43CAF336A0599327C0133336221
:101390000B68012003EBD2030B6009B0BDEC028B9C
:1013A000BDE8F08F059A7368136021E7BCF1100F58
:1013B0005CD196F812C0BCF1000F00F09A800029B1
:1013C000A9D04FEA0E42043BA7F1040E4FF0000CE7
:1013D00053F8048F32FB08F032FB18F820F3CF30BB
:1013E00028F3CF38C0EA08405EF8048F90FA18F06E
:1013F0000CF1010C6145CEF80000E9D189E7606984
:1014000058E74A00944686D04FEA0E42CDF81CA019
:10141000D646023BA7F102088A46E14633F8020F9E
:10142000B17C4FEA004C00020CF07F4C80B24CEAD9
:10143000000009B990FA4BF032FB00F132FB10F0DA
:1014400021F3CF3120F3CF30C1EA0040010C01F489
:101450007F41C0F307200EF1010E0843CE4528F866
:10146000020FDBD15146DDF81CA052E74A0094463A
:101470003FF451AF4FEA0E42CDF81CA0023BA7F15A
:1014800002084FF0000E8A46E14633F8020FB17CA5
:101490004FEA004C00020CF07F4C80B24CEA000096
:1014A00009B990FA4BF032FB00F132FB10F021F356
:1014B000CF3120F3CF30C1EA004C38F8020F0104DD
:1014C000000280B201F07F4101439CFA11FC4FEA17
:1014D0001C4101F47F41CCF3072C0EF1010E41EACF
:1014E0000C0CCE45A8F800C0CFD15146DDF81CA0A9
:1014F0000FE700293FF40FAF4FEA0E40043BA7F17E
:10150000040E53F8042F92FA4BF230FB02F830FB32
:1015100012F228F3CF3822F3CF32C8EA02425EF843
:10152000048F92FA18F20CF1010C6145CEF80020FC
:10153000E7D1EEE600293FF4EEAE4FEA0E42043B5F
:10154000A7F10408D64653F8040F90FA4BF032FB8B
:1015500000FC32FB10F02CF3CF3C20F3CF30CCEA70
:1015600000400EF1010E714548F8040FEBD1D0E6B2
:10157000A060BAF1000F7FF4D7AE002D4FEA8502CC
:10158000514608BF0422384623F064FFCCE6039B93
:10159000002B3FF4D6AE039B06989A00002123F05F
:1015A00059FFB37C002B7FF4E3AECCE6002B3FF475
:1015B000DFAE069A02EB83010439131F4FF080203F
:1015C00053F8042F92FA40F299421A60F8D1CFE60C
:1015D0004FF0000C82F800C0827C1A70009AC36839
:1015E0001360019B11B1C27C1A70704701221A70FE
:1015F000704700BF2DE9F047084688B011461A46EB
:10160000384B02ACCDE90034062324F0BFFD029F25
:101610007B1EFE2B50D8049B5A1E012A5FD8079EC2
:10162000002E59DD059D082D01D0102D51D107F157
:101630000B00002180005FFA83F823F02DFA2A4B7B
:101640000360044603989DF81890C0088000E0608D
:10165000002123F021FAEDB2034660605FFA87FAB9
:1016600090B3E068002123F017FA0346A06030B37E
:1016700084F81380DFF890802574666184F81290F6
:1016800084F824A004F12806002500231A461946F0
:10169000404600F0D9F80135AF4246F8040F4460E7
:1016A000F3D194F8240004F12C012CF0BFF9A062CE
:1016B000204608B0BDE8F0870C482EF0FBFC0C4932
:1016C0000C4863602EF026FD0B490A48A3602EF0FB
:1016D00021FD0A482EF0EEFC09482EF0EBFC0948EB
:1016E0002EF0E8FCC8C0080084D908009CB60900A8
:1016F000D4BA09004C560900F0BA0900A4A909009F
:10170000C4B1090044B7090054DA08000B6800228C
:10171000C3E901220E20704710B5044607F082FD90
:1017200094F824208AB1013AD3B204F12C0204F1D6
:10173000280002EB830201E0904206D050F8043FFB
:101740009B68002BF8D03E2010BD1E2010BD00BFAE
:1017500010B5044607F066FD6069400040F00100E6
:1017600010BD00BF10B5044607F05CFDA06A10BDB7
:1017700070B50C4688B054F8045B039206462846C0
:1017800007F050FD05AB01930D4B039A00932146E2
:101790000323701E24F090FC95F824209DF8183047
:1017A0009A420AD905EB83059DF81C20E86A059941
:1017B00008F05EFE0E2008B070BD02482EF07AFCE4
:1017C00078CE0800A8B6090070B50C4686B054F86B
:1017D000045B03920646284607F024FD05AB0193FF
:1017E0000C4B039A009321460123701E24F064FCE5
:1017F00095F824209DF814309A4207D905EB83050B
:101800000022EB6A0E209A6006B070BD02482EF0EE
:1018100051FC00BFA8CD0800A8B6090090F82430FC
:1018200083B1002210B41346144600EB8303013247
:10183000D96A8C6090F82410D3B29942F5D85DF83B
:10184000044B7047704700BF10B508461146002290
:1018500024F006FC00211C2023F01EF9034C046038
:1018600000214FF400428160028310BD54DA080069
:10187000008B07EE900AFBEEE87A17EE900A20F054
:10188000030040F00200A0F1FF4070478368002B86
:1018900014BF3E201E20704710B584B002AB51F833
:1018A000044B0193074B00930138022324F004FCFE
:1018B00020469DF80C20029908F0DAFD0E2004B0B5
:1018C00010BD00BF90CE080010B584B003AB0193EB
:1018D000124B51F8044B00930138012324F0ECFB28
:1018E00003982AF071FBF7EE007AB4EEE70AF1EE06
:1018F00010FA10DCB5EEC00AF1EE10FA0BD4DFEDF1
:10190000087A20EE270A0E20BCEEC00A10EE103A2C
:10191000238304B010BD03482EF0CCFBF8C00800B0
:1019200000000047F49F090010B584B003AB019399
:10193000064B51F8044B00930138012324F0BCFB03
:1019400000230E20A36004B010BD00BF60CA0800D1
:1019500008B508F03FFE0E2008BD00BF2DE9F04F8E
:101960002DED028BC7B01D908069002801F03C86E8
:1019700081B311461D9C529D206B286094F93F0055
:10198000884229D01D9890F83C10B1FA81F149099C
:10199000C2F1010280F83F2000EB810280F83C1088
:1019A00080F84010526A1A600446219224F0C4FA6A
:1019B000204624F061FA28BB529B186094F83E3010
:1019C000002B204614BF0020022047B0BDEC028B44
:1019D000BDE8F08F0A46CDE794F9401004EB810191
:1019E0000120496A01EB4202FF211A6084F83F108E
:1019F0002A68636C03EB5203636447B0BDEC028B4F
:101A0000BDE8F08F1D9AD2E90634156A03EB05088C
:101A100053680B93621B1E460592002B00F048830F
:101A20004146184653F034F9021E0492C2F267820E
:101A3000366808EB02030393002E02F05C820B9BD6
:101A4000D3F804A0BAF1000F02F055823378002BCE
:101A500000F03683337F032B039B2F932FAB1C4661
:101A600014BF4FF0110B4FF0090B082108EE103A8C
:101A700020460023CDE93033CDF808B0CDF8C8B00A
:101A800052F0E2FDCAF80000337F032B0CBF0121A6
:101A90000221204652F0D8FDCAF804000B9BD3F86F
:101AA000C457002D1A467CDDCDE9068AD3F8BC3731
:101AB00018EE108AD14600279246002B6ADD4C466C
:101AC00000250C21404652F0BFFD0921A06240468E
:101AD00052F0BAFD0821E062404652F0B5FD2063A5
:101AE0003378002B0CBF04210921404652F0ACFD95
:101AF00001216063404652F0A7FDA063002801F079
:101B000002830221404652F09FFD0121E0634046DE
:101B100052F09AFD05212064404652F095FD0521C2
:101B20006064404652F090FD0023E364A06403210A
:101B3000404652F089FD03212065404652F084FD65
:101B400003216065404652F07FFDE36BA065002BEA
:101B500041F05F84C4E90A336363E36DC3F11403A6
:101B600023663378002B01F0ED82002060660121AE
:101B7000404652F069FD0121A066404652F064FDE6
:101B8000E066DAF8BC3701359D4204F1480498DB81
:101B9000DAF8C4570137AF4209F190098DDBDDE96E
:101BA000068A039B0B9A04990298DAF80070C2F82F
:101BB000D8775B440C189B460599D2F8B8370C1BB4
:101BC000002B01F0B084D2F8B037002B41F02F8504
:101BD000D2F8CC279442C2F2BA810B9DD5F8DC37FB
:101BE000BB42C2F2968129461C31DB1B0E463A46A7
:101BF00005913046194423F0ADFBD5F8D807D5F848
:101C0000CC275946304423F075FBD5F8CC37D5F8AE
:101C1000D827E11A1344C5F8DC37DB000693D5F862
:101C2000C4372391002B41F3C5800B9A002302F5A2
:101C3000FC62CDE924322293029308930B9BD3F8E4
:101C4000BC37002B40F3E083089A2499C2EB42137F
:101C500052019B001F92229A2093443100230F923D
:101C6000259A149316911A9203930B9B1C68002CCF
:101C700000F015825A680492002A00F01082D3F80E
:101C800008B0BBF1000F00F00A82059B27930023E8
:101C9000CDE92833069A029B9A18D31D48BF02F15A
:101CA0000E03DB102A93029B002B41F0F78123786F
:101CB000002B41F0E180089E039F06EBC60307EB73
:101CC000C7021B0103EBC203049A1344B74A586BC3
:101CD000D96B12F8108002EB4004FA000A92022934
:101CE0004FEAC60265780D9201F08782089B002BAF
:101CF00001F0FB82039B049A1B010833D718D358C9
:101D0000002B01F0128314990F9A4B1E013A0BF12C
:101D100005005B445A44084413F8011F02F8011FF0
:101D20008342F9D17B68002B01F01383089A1F9B33
:101D300003989B1A9B00C0EB401203EB42030BEB92
:101D400042025B4491799971D179D971117A1972F2
:101D5000517A5972927A9A72BB684FEA4018002BF6
:101D600001F00E8314990F9A0B460B330B320BF1D3
:101D700010005B445A44084413F8011B02F8011B8D
:101D80008342F9D1FB68002B01F00E8314990F9A5E
:101D90000B46103310320BF115005B445A440844D3
:101DA00013F8011B02F8011B8342F9D1039B089A27
:101DB000A8EB03081F9B9B1A9B0003EB48039B4463
:101DC00000238BF815308BF816300D9B089A039979
:101DD000059C9A180A9B12010B4402EBC302049B58
:101DE0001344996A1A9B43F8041B1A93279B181BE8
:101DF000299BC3EBC003029804EBE304181A109468
:101E000003F0070417940C1A0294069C002BA4EB11
:101E100000001B90C0F24381A14200F340810B9B64
:101E20001968002900F03B815C6813941846002C67
:101E300000F035819B68002B00F03181C368189356
:101E4000002B00F02C81029B002BC0F22881224441
:101E5000936B1BB1D36B022B01F01F82089A0D9B71
:101E60000398496B13440A9A1B01024403EBC20313
:101E7000139A1344D3E9172301321344013331F980
:101E8000122031F9131008980D9B039C139D189E86
:101E900003440A981B01204403EBC0032B4406EBC8
:101EA0000020DB6A15905B00B3F5107FA8BF4FF4EC
:101EB00010739942A8BF19469A421846A8BF1A46FD
:101EC00032931E9306EB8403319103F58051002376
:101ED0002F930C9330AB0793169B3092EB1809931A
:101EE000179B0693109B1C91C1F800020593079A5B
:101EF0000C9E52F8043B0C93981B0028079240F369
:101F00009E81029B002BC0F2CA80099BDFF8A09043
:101F10001968069B059D159C5A4209EBC10312F0F6
:101F200007021F791DBF15F801CBC2F120030CFA7F
:101F300003F3134604EB8606002F00F09187DFF8C9
:101F400074C0029C5CF82180DFF86CC0012FA4EB08
:101F5000020B0CEB480E01F02880A7F1020CBCF13B
:101F6000010F00F29C8059F831100E914C1CBBF10E
:101F70000F0FC1F1200111944FF000091291BA46E0
:101F800074464DDD6F7815F802CB0495C2F1180147
:101F90000CFA01F1C2F1100C07FA0CF70F43ABF188
:101FA000100B3B4310320A2A36DD07E038B908002F
:101FB0002CD109002CD20900ACD20900278807F0E7
:101FC0000F07C7F1200123FA01F1013134F8111094
:101FD0005FEA113C00F0B380C1F30317C1F303249F
:101FE0000F2FA2EB0C0203FA0CF321463DD0002F79
:101FF0003ED10F2C46D0002940F0A6804A454EDB4A
:1020000002383446002844F8087B716041F3858229
:102010000A2A26467446D1DCBBF10F0F049DB1DCC1
:102020000BEB020100293ADDBBF1000F06DD15F8CC
:10203000017BC2F1180C07FA0CF73B43BBF1080F08
:1020400005DDC2F1100715F8012BBA4013434A1EF3
:102050004FF0004747FA02F213404FF00B0901F12D
:102060000B024FF0000B04959DE7BAF1030F6DD002
:1020700003F0004C0F2C02F1FF324CEA07074FEA45
:102080004303B8D1BAF1030F00F09F80013A03F087
:1020900000414A4541EA04014FEA4303B0DA21997D
:1020A0000B98F7F7A3F91D9A2399D3695B1A13626A
:1020B000529B0020186047B0BDEC028BBDE8F08F4A
:1020C000337F032B039B2F932FAB14BF4FF0200BB9
:1020D0004FF0110B0921002518461F4608EE103A53
:1020E000CDE93055CDF808B0CDF8C8B052F0ACFA13
:1020F000CAF80000337F032B0CBF052103213846AB
:1021000052F0A2FA0B9BCAF80400D3F8BC37AB42DA
:102110007FF7C4AC0AF11804A4F110090121384674
:1021200052F092FA49F8040BA145F7D10B9BD3F872
:10213000BC3701359D4204F11004EDDBAEE404EB45
:102140004104D21BBB402EE70C469FE7119D02EBDA
:102150000B0C002C18BF013565452F469FDCAA42A9
:1021600081F2BB806FEA020C6744FD0805F10108AB
:102170001995049DC2F1180CA84415F8017B07FAC3
:102180000CF7454543EA0703ACF1080CF5D1199D5E
:102190000832ABF1080B02EBC502C5EB45751BEB32
:1021A000C50B08D55A44551E4FF0004747FA05F5B0
:1021B0002B404FF0000B129F0E9DCDF8108023FA9C
:1021C00007F7521B0F37AB4011E7119C02EB0B01D5
:1021D0008C423FF764AF944241F383800E99049D93
:1021E000A1EB02084FEAD80808F1010CAC44C2F197
:1021F000180415F8011BA140654543EA0103A4F149
:102200000804F6D10832ABF1080B02EBC802C8EBA8
:1022100048781BEBC80B08D55A44511E4FF00044B8
:1022200044FA01F10B404FF0000B12990E9CCDF8CF
:1022300010C023FA01F1121B0F31A340DBE600238B
:1022400002998B423FF72BAF069A1A44CB1A02939E
:1022500002F007030693059B03EBE2030593099B3A
:1022600004330993079B33AA9A427FF440AE029B42
:10227000002B40F32D87089A0D9B0399DDF814A0DD
:1022800013440A9A1B010A4403EBC203139A1A442B
:10229000D36E8B4A52F823008A4A52F82340069B99
:1022A000594211F0070100F010871AF8015BC1F1E3
:1022B000200205FA02F21E9B029DC3F50F7E0EF16D
:1022C000010EBEF1000FA5EB010B40F30187159D38
:1022D000C4F120097C4C4FF0000C05EB830304EBA8
:1022E00000086746BBF10F0F40F394859AF8014050
:1022F0001AF8020BC1F11805A840C1F11005AC4055
:102300002043ABF1100B0243103103F1100003E046
:10231000092900F11000E5DD22FA09F318F803306D
:102320001C0913F00806A1EB131102FA04F205D000
:1023300002F00046013946F00106520013F0040590
:1023400005D002F00045013945F00105520013F0B7
:10235000020405D002F00044013944F001045200A7
:1023600013F0010305D002F00043013943F00103EB
:102370005200614507DB0437BE4540E9024340E9AE
:1023800004650346C4DC1C9AD2F800323B44B3F522
:10239000107FC2F800320DDA03990A9A0A4403EB5F
:1023A0008210189AC3F5107302EB800000219A0086
:1023B00023F050F8029B069A1344059A02EBE302BD
:1023C00003F007030293109BD21A3FF568AE179BE8
:1023D0001099C3EBC2031144029A059113441B9A4E
:1023E000D31A0693169B039A48331693149B3E33D5
:1023F00014930F9B3E330F930B9BD3F8BC370132E2
:102400009A420392FFF631AC0B9A12680792002AA7
:102410003FF445AE0B994A68002A3FF440AE886805
:10242000149000283FF43BAEC868139000283FF496
:1024300036AE09690E9100293FF431AE002B40F30E
:102440004D81249B5033D3181193229B149A013B46
:10245000D318179300231693139B0F9303F59052F1
:102460000E9B0C921593119B53F8143C022B01F018
:1024700017810D2309934FF01608119A179ECDF876
:10248000288000232F93936952F8202C1092013357
:102490005B000393079B0D4D1B6ADDF81C800496BF
:1024A0005B0804BF02321092109B4FF0000BC3F187
:1024B000D209CDF834905C46DDF84490DA4632E03B
:1024C00038FA090030FA090040FA0900A47009003E
:1024D000D8F83430049E03EB440233F91430B2F9D7
:1024E0000220D21A0F9B03EB8A0116F8013F0496D3
:1024F000D9F81460671C9244084616B195F800C0DC
:1025000063440D9EB446039E03FB06C3F5F7ACFE81
:1025100001354BEA000B00B92F9C0C9B2F941B68D4
:102520009A4504DA3C460A9B9C42D1D12F9C159BCC
:102530000021C3E9C811C3F82C43C3F81813C3F82A
:102540001C13C3F82813099B0B2B01F39B80109BD2
:10255000169A09993191C3F1D2030A93229BCDF8BF
:1025600010A0C2EB4212173303EB420301EB41020E
:102570001344149ACDE92F11D3180D93079B099A90
:102580005B6B109203EB420301320992B3F93020E6
:10259000B3F92E300499DDF83880DDF834A0DDF889
:1025A0004490D21A0F9B18EE106A03EB8104274661
:1025B0001294950014460A9A59F8043B1AF8011B24
:1025C00002EBC303039A384602FB0133414622461D
:1025D000F5F74AFEA8442F444BEA000B08B1109BC4
:1025E0003360043632ABB342E5D122460499129CE3
:1025F00002EB42031944002A04914FEA420119DD1B
:1026000002F1804301F180410E9A013B013902EB56
:10261000830302EB8101043A154452F8040F206051
:1026200053F8040F606051F8040FA060954204F164
:102630000C04F2D10C9B049A1B689A4281F22E8101
:102640000D9B03330D93099B0D2B97D1DDF810A043
:102650000C9B159AC3F800A0119B53F8103C002B5B
:1026600014BF02230123C2F818332F9BC2F81C3376
:102670001146309AC1F820239342B8BF1346319ACD
:10268000C1F824239342B8BF1346BBF1000FC1F831
:10269000283301F0F980C1F2D58300235FEA4B0BA8
:1026A0001A4603F10103F9D50C9B9A6004330C938D
:1026B000159B169A183315930F9B03F510630F9310
:1026C000119B48331193179B3E3317930B9BD3F801
:1026D000BC3701329A421692FFF6C5AE079A146AC9
:1026E0002146002C40F0FB87002B40F39981249B6E
:1026F0002833099300231C460B9B1B68002B3FF4D7
:10270000CEAC0B9A55680A951146002D3FF4C7AC24
:10271000D6680396002E3FF4C2AC52690C92002A90
:102720003FF4BDAC1A78089F5B6B002A0CBF0821F0
:10273000062107EBC70233F91130AC49120104EB53
:10274000C40002EBC0022A4481FB0351DB17C3EB38
:10275000A1031BB20793D36BE1001091022B4FEA48
:10276000C7010F9100F0AF8604F5906340F2262276
:1027700056F82330934240F3898620232F93030297
:102780000D9306EB0023049340F236230E934FF093
:102790001F0E049BDFF870C2954F964E11940EEBFE
:1027A000CE0E03EBCE0ED3E91102934C014684FB0F
:1027B000018190468CFB0898A1EB080149005964FF
:1027C00084FB021201468CFB0101186C0A4404F1DF
:1027D0004674520004F525349A640146DA6C04F517
:1027E0007D7484FB0181854D904685FB0898A1EBA3
:1027F00008014900196484FB0212014685FB0101AE
:10280000D86B0A445200DA6401461A6D87FB0181D5
:10281000904686FB0898A1EB08014900D96387FB25
:102820000212014686FB0101986B0A4404F15064D0
:10283000520004F5A9441A6501465A6D433484FBDD
:1028400001816F4D904685FB0898A1EB0801490076
:10285000996384FB0212014685FB0101D3F83480A1
:102860000A4404F1C774520004F5F0345A65414635
:102870009A6D103484FB01016248914680FB09A9DE
:10288000A1EB09014900596384FB0212414680FB18
:102890000181186BDFF874910A4452009A65014671
:1028A000DA6D89FB0181DFF86881924688FB0ABAFC
:1028B000A1EB0A014900196389FB021288FB001091
:1028C0000244D86ADFF84C915200DA6501461A6E6C
:1028D00089FB0181DFF84081924688FB0ABAA1EBAF
:1028E0000A014900D96289FB021288FB00100244E8
:1028F000986A520009F545391A6609F131095A6E8C
:10290000014689FB0181DFF81481924688FB0ABAEF
:10291000A1EB0A014900996289FB021288FB0010B1
:10292000024452005A6648339E457FF43CAF119CE6
:10293000039B089A0C9803EB840C0F9B1344109A8A
:102940001D01224405EBC20511460A9A05EB020857
:10295000099D0CF5805C2E464836531909960E9D4C
:10296000DCF800620D9AB542B8BF3546CCF800528B
:102970002E461E4D113600EB840785FB065EF617CA
:1029800007F58057C6EBAE063096D7F8006B319648
:10299000D7F8086B3296D7F8106B3396D8F84060AA
:1029A000002E079E08BF002600EBC1113496DCF80C
:1029B00008628DED008A024401F590510498359625
:1029C000F5F700FFC7F8000BD8F83C30C7F8083B14
:1029D000349BC7F8103B369BC7F8183B0B9BD3F8CA
:1029E000BC3701349C42FFF687AE19E0398EE338DC
:1029F000736E8D794A3FE3D7F053C26D49499EC348
:102A00007611B7E82FFEE4F3AA0025BE407EE47FEE
:102A1000C7A3C1FA63B2FC7FC6BD2EFE5DC286FFAE
:102A20000B990898D1F8C82702FB00F5219A03FBFF
:102A300005F502EB4505CA68002A3FF430AB0A46AB
:102A400049690C9100293FF42AAB92690D92002A42
:102A50003FF425AB022B01F00F8205F140030493F4
:102A60000D9B03F500530993D3F800220C9B002122
:102A700003F5805307910E9388464FF000794FF08D
:102A80000C0A0E9B0D9D07980C9CD3F8183B0093E5
:102A9000294600F0010304EBC0101E460A9351F0D2
:102AA00061FA0998D0F8003206EB061203EB8213A4
:102AB00005EB830455F82300E16D4B464246C0FB0D
:102AC00008326FF07300C1FB00324FF4557C606830
:102AD000A16DC0FB0C32C648C1FB003241F6D47771
:102AE000A068616DC0FB0732C248C1FB003246F2EC
:102AF000B865E068216DC0FB0532BF48C1FB0032FC
:102B0000BE4E2069E16CC0FB0632BD48C1FB0032FD
:102B10006069A16CC0FB053245F28400C1FB003244
:102B2000A069616CC0FB073240F22C70C1FB00321F
:102B3000E069216CC0FB0C327420C1FB0032142010
:102B400002FA0AF142FA00F223FA00F343EA01031F
:102B50005915B1EBE37F4FEAE37218BF82F4FF43EC
:102B6000049A0CBF9B1183F07F0304F5805022F878
:102B7000403C03684FF4D07549464246C3FB0512FA
:102B800041F67C054368C3FB051249F2FC75836876
:102B9000C3FB05129B4DC368C3FB05129A4D0B4640
:102BA0000169C1FB05326FF0B3054169C1FB053214
:102BB0004FF412758169C1FB0532C1696FF01300D2
:102BC000C1FB0032142002FA0AF142FA00F223FAA1
:102BD00000F343EA01035915DA17B1EBE37F18BF9D
:102BE00082F4FF43049A894D03920CBF9B1183F03A
:102BF0007F036FF0030722F8203CA2F1400E682605
:102C0000BC4601E055E910C6D4F800B1D4F85C71B7
:102C10004A464046CBFB0C204B464146CBFB063197
:102C20007642C7FB0620C7FB0C3155E90E7CD4F871
:102C300004B1D4F85861CBFB0720CBFB0C31CCF1AD
:102C4000000CC6FB0C20C6FB073155E90C7CD4F800
:102C500008B1D4F85461CBFB0720CBFB0C31CCF18D
:102C6000000CC6FB0C20C6FB073155E90A7CD4F8E2
:102C70000CB1D4F85061CBFB0720CBFB0C31CCF16D
:102C8000000CC6FB0C20C6FB073155E908CBD4F875
:102C90001061D4F84C71C6FB0C20C6FB0B31CBF194
:102CA0000006C7FB0620C7FB0C3155E906C6D4F861
:102CB00014B1D4F84871CBFB0C20CBFB0631764223
:102CC000C7FB0620C7FB0C3155E904C6D4F818B180
:102CD000D4F84471CBFB0C20CBFB06317642C7FB0A
:102CE0000620C7FB0C3155E902C6D4F81CB1D4F854
:102CF0004071CBFB0C20CBFB06317642C7FB062094
:102D0000C7FB0C31142700FA0AF640FA07F022FA42
:102D100007F242EA06025615D017B6EBE27F16BF5D
:102D200080F4FF42921182F07F022EF8022F1420CD
:102D300001FA0AF241FA00F123FA00F343EA02032E
:102D40005915DA17B1EBE37F18BF82F4FF43039AFA
:102D50000CBF9B1183F07F0322F8023D2C4B0392A2
:102D600040359D4204F580747FF44CAF049B099874
:102D700007990A9A40330493D0F8003201319B1A24
:102D800003F0070212290791C0F800227FF479AE00
:102D9000249B089A90332493229B7C332293259B77
:102DA000083325930B9BD3F8C43701329A4208921B
:102DB000FEF644AF1D9C2398E269636C121A2262EE
:102DC000529A126803EB52036364204623F0B4F86E
:102DD000204623F051F8236AB3F5007F044680F0C3
:102DE0007384204647B0BDEC028BBDE8F08F00BF76
:102DF000D4F8FFFF7CAFFFFF3CB6FDFF78940400E2
:102E0000C44902004CE803002464FFFF90F6090067
:102E100050FA09000BEB010000287FF7B4AABBF1C0
:102E2000000F06DD1AF8015BC1F1180405FA04F47D
:102E30002243BBF1080F05DDC1F110041AF8011B94
:102E4000A1400A43411E4FF0004444FA01F10A40F8
:102E50004FF00A0C00F10A014FF0000BFFF755BAD2
:102E6000331D002246F8272043F827200237B842B6
:102E7000F7DC069AFFF7EFB9226A089C039804EB87
:102E8000C40300EBC0011B0103EBC10304990B4415
:102E90000146C0000A9012F001024FEAC4005B6BC9
:102EA0000D9002D0012900F0CF82B3F5C87F80F2E7
:102EB0001281A74C181184FB0014D917C1EB6401CF
:102EC0002B9101EB8101411A2C91C3F38100002168
:102ED00003F003032D902E930C460846089D0D9B8E
:102EE000039E2B440A9D1B01354403EBC503049D3F
:102EF0002B44DD6B022D00F0CB81002500EB400060
:102F00004319944D05EB830015F823508778C37857
:102F100046782F95CDE93173309692B1039A012A04
:102F20000FD1CBE945732BAFCBF8F8100FCFCBE91E
:102F30004356CBF8FC00CBF80011CBF80421CBF8BA
:102F40000831089A0D9B039913440A9A1B010A44FD
:102F500003EBC203049A1344DA6B5C66022A00F0A6
:102F6000FD800F9B5B440DF1C0082BAF002607933B
:102F7000002D11DD0F9BD7F80090F3180BEB030A1F
:102F8000079B9C192C44494627A851F05DFB0AF881
:102F9000010BA245F7D12E4433AB984507F1040746
:102FA00000F0828058F8045BE2E73CF818C00CF0AF
:102FB0000F0CCCF1200C4FF000083146BBF10F0F85
:102FC00047DD6E7815F8024BC2F11807BC40C2F11C
:102FD0001007BE403443ABF1100B2343103201F114
:102FE000080401E00A2AE9DD23FA0CF101313EF878
:102FF00011100E0BB34011F0F00FC1F3031603F0E4
:103000000047A2EB11321BBF37435B00374602F18A
:10301000FF3211F4706FC1F3032603F0004102D0B8
:103020000E435B00013A4245A0F102002146FFF643
:1030300036A8002844E9027604F10804D2DCA2EBA9
:103040000803029A5B44D31A002BBFF6F9A8FFF7D6
:1030500026B80BEB0204002C7FF721A8BBF1000F70
:1030600006DD15F8017BC2F1180607FA06F63343B0
:10307000BBF1080F05DDC2F1100615F8012BB240B7
:103080001343621E4FF0004646FA02F213404FF01F
:103090000B0804F10B024FF0000BA0E7194627A81C
:1030A00051F0D2FAFEF703BE089A1F9B9B1A039AAF
:1030B0009B00C2EB421203EB42039B4400238BF8BC
:1030C00016308BF81530FEF780BE0A46FFF7F3B8CE
:1030D0000027FFF758B9B3F5FA7F80F27781A3F59F
:1030E000C8731D499810A1FB004189082B9101EB81
:1030F0008101411A03F003032C9100212D932E919D
:103100000C460120EAE6C4E90F000521404651F0D3
:103110009BFA05216064404651F096FA0521A064AF
:10312000404651F091FA0421E064404651F08CFA97
:103130000321E065404651F087FA20663378002B82
:103140007EF413AD0121404651F07EFAFEF70EBD2C
:1031500067666666B8B80800CDCCCCCC1F6C002F73
:1031600000F05F810F9BDDF8AC805F1E0BF1050561
:103170005F441D4427AC4146204651F065FA07F8EC
:10318000010FAF42F7D1354603230127209A0BEBFD
:103190000208149A2E469044002E26DD149A209997
:1031A0001E440A4403EB430313440BEB030A2BAB0B
:1031B00006EB460553F82790454427AC4946204680
:1031C00051F042FA49468AF81700204651F03CFA7D
:1031D00049468AF81800204651F036FA0AF1030AE7
:1031E0008AF81600AA45E9D133460137042F3ED0AC
:1031F00018EE102A52F82760CEE71B6C002B40F027
:10320000128127AC149A209903EB430357181F44EB
:103210000F9B0BF112065F441E444146204651F0BD
:1032200013FA4146F875204651F00EFA41463876B9
:10323000204651F009FA0337B875BE42EDD10F9B15
:103240000BEB03072946204651F0FEF9294687F883
:103250002900204651F0F8F9294687F82A0020462F
:1032600051F0F2F9033787F82800B742EAD1089AFB
:103270001F9B9B1A039A9B00C2EB421203EB420373
:103280009B4400238BF83B30ABF83C30FEF79DBDF0
:103290001B6C002B08BF012530E6136C002B40F09F
:1032A00022814A6B0D9B089903980B440A991B01D4
:1032B000014403EBC1032344C749DB6D013381FBA8
:1032C0000301A1EBE37302EB43024FF41071B2F977
:1032D0002E2002EB4202FEF7D6BDDDF81080FEF78D
:1032E0006ABFDDF810C0FEF7A0BF149B0BF10A0601
:1032F0005F1E5F441E4427AC4146204651F0A4F9AE
:1033000007F8010FB742F7D1149B0BF1150603F133
:103310000B075F441E442946204651F095F907F8F3
:10332000010BB742F7D1FEF750BD0F9B0BF105061D
:1033300003F1FF39D9441E4427AC4146204651F0E1
:1033400083F909F8010FB145F7D17B68002B7EF4B2
:10335000EDAC0F9B0BF10B0603F10609D9441E449B
:1033600027AC4146204651F06FF909F8010BB145F1
:10337000F7D1039B4FEA4318BB68002B7EF4F2ACF5
:103380000F9B0BF1100603F10B09D9441E4427AC27
:103390002946204651F058F909F8010BB145F7D1FB
:1033A000FB68002B7EF4F2AC0F9B0BF1150603F1CA
:1033B00010075F441E4427AC2946204651F044F9CB
:1033C00007F8010BB742F7D1FEF7F0BC08980D994A
:1033D000039D01448148A3F5FA73A0FB03400A9CB6
:1033E00009012C4401EBC401049C2144400800EB7A
:1033F0004004096C2B901B1B0024CDE92D442C9319
:10340000002900F08780CDE92C0321460220012409
:1034100064E5022B00F01D810723E3650D23FEF711
:103420009FBB3B46B2E60F9B0BF107065F1E5F4456
:103430001E4427AC4146204651F006F907F8010F1B
:10344000BE42F7D10323DDE6B3F5B47F03F00101FB
:103450004FEA630080F2DB80614CDB1784FB005491
:10346000C3EBE4032B9303EBC303A0EB83035D489F
:1034700080FB0340A0EBE3702C9000EB4000A3EB3B
:10348000400300242D932E94032027E5544A07334C
:1034900082FB032EDB17C3EBAE0E0EEBCE035B00FD
:1034A00008330E930EF101032F93E30023441A0215
:1034B0000D92039ABEF1000F02EB032304933FF732
:1034C00068A9FFF735BA136C002B00F09580079BB5
:1034D0002F9303F1FF3E0FFA8EFE122208231EFBEC
:1034E00002330E93E1E70B784A6B002B67D1089902
:1034F0000D9B03980B440A991B01014403EBC10384
:1035000013990B444FF41071DB6D013332F9132022
:10351000FEF7B9BC01240220E0E4A2EB0903029A01
:103520005B44D31A90E50B9BD3F8B037002B7ED1C8
:103530000B9A0123C2F8B037D946A24601E0AAEBA4
:10354000020A51464846F5F773FF002809EB0003CD
:1035500000F10302C0F2F68419F8000098F8001098
:10356000884203F10309EAD1587898F8011088429B
:10357000E5D198F802009978414011F0FC0FDED1B6
:10358000860748BF03F1FF33A3EB0B030B9A002B15
:10359000C2F8B437C0F2DB84049A0B9802991A443B
:1035A0000A44D0F8C01701FB02F2D0F8C817D200C5
:1035B00001FB05F592FBF5F2C0F8B8273AE0B2F945
:1035C0003600B2F93430B2F90C20C31A4FF410713E
:1035D00002EB4302FEF757BC56555555ABAAAAAAB3
:1035E000398EE338ABAAAA2A529B1860022047B052
:1035F000BDEC028BBDE8F08F2F9303020D93039B6C
:1036000003EB0023049308230E93FFF791B9F328EB
:1036100028DCA0F1B403181100242B90C3F381001F
:1036200003F003032C902E942D93042056E40B9B5F
:10363000D3F8B4370B9A1268002A00F06F815269F0
:10364000003A18BF01221A440B9BC3F8CC27FEF79F
:10365000C1BA236C002B7FF4DFAE0823E3650C2393
:10366000FEF77EBAC04CA0F1F403A4FB0304640887
:103670002B9404EB44041C1B2C940024CDE92D4412
:1036800005202BE48B4500F0FF80C0F2DB830B4666
:103690005FEA4B0B1A4603F10103F9D5FFF704B8B3
:1036A000119B53F8108CB8F1000F00F0E980079BD4
:1036B0001B78002B4FF0030309930CBF4FF0080851
:1036C0004FF00608FEF7D9BE1D9AA84B02F108007C
:1036D000C2E9023200F0B0FF2046FFF783BB139B24
:1036E00003F580530F93D3F80832002B40F3218168
:1036F0000F9BD3F80C32002B40F31B815FEA640A66
:1037000000F02D8414F0010000F00B810E9AD2F825
:103710003033002B40F09C83D2F84433079A0133B6
:10372000526B32F913C0BCF1000F4FF0000940F3A7
:103730001484139BCA46191F03F6FC074C464D46DA
:1037400051F8043F57F8040F1E181B1A0E603B6017
:1037500008682A4680EAE072A2EBE0724AEA020AAE
:103760002A4683EAE372A2EBE3720134A44549EAF4
:103770000209E5D1079B1C6A214604F001000028DC
:1037800000F09A8007990F9B0878D3F800E2002890
:1037900040F013810E9BD3F830A366101296BAF155
:1037A000000F40F04682D3F844034F6BD3F82C53FC
:1037B0006F4B00F10108C6EBC60237F918C0A842EA
:1037C00003EB820BAEEB0C0163464FEAC60280F2BC
:1037D0003482002940F33182229C2044149C3E30E4
:1037E0000444681C03906348049482180992D146EB
:1037F0005646049810F8012F0490072A47D05BF82A
:103800002250DBF81840641B08F1010837F91870E2
:10381000A7EB0C07002F40F32983139A02EB8300D8
:10382000CF1B043801EB030C01E0002942D050F813
:10383000043F1A4684FB02E29200C0F80029B64613
:1038400082EAE27EAEEBE27E49EA0E0985FB0323C3
:103850009B000360324683EAE372A2EBE372013914
:10386000B9424AEA020AACEB0103DED1039A904561
:1038700020D0FFB1079A3946576B37F918C0B8E71F
:10388000CDF82480FEF7F9BD1F22FEF70DBF394A9F
:10389000129852F83050099A5468B5E79246FEF7EC
:1038A000D7BE099B049A01330132032B099304927A
:1038B00040F04E81079B196A59B3BAF1000F00F02E
:1038C000D382C0F2478300235FEA4A0A1A4603F113
:1038D0000103F9D50F9BB9F1000FC3F8082200F0DE
:1038E000B582C0F2138300225FEA4909134602F150
:1038F0000102F9D50F9AC2F80C321146D2F80432FF
:10390000D2F800229342B8BF1346C1F80032C1F882
:1039100004320B9BD3F8BC37FEF7E6BE4FF0FF3204
:1039200091E60F9BD3E980329A42B8BF1A4694467B
:10393000F9E60F9BD3F80022002A1FDD139B0E4CE3
:10394000043B03EB82026FF0404002E01C609A42AD
:1039500014D053F8041FB1F1404FF7DDB1F1804F9F
:10396000A8BF1860F3E700BFABAAAAAA4D60050084
:10397000E4CE0900D4CE0900010000C00F9BD3F8AB
:103980000422002A15DD139BB04C03F6FC0303EB65
:1039900082026FF0404002E01C609A4209D053F866
:1039A000041FB1F1404FF7DDB1F1804FA8BF18609F
:1039B000F3E7079B1C6A2146A0E6149AD2F8F83078
:1039C0004FEA430963100393A14B09EB640918EE16
:1039D000107A03EB891B02F1FC0402F586750023C3
:1039E000012654F8042BE16806FA02F2002902F1DC
:1039F000FF3209DD194407EB810007EB830343F82D
:103A0000042B9842FBD10B46A542EAD10E9AD2F87C
:103A100030A3BAF1000F7FD10123CDE9443313461F
:103A20002299D2F84423D3F82C330A93531C0A4426
:103A30001499884F3E321144079A0991526B32F91A
:103A4000135018EE102A02EB83020492039A07EB3C
:103A5000C202AEEB0508D1460D92D6460A9A9A42AA
:103A6000FFF628AF099A049812F8011F099250F83E
:103A7000042B0490914249D04A1CCC074FEA6202C1
:103A80003FD55BF822105A461068079A526B5C1CAF
:103A90000C9402EB430432F91330B4F90220D31A28
:103AA0004345A8BF4346002B1C4624DD5E19139BEB
:103AB00003EB850203EB860552F8043B80FB03C34E
:103AC0009B00C2F8FC38F44683EAE37CACEBE37C71
:103AD00052F8043C49EA0C0981FB03C39B0042F8FD
:103AE000043CF44683EAE37CACEBE37C95424AEA8F
:103AF0000C0AE1D13546B8EB04083FF4DBAE0C9B71
:103B0000ACE7DBF800100BEB8202BDE7039A57F835
:103B100032100D9A5068B8E70E9B039A139903F57B
:103B200047730A9301233B93229B03F1550A149B8D
:103B300053449C46474BCDF810C04FF0000903EBAF
:103B4000C203CA46CDF824900D9301F510674D4687
:103B50000A9B07989A69466B53F8040B0A9306EB85
:103B6000420302F1010CB3F930800C9003231A4692
:103B7000099B844518FB02323FF793AE0CEB4C03D4
:103B80000498C05C18EE103A53F82C30984247D095
:103B9000431CC0074FEA63033DD55BF823005B4637
:103BA0001C680CF1010C0CF1140E06EB4E06B6F974
:103BB0000630A3EB0803002B39DD03EB43039E180B
:103BC00051F8223084FB03839B0047F82230A8463B
:103BD00083EAE378A8EBE37851F8223049EA080950
:103BE00080FB03839B0041F82230A84683EAE378F8
:103BF000A8EBE378033296424AEA080AE0D10C9B2C
:103C00006345FFF64EAE079B32465E6B06EB4E0EEB
:103C1000BEF90680B2E7DBF800000BEB8303BFE7D9
:103C20000C4B039853F830000D9B5C68B9E71646BF
:103C3000E5E70AF1FF33012B0ED9002C3FF469AE02
:103C40000F9A1F23C2F8083254E600BF010000C0DB
:103C50001CCF0900D4CE09000E9AD2F84033D2F816
:103C60002873079A1597566BBE4A06EB4301BB4271
:103C7000B1F930501299C1EBC10102EB81021299E6
:103C8000169205EB450503F101021092AEEB050E0D
:103C90004FEAC102D1DABEF1020FCEDDB24B10996C
:103CA00013441793229B01EB410255331344149A9A
:103CB0001A44814611924F008246844618EE101A2B
:103CC0001198169CDDF85C802BABAB4610F8012BED
:103CD000072A00F0A48054F82220A5691A60AA1AC5
:103CE0000A6004332EAA9A4201F10401EED1109B1E
:103CF00037440133B7F92E201493B7F930309B1AAB
:103D0000002B5D4640F3948003EB4303AEEB0308C6
:103D10002B9B0393309B04932C9B0993319B0A9319
:103D20002D9B2F9F0C93139B0EEB0B02CDE90D27C0
:103D300003EB8B0303E0BEF1020F7FF7BBAD1A6804
:103D40000E981146044684FB01018900C3F800194E
:103D5000604681EAE170A0EBE17003990C4684FBB8
:103D6000021292001A60614682EAE271A1EBE271EE
:103D70005A68049D14462E4686FB0454A400C3F8DA
:103D80000449664684EAE476A6EBE476099C254677
:103D900085FB024292005A60654682EAE275A5EB15
:103DA000E2759A680A9F144687FB04B4A400C3F81E
:103DB0000849E34684EAE47BABEBE47B304340EA2A
:103DC0000B0049EA00090C98044684FB02029200A9
:103DD0009A60604682EAE270A0EBE2702943AEF19D
:103DE000030E0D9A0143C6454AEA010A03F10C038A
:103DF000A2EB0E059FD1109B159A93423FF45AAD4A
:103E0000119BB8F1020F03F1030311937FF752AD39
:103E1000079B5E6B149B1093C6465F004EE7129D96
:103E2000514A52F835201A60D8F804200A6058E741
:103E3000109B159A93423FF43DAD119B03331193B0
:103E4000F046E7E74FF0FF32FEF72EBC1F2351E5A7
:103E5000079B0E9A5B6BD2F8402303EB4203B3F946
:103E6000303003EB430C5EE41F2233E5039A9045A8
:103E70003FF420AD0F46FDE40C4602F50051134619
:103E800002F1800704F58050D1F8002200269946FF
:103E90008846824606F0010BDAF8183B009320466C
:103EA0005B46494650F05EF8DAF81C3BD8F8002231
:103EB000009304F510605B46394650F053F8D8F88B
:103EC00000320BEB0B1203EB8213284609EB830144
:103ED00050F018FCD8F800220136A2EB0B0202F0D9
:103EE0000702122E04F1800405F18005C8F80022B3
:103EF000D0D1FEF74DBF21990B98F5F777FA1D9AAF
:103F0000D3692B441B1B1362FEF7D2B84FF0FF336B
:103F1000F0E40B9D28461C305946184421F0EAF97C
:103F2000D5F8CC27D5F8DC37219913442846A41AB4
:103F3000C5F8DC37F5F75AFA1D9AD3691B1B1362D3
:103F4000FEF7B6B80B9A4FF0FF33C2F8B437219999
:103F50000B98EFE74FF0FF32BCE4CA460FE420466F
:103F6000D1460CE4E4CE0900D4CE09004FF0000C99
:103F700010B482F800C001221A70019C036B236008
:103F8000029B09B190F83D201A705DF8044B704710
:103F900070B50D4684B011462846164A1E4622F0DA
:103FA0005FF80021482020F077FD134A0260316855
:103FB00011F003021BD1114B04460868984216D138
:103FC000012D06D82046134606F0AAFA204604B072
:103FD00070BD706801A9022225F08EFD2046DDE942
:103FE0000123316806F09CFA204604B070BD0448F5
:103FF0002CF04CF804000200E8DB0800E463090040
:10400000E8A4090008B5086806F0E4FA0E2008BD27
:1040100008B5406A05F00CF9212008BD10B504462A
:10402000406A05F005F994F83D00400040F00100B9
:1040300010BD00BF10B50446406A05F0F9F8A06B4A
:1040400010BD00BF10B50446406A05F0F1F894F8C1
:104050003C00216B04EB80044908636A20D003EB29
:1040600041029FED127A023B023A33F9020F07EE4A
:10407000900AF8EEE77A9A42A7EEA77AF5D1F1EE28
:10408000C76A07EE901AF8EEE77AC6EEA77A17EE3F
:10409000900A20F0030040F00200A0F1FF4010BDA4
:1040A000DFED027AF0EE676AEFE700BF0000000084
:1040B00010B50446406A05F0BBF8606B400040F064
:1040C000010010BD10B50446406A05F0B1F8606CFF
:1040D000400040F0010010BD38B50C460546406A6E
:1040E00005F0A6F8A30709D1064B22689A4205D12C
:1040F0002846214606F082FA0E2038BD02482BF0F1
:10410000C5FF00BFE4630900E8A4090038B50D4607
:104110000446406A05F08CF8284627F0ABFF606340
:104120000E2038BD10B5044609B1012A1BD00AF093
:1041300015FBA06B00220023083051F06DFCE169F3
:10414000216200224FF47F436264E387204621F01E
:104150007FFF204621F0F0FE204621F08DFEBDE8D5
:1041600010400AF035BB10BD08B583680BB106F0EE
:1041700087FA0E2008BD00BFF0B587B02F4C009421
:1041800003AD0846019511461A46032321F0FEFFB0
:1041900003984DF00BFE074604984DF00FFE0021EA
:1041A0000546242020F078FC254A264B0260D3F8EF
:1041B0000025BDF8146012F00102044617D003F583
:1041C000A043D3F80015C80711D503F58053D3F8E1
:1041D0000025D1070AD503F53043D3F80025D207CF
:1041E0002AD500231848A3602BF03CFF0222174970
:1041F000A3608A5C22770022C3F80C25A368012201
:10420000C3F81025A2683B792376C2F86035387967
:1042100005F05EFA3DB1A2682B796376C2F8683585
:10422000287905F055FAA368360A01222046A682AD
:10423000C3F8002507B0F0BD0322D8E700C108008D
:104240000CDD080000C001407CBF0900C8720900F5
:1042500008B5086883680BB106F012FA0E2008BD95
:1042600010B50446806804F0E9FFE37F002B14BF1B
:104270003E201E2010BD00BF38B585680446284684
:1042800004F0DCFFE37F2BB9D5F8042112B163778A
:10429000C5F80431637F002B14BF3E201E2038BDBB
:1042A00038B585680446284604F0C8FFE37F13B993
:1042B000D5F804214AB9637F5BB1A36801210222CA
:1042C000E177C3F800220E2038BD6377C5F80431CA
:1042D000F1E7FCF7FDFA00BF70B50D4688B055F860
:1042E000044B03920646A06804F0A8FF06AB0193B6
:1042F000614B009329460223701E039A21F0DCFED5
:10430000E37F069D9DF81C602BB9A268D2F80411CA
:10431000002940F09580637F002B40F09880656015
:1043200084F82060284600F027F90646284600F069
:10433000CFF80DF11303C00805AAE0760021284646
:104340000193009204F1210304F1220200F0F0F83D
:10435000284600F0CBF8059DA076B5F5803F80F0AB
:104360008480AD000021284620F096FB94F82210AE
:10437000E06000296FD006F574452335B5FBF6F5EE
:1043800006FB05F35D0805F5740505F51055B5FB4D
:10439000F3F56A08A16802F5740303F51053B3FB43
:1043A000F5F202EB5602B2FBF6F3013BC1F84835D9
:1043B000A168C1F82835A3686A1EE282C3F80855CF
:1043C000A3680122C3F81425606800F0C7F82B48E1
:1043D0000023024652F8041B002941D00133042B6C
:1043E000F8D1A36800250422A5772046C3F800224F
:1043F000294619F0CFFBA368D3F82025C3F8402540
:10440000A368D3F82425C3F84425A268C2F808514C
:10441000A268C2F80C51A268C2F81051A268C2F892
:104420001451A268C2F80451A2680C21C2F8041306
:10443000A26801230E2093606377E57708B070BD12
:104440006377C2F80431637F002B3FF468AF2046E6
:1044500006F05AF963E7284620F01EFB20618AE740
:1044600040F8234047F050FEBBE705484FF6FF7287
:1044700029462BF027FE00BF68CA0800F04501203E
:10448000D8BD090038B585680446284604F0D6FE34
:10449000E37F0BB90E2038BD04230022E277C5F874
:1044A0000032A368D3F804110029F3D0C3F8042123
:1044B000A36801229A600E2038BD00BF10B50446E3
:1044C000806804F0BBFE204606F01EF90E2010BDE9
:1044D00010B50146044640F287402BF0F1FC03463C
:1044E00020469B68BDE81040184700BF10B5014644
:1044F000044640F287402BF0E3FC03462046DB688D
:10450000BDE81040184700BF30B5044685B00B46E3
:1045100040F287402146154603932BF0D1FC0095CD
:1045200000224569039B11462046A84705B030BDCF
:1045300070B5044682B00D46014640F28740CDE991
:1045400000322BF0BDFC8669009B019A294620466B
:10455000B44602B0BDE87040604700BF10B50146E8
:10456000044640F287402BF0ABFC00220369114661
:104570002046BDE81040184710B50146044640F2F9
:1045800087402BF09DFC034620465B68BDE8104049
:10459000184700BF10B50C4C206818B10B4B1B68B6
:1045A0000BB1002010BD48F093F9236898422368AE
:1045B00036BFDB43C01AC01840F2EE23984294BFC6
:1045C0000020012010BD00BF204E01203C460120EC
:1045D000024A136823EA0000106070473C4601203D
:1045E000024A136818431060704700BF3C46012020
:1045F00008B50C4B1B6813B90B4B1B7803B908BDEE
:1046000048F066F9094B18601A6812B91A68013245
:104610001A60074B0749012003F1540208705A62DF
:1046200008BD00BF3C460120AC5B0120204E0120AC
:104630000C520120A95B012010B504460AF08EF847
:10464000E36873B90A490A68A2420AD0094AA3601A
:1046500010681368E0600BB113689C600B6823B1AD
:104660001460BDE810400AF0B3B80C60F8E700BF72
:104670004846012050460120F0B5144D2B6883B008
:1046800013B3134F0AF06AF83E78C6B92C68114B81
:104690002E6001223A701E607CB12346A4681D681A
:1046A00058680190C3E902660AF092F8019805B1D2
:1046B000A8470AF053F8002CEFD100233B7003B059
:1046C000BDE8F0400AF084B803B0F0BD48460120D0
:1046D000B55B01205046012008B527F025FD0346B3
:1046E0000348D98897290CBF422297222BF0D6FC89
:1046F000B8A80900F0B587B0254C009402AD084673
:10470000019511461A46042321F040FD02984DF010
:104710004DFB054603984DF049FB0021064620203D
:1047200020F0BAF91B4B0360DDE9042383611A4BC7
:104730009A4288BF012300F1040798BFB3FBF2F34C
:10474000044643612946384608F00EFC10B1204665
:1047500007B0F0BD04F10C053146284608F004FC12
:1047600078B901221146384608F0A0FC0122114612
:10477000284608F09BFC204644F044FE204607B043
:10478000F0BD384605F058FD204607B0F0BD00BF2B
:1047900078CA08009CDE080020A1070008B5086858
:1047A00042F0DCFE0E2008BD08B542F0D7FE0E2018
:1047B00008BD00BF10B5044604F0D8FC09F0CEFFD8
:1047C000237F1BB10AF004F81E2010BD01232377BC
:1047D00009F0FEFF3E2010BD10B5044604F0C6FCF3
:1047E000002323770E2010BD70B50C4688B054F816
:1047F000045B03920646284604F0B8FC284604F001
:1048000083FD04AB0193094B039A00932146701E6C
:10481000042321F051FC079C049900942846DDE90B
:1048200005233EF0AFFF0E2008B070BDA0CF0800FA
:10483000F8B5064604F09AFC304604F065FD002009
:104840001FF0E0FB1024074602E00234F02C14D0E5
:10485000304644F075FAE1B230464FF025F805468F
:10486000304644F0CFFD002DEFD044F00101384632
:10487000023428F019FDF02CEAD13846F8BD00BF0B
:1048800070B50C4688B054F8045B0392064628467F
:1048900004F06CFC284604F037FD04AB01930A4B8E
:1048A000039A00932146701E042321F005FC07990A
:1048B0000124CDE900142846DDE9052304994FF0D1
:1048C00007FA0E2008B070BD18C1080070B50C467C
:1048D0008CB054F8045B03920646284604F046FC6C
:1048E000284604F011FD05AB01930E4B039A00938B
:1048F0002146701E072321F0DFFB0999089B069AC9
:104900000020CDE90010059928464FF0E1F90B9CF5
:104910000A9B079A0599009428463EF033FF0E2023
:104920000CB070BDA0CE080070B50C4688B054F82D
:10493000045B03920646284604F01EFC284604F059
:10494000E9FC04AB01931C4B039A0093214604231A
:10495000701E21F0B1FB059BDAB2012A28D8069916
:10496000CAB2012A21D8079A083AD2B2012A19D824
:10497000049C124AB2FBF4F004FB102202B1013095
:1049800095F82020E86103F0010301F001019B008C
:1049900043EAC10322F00C0213430E2085F82030B5
:1049A00008B070BD06482BF085FB06482BF082FB53
:1049B00005482BF07FFB00BF98D0080020A107001E
:1049C000FCB60900F4B60900DCB609002DE9F04197
:1049D00086B0364C009403AD0846019511461A4640
:1049E000032321F0D3FB03984DF0E0F9054604982A
:1049F0004DF0E4F9064605984DF0E0F90021074630
:104A0000242020F049F829460546294B45F8043B67
:104A10000446284608F0A8FA98BB94F820100246ED
:104A2000C1F38001284608F041FB8EB104F10C0867
:104A30003146404608F098FA024680BB94F8203090
:104A400043F00203404684F82030114608F02EFB64
:104A50005FB1394604F1140008F086FAA0B994F861
:104A6000203043F0010384F8203094F820300522F0
:104A700023F00C032046E26184F8203006B0BDE844
:104A8000F0810C482BF016FB284605F0D5FB1EB133
:104A900004F10C0005F0D0FB07482BF00BFB284677
:104AA00005F0CAFB05482BF005FB00BF38C1080024
:104AB0009CDF080094BB090028B609001CB6090059
:104AC00008B5086842F0B8FD0E2008BD08B542F0F0
:104AD000B3FD0E2008BD00BF10B5044604F04CFB2A
:104AE00009F03CFE94F82030DB0603D509F070FE97
:104AF0001E2010BD94F8203043F0100384F82030BD
:104B000009F066FE3E2010BD10B5044604F034FBEB
:104B100094F820306FF3041384F820300E2010BD79
:104B20002DE9F04F0D468FB055F8044B0392064621
:104B3000204604F021FB204604F0ECFB0AAB019375
:104B4000464B039A009329460423701E21F0B4FAC1
:104B50000A98022207A924F0CFFF0B98089B069021
:104B60000C99059305AA06A836F07CFA059D1DB997
:104B70000E200FB0BDE8F08F94F820109DF834B0EF
:104B8000CA07DDE9066765D58B07D4F81C805AD4BF
:104B900007EB060909EB050A5D460826002727E012
:104BA000404609F0CFFD94F82010A068C1F38001C1
:104BB00081F0010101F0010108F046FAA06908F056
:104BC000FDF994F8201040EA47000B07C7B220D443
:104BD000404609F0B7FD94F82010A068C1F38001A9
:104BE00008F032FA6D00013EEDB21ED094F82010AC
:104BF000880721D40A07D3D5C1F3800181F00101D0
:104C0000A06801F0010108F01FFA404609F09AFD82
:104C1000D4E7A068C1F3800108F016FA404609F015
:104C200091FD6D00013EEDB2E0D109F8017BCA456E
:104C30009ED094F82010AFE7E909206908F004FA43
:104C400094F82010D6E70021206908F0FDF994F8C7
:104C500020109DE702482BF02DFA00BFD8CE0800A7
:104C600084BC09002DE9F0430D468DB055F8044B86
:104C700003920646204604F07FFA204604F04AFBE1
:104C800009AB0193384B039A009329460323701E06
:104C900021F012FA0998012206A924F02DFF0A98A2
:104CA000079B05900B99049304AA05A836F0DAF93E
:104CB000049B1BB90E200DB0BDE8F08394F82000D2
:104CC0008007DDE905214CD501EB0208E76908EB17
:104CD000030918F8015B08261BE0384609F032FD8D
:104CE00094F82010A068C1F3800181F0010101F067
:104CF000010108F0A9F9384609F024FD94F82010C4
:104D0000A068C1F3800108F09FF96D00013EEDB28B
:104D100021D0E909206908F097F994F820100B07D1
:104D2000DBD5C1F3800181F0010101F00101A06830
:104D300008F08AF9384609F005FD94F82010A068BB
:104D4000C1F3800108F080F9384609F0FBFC6D00E2
:104D5000013EEDB2DDD1C145BBD10E200DB0BDE8A5
:104D6000F08302482BF0A6F9C0CF0800E4BB09008D
:104D70002DE9F04F0D4695B055F8044B03920646C9
:104D8000204604F0F9F9204604F0C4FA0EAB019372
:104D90004C4B039A009329460623701E21F08CF990
:104DA0000E9801220BA924F0A7FE10980C9B1199D4
:104DB000079006AA07A8069336F054F90F98022226
:104DC00008A924F099FE1298099B059004AA13994A
:104DD000049305A836F046F9069B049A93426ED1D7
:104DE0001BB90E2015B0BDE8F08F94F820100B9E73
:104DF000059A8F07DDE907505ED5C9075CD506EB3C
:104E00000509013AD4F81C8000EB020A09EB030BF8
:104E100019F8015B0826002725E0404609F092FCBE
:104E200094F82010A068C1F3800181F0010101F025
:104E3000010108F009F9A06908F0C0F894F8201001
:104E400040EA47000B07C7B222D4404609F07AFC7B
:104E500094F82010A068C1F3800108F0F5F86D0007
:104E6000013EEDB220D0E909206908F0EDF894F890
:104E700020100A07D1D5C1F3800181F00101A0689B
:104E800001F0010108F0E0F8404609F05BFCD2E7D0
:104E9000A068C1F3800108F0D7F8404609F052FC41
:104EA0006D00013EEDB2DED1CB450AF8017FAFD1F6
:104EB0000E2015B0BDE8F08F03482BF0FBF8034837
:104EC0002BF0F8F898CA080030BC090070A9090056
:104ED000930702D590F82230C3B98389C28802FBB8
:104EE00003F39B004B6083680B60837B102B09D01E
:104EF000202B03D042238B600020704749238B6016
:104F00000020704748238B600020704701207047C5
:104F10002DE9F0430E2A85B05ED017468A07054674
:104F2000084603D1314A0968914252D0C3073BD4A5
:104F300001AA022127F036F8019B186827F09AF899
:104F4000019A84B2506827F095F8AB88A34286B2E4
:104F500045D9EB88B34242D9042F2FD0384627F0E9
:104F600089F8AB7B30FA03F307463BD104F1010C1F
:104F70000FFA84F801A90FFA86F92846741C0393E6
:104F8000ADF808C0ADF80480ADF80A40ADF8069061
:104F900012F062FE28463B464A46414612F07EFE2B
:104FA0000E2005B0BDE8F083AC884310042F93FBBE
:104FB000F4F604FB16339CB2B6B2CFD132B221B2B2
:104FC000284608F037F9400040F0010005B0BDE880
:104FD000F08307482BF028F806482BF001F8064824
:104FE0002BF00EF805482BF065F800BF846209002D
:104FF00090B10900E0BC090034C5090028C50900CA
:105000002DE9F04F2DED028B91B00AABB94C019315
:105010000094062321F050F8B7490A9840F227324D
:1050200021F0F8F8B44940F2215207460B9821F0DC
:10503000F1F8B149034640F222520C98049321F052
:10504000E9F80E9B05900E2B00F0F380184626F031
:10505000BBFF0F980E28F0EE408A00F0F08026F09B
:10506000B3FFB0EE408A0D99A44810F07DF9049981
:105070007A684B689A425FFA80FA40F03481BB7BD1
:10508000897B994240F02F81059841688A4240F01F
:105090002A81827B9A4240F026810AF1FF32082A57
:1050A00000F21E81DFE812F009001C0109001C015A
:1050B00009001C0109001C01AC00102B40F01681F6
:1050C000BB88ADF820300026FB88079607A9384634
:1050D000ADF82230099612F0BFFDF0EE687AFEEED0
:1050E000CC7ABAF1090F17EE905AF0EE487AFEEE3C
:1050F000CC7A17EE904A00F0A780F9880AF0FB0AF4
:10510000002900F09080BA88029641F6F07BCDED40
:10511000037A049E0598029BB7F80CE0B6F80C9051
:10512000B0F80C8003FB0EFE03FB09F903FB08F843
:10513000BB6803EB8E0EB36803EB8909836803EB4E
:105140008808002A69D0039C4FF0000C40E012F55B
:10515000F84248BFFF32121222EAE27202F47842A9
:1051600012B203F4FC6601F4FC6004FB06F605FBD6
:1051700000666348864249DC16F57C7048BF06F23B
:10518000EF40001220EAE07000F4FC6003F01F031F
:1051900001F01F0104FB03F305FB0131594538DC25
:1051A00011F10F0648BF01F58776331223EAE37346
:1051B0001BB202431A43BAF1030F92B201D152BAA1
:1051C00092B22EF8022BBA880CF1010C944522DA27
:1051D000BAF1030F39F8021B38F8023B03D149BA80
:1051E0005BBA89B29BB203F4784201F4784004FBC5
:1051F00002F205FB002243488242A8DB424AB0E7A4
:10520000082B3FF45DAF41482AF054FF4FF4FC6097
:10521000BCE71F23CDE7F9880394029B01338B423F
:105220000293FFF676AF0E2011B0BDEC028BBDE805
:10523000F08F0F980E28F6EE008A7FF410AFB7EECD
:10524000008A38EE688A0EE7F9880029EBD0DDE99C
:105250000489BA884FF67F70B7F80CC0BB68B8F8FD
:105260000CE0B9F80CA006FB0CFC03EB8C0CD8F896
:10527000083006FB0EFE03EB8E0ED9F8083006FB55
:105280000AFA03EB8A0A12B300210EE013F180023E
:1052900048BF03F27F12131223EAE373DBB20CF868
:1052A000013BBA880131914210DA1AF8013B1EF82D
:1052B000012B04FB03F305FB02338342E6DDFF23EE
:1052C0000CF8013BBA8801319142EEDBF9880136D6
:1052D0008E42C1DB0E2011B0BDEC028BBDE8F08F19
:1052E0000B482AF0E7FE0B482AF0E4FE0A482AF0B1
:1052F000E1FE00BF98D1080070FC0800F0FD080036
:105300000FDD07000085F70000F8FFFFD0B80900A7
:1053100014AD09006CBE0900B8B809002DE9F04FC2
:1053200097B00FAB584C01930094072320F0C4FEB4
:1053300056490F984FF42E7220F06CFF01228146DF
:1053400009A9109824F0D8FB139F119B0493129B7A
:1053500007937B1C149B069308BFB9F804700133B4
:1053600004BFB9F806300693049B002BC0F2868078
:10537000079A002AC0F282809F427FDB0699914201
:105380007CDBB9F80430BB4278DBB9F806308B42DD
:1053900074DB049B9DF82C10FC1ADDE906324020DA
:1053A0009B1A002203FB04F420F044FFDDF8548034
:1053B0000A9BB3FBF0F6B8F10E0F05465BD04046F2
:1053C00026F058FE8346B4425BD899F80E30099E09
:1053D0004FF0010A0AFA03FADDE9063293420AF1B4
:1053E000FF3A33DD079B07EE909A9946049B9F4254
:1053F00025DD0FFA89F2CDF81490049C17EE909AEF
:1054000011E016F8013BB8F10E0F01D09B4507D013
:105410000AEA030321B24846039212F03FFC039AC2
:105420000134A74209D0022D04D0042DE9D156F849
:10543000043BE8E736F8023BE5E7DDF81490069B0D
:1054400009F101094B45D1D117EE909A049B079AB7
:10545000ADF8303048460023ADF832200CA9069A4A
:10546000ADF83470ADF836200E9312F0F5FB0E2037
:1054700017B0BDE8F08F4FF0000BA4E704482AF006
:10548000BFFD04482AF0BCFDF8CE080070FC0800FF
:1054900034C5090098A2090070B586B0274C009465
:1054A00002AB0193042320F007FE254903984FF433
:1054B000A46220F0AFFE40F227322149054602984F
:1054C00020F0A8FE059904461E480FF04DFF0499F0
:1054D00006461D480FF048FF61686B688B4224D177
:1054E000A17B1029F6B2C2B201D0012920D1511EF0
:1054F000082917D8DFE801F0051605160516051668
:105500001000AB7B102B16D120463346294605F000
:1055100033FA0E2006B070BDAB7B082BF4D00B48DD
:105520002AF0B4FD0A482AF0B1FD0A482AF0AEFD7F
:1055300009482AF0ABFD09482AF0A8FD50C108002F
:1055400070FC08001CE00800F0FD0800BCC2090067
:1055500078A30900C0A90900F8C20900E4C2090043
:105560000A46014640F2B9200FF0EABE10B588B0F5
:1055700003AB1D4C01930094052320F09DFD1B49B6
:10558000039840F2273220F045FE817B069B0122E2
:105590008A40934221D2079C6FF000418C4201D097
:1055A000A2421DD9BDF91010BDF91420002911DB4C
:1055B000B0F804C061450DDA002A0BDBB0F806C074
:1055C000624507DAA34202D0009405F0AFF80E203E
:1055D00008B010BD06482AF06DFD06482AF06AFDA5
:1055E00005482AF067FD00BFB8D0080070FC08002D
:1055F000AC9B09000CA00900DCA9090030B51A4BCE
:1056000089B002ACCDE90034062320F055FD0298A4
:10561000079D827B012393409D4222D2BDF90C104D
:10562000BDF91020BDF91430BDF91840002918DB70
:10563000002B16DB002A14DB002C12DBB0F804C0B0
:1056400061450EDA9C450CDDB0F806C0624508DA0B
:10565000A44506DDCDE9004505F00EFB0E2009B09E
:1056600030BD02482AF026FDD8CF0800AC9B0900C7
:10567000F0B52B4B8FB008ACCDE90034062320F0F9
:105680001BFD089E0D9FB27B012393409F4244D295
:10569000BDF92830ADF80A30BDF92C30ADF80C302A
:1056A000BDF93030ADF80E300021099B049102A8FD
:1056B000ADF8083012F0A0F8B38805910246ADF8B5
:1056C0001830F388079105A9ADF81A3012F0A6F842
:1056D0001146304612F0C0FABDF90850BDF90C3041
:1056E000AB4217DDBDF90E20BDF90A40A2420DDD27
:1056F00022463B462946304612F0D0FA0134BDF925
:105700000E2024B2A242F3DCBDF90C3001352DB2DB
:10571000AB42E9DC0E200FB0F0BD02482AF0CAFC13
:1057200040D10800AC9B09002DE9F0432DED028B20
:10573000534B9FB011ACCDE900340D2320F0BCFCDD
:10574000DDE91154AA7BA37B9A42C0F0968013989E
:105750000E2800F08F8026F08DFC06B214980E28DB
:1057600000F0858026F086FC07B217980E2879D0C5
:1057700026F080FC0FFA80F818980E286DD026F0DD
:1057800079FC0FFA80F9169B00930FAB02930DF191
:105790003E03159901930DF1420210AB28464CF0DF
:1057A000C5F91A9B00930DAB02930DF136030193DB
:1057B000204619990EAB0DF13A024CF0B7F91B983F
:1057C0000E2844D026F000FCF0EE408A1C980E28EB
:1057D00008D026F0F9FBB5EEC00AF1EE10FAB0EEF3
:1057E000408A01D5B7EE008A1D980E2832D026F0E7
:1057F00041FC0023CDE90A03BDF93C30BDF93E2050
:10580000CDF81490CDE90234BDF934400994BDF9C6
:105810003640BDF940300894BDF938400794BDF9D1
:105820003A40CDF81080CDE900322846BDF942302B
:105830000694B0EE680AF0EE480A3A46314605F0A2
:105840000BFC0E201FB0BDEC028BBDE8F083DFED3A
:105850000D8ABBE701230020CCE7B4F806904FEA9D
:10586000590990E7B4F804804FEA580884E7EF88B4
:105870007F087AE7AE88760870E703482AF01AFCBA
:1058800000D20800000000000CC3090010B58CB065
:10589000484C009405AB0193072320F00DFC4649CA
:1058A00005984FF42E7220F0B5FC089C0699631EF3
:1058B000012B28D9042C78D1079B5A1E1F2A6BD89C
:1058C000DFE802F012126A126A6A6A126A6A6A6A87
:1058D0006A6A6A126A6A6A6A6A6A6A6E6A6A6A6A7C
:1058E0006A6A6A12012C5BD19DF82C2002929DF805
:1058F000282001929DF824200092224605F07CFA8F
:105900000E200CB010BD079B5A1E1F2A44D80FF260
:10591000080C5CF822F000BFE9580300E9580300C6
:1059200099590300E9580300995903009959030054
:1059300099590300E9580300995903009959030044
:105940009959030099590300995903009959030083
:1059500099590300E9580300995903009959030024
:105960009959030099590300995903009959030063
:1059700099590300E5580300995903009959030008
:105980009959030099590300995903009959030043
:1059900099590300E9580300084819462AF092FB78
:1059A0000748182221462AF08DFB064821462AF096
:1059B00089FB00BFC8CA080070FC080024A10900C8
:1059C00010A10900F8A0090038B50D4BD3F8E43058
:1059D00004460D4613B908E01B6833B19A68A24229
:1059E000FAD15868A842F7D138BD01210C201FF028
:1059F00053F82A462146BDE8384000F003B800BFFE
:105A00000C52012070B40B4DD5F8E4405CB1234634
:105A100001E01B683BB19E688E42FAD15E689642F7
:105A2000F7D170BC7047C0E900428160C5F8E4005E
:105A300070BC70470C5201200B4AD2F8E4308BB195
:105A400002F1E40C02E09C461B685BB19A6882425A
:105A5000F9D15A688A42F6D11968CCF800100022B0
:105A60001A607047704700BF0C52012008B5074B01
:105A7000187800B908BD064B58680028FAD01846B7
:105A800006F07AF8003818BF012008BDA75B012096
:105A90003C44012008B50348012105F0E9FD0E2032
:105AA00008BD00BFD446012010B584B002AB0B4C3A
:105AB0000193009402230431013820F0FDFA0849D3
:105AC000029840F2862220F0A5FB0446039826F0B7
:105AD0007BFA204605F0E8FC04B010BDC0CD0800FC
:105AE000B4E2080008B501F0D1FD0E2008BD00BFEA
:105AF00010B5012182B005F0BBFD684640F05EFCA8
:105B000003F038FC00210C201EF0C6FF064B03609A
:105B10009DF800200DF101015208044605F06EFFCA
:105B2000204602B010BD00BFB4E20800C368002BDD
:105B300014BF3E201E20704708B505F075FD0028F3
:105B400014BF3E201E2008BD2DE9F04106468069A5
:105B500086B010B106B0BDE8F081114C054604F5E1
:105B60002A784FF6FF772388BB4208D0E06D0E28D5
:105B700010D006AB03EB8503013543F8140C8834D1
:105B80004445F0D101A9284627F050FFB06106B086
:105B9000BDE8F081204600F05FFEE065E9E700BF68
:105BA000A805012008B505F053FD002814BF3E20CC
:105BB0001E2008BD90B583B0002400AFB91D20465B
:105BC000FC8040F011FCFB8807336A46DB08A2EB3F
:105BD000C3039D46B91D684640F006FC30B9F988FC
:105BE000684627F08DFE0C37BD4690BD20460C3729
:105BF000BD4690BD08B501482AF016FAECBC090074
:105C000010B586B088680C46012203A923F060FF16
:105C100010B90C482AF062FA9DF804202179039B00
:105C200061F347028DF804201A68CDF805209B889F
:105C3000ADF8093001A840F0C3FB0028E9D10E20DF
:105C400006B010BD28BB090010B50446084627F071
:105C5000C5FA0146204605F00BFD0E2010BD00BF21
:105C600000B5084685B028F00BFD00238DF80C30F8
:105C7000019045F0ABF9019982B203A840F0B6FB60
:105C80000E2005B05DF804FB2DE9F04F2DED028BE1
:105C900095B00CAB51F8044B01936A4B009301385B
:105CA000082320F009FA0C98012209A923F024FF07
:105CB0000D9800230E28CDE90633089303D0012266
:105CC00006A923F019FF1198002800F0958026F00E
:105CD0007BF9DFED5D7AB4EEE70AF1EE10FAB0EE93
:105CE000408A00F1A180DFED597AB4EEE70AF1EEC7
:105CF00010FA00F399800A9E9DF838509DF83C9068
:105D0000DDF840801F2E60D813980E287AD0002D21
:105D100000F092804E4940F2333220F07BFA074681
:105D200094F84430DDF848B0002B40F08280E368FE
:105D30001BB1204605F030FE0A9E2946304603F08E
:105D400003FADDF81CA02946504603F0FDF91F2E8A
:105D500043D9BAF1000F61D1002F62D1B8F1000F21
:105D600040D1B9F1000F18BF4FF0B40861680029A5
:105D70004FD0A168002947D0DDE9091260681FF003
:105D8000B9FADDE90612A0681FF0B4FACDE904B74C
:105D9000BDF81C300393A3680293BDF8283001932B
:105DA000606800904346B0EE480A4A4629462046BD
:105DB000F5F76CFE03F0DEFA01230E2084F8443080
:105DC00015B0BDEC028BBDE8F08FC5B1079F002F69
:105DD00035D113980E289DD1A2E7002EBCD1B8F181
:105DE000000FBED01B4B1C4A03FB08F39342BDD9E6
:105DF0001A48B4212AF072F91948119067E7139BE9
:105E00000E2B19D100278BE7FF201AF053F8A06062
:105E1000B2E7FF201AF04EF86060AAE711482AF0B6
:105E20005DF911482AF05AF9104A114911482AF02F
:105E300049F911482AF052F910482AF04FF9104850
:105E40002AF04CF910BE08000AD7A33C0AD7234118
:105E5000B4E2080040420F000FBCBA0A08AF0900C4
:105E6000CECC4CBE88B9090084BA0900E47608009B
:105E7000EC76080048A109006CBF0900A4B3090032
:105E800094BC09002DE9F04F2DED048B93B00AABC3
:105E900051F8044B0193944B00930138082320F0F0
:105EA0000BF90D980E2800F0E48026F08DF80E987E
:105EB000B0EE409A002800F0E2800F9B002B00F02B
:105EC000E48026F081F8DFED897AB4EEE70AF1EE9E
:105ED00010FAB0EE408A00F1F080DFED857AB4EE82
:105EE000E70AF1EE10FA00F3E880B5EE409AF1EE21
:105EF00010FA05D0B4EEC09AF1EE10FA00F1EB8082
:105F00000F9826F061F8B4EEC08AF1EE10FAF0EEC8
:105F1000408A00F1DA800A9800230493002800F0F8
:105F2000B780012203A923F0E7FDDDF80C90484675
:105F30001AF09AFC002800F0CB80DDF8108023696D
:105F40009DF83050DDF82CB0DDF840A09DF844708D
:105F500033B193F82530002B00F0C3800023236178
:105F6000E36833B16268934200F0A480204605F0F4
:105F700013FD002128201EF08FFD5E4B06460022F7
:105F800040F8083B59463FF055F8002DC6E9069801
:105F90004FF00001C6F820A040F2071026610ABFAA
:105FA00027204FF0FF084FF01F081EF075FD2369F2
:105FB000586000F108030360A0F804800646012041
:105FC000F7F73CFF03F0D6F921694B48FFF7FCFCDB
:105FD0009FED4A7A9FED4A6A29EE077AF6EE006A4B
:105FE000C7EE067A77EEA67AFCEEE77A17EE903ADD
:105FF000B3F5803F66D223B9B5EEC09AF1EE10FA40
:106000006CDC9FED3E0ADFED3F6AADF81E3028EEF6
:10601000008A68EE808A88EE267A45F4807545EA23
:10602000870525F0FA053146ADF8185006A8002579
:106030000895ADF82450C8EEA67AF6EE006A37EE61
:10604000267A77EEA67ABCEEC77AFCEEE77A17EEF0
:10605000103AADF81A3017EE903AADF81C3040F017
:10606000D3F90646C0B9206913B0BDEC048BBDE876
:10607000F08F0E989FED249A00287FF41EAF0F9B9F
:1060800022480E90002B7FF41CAF204B0F9318E793
:10609000DDF80C90804652E721691748FFF7CCFCE9
:1060A0003046256103F066F9284613B0BDEC048B39
:1060B000BDE8F08F112003F063F9154A1549164821
:1060C0002AF000F8154829F0F5FF154829F0F2FFED
:1060D000144829F0EFFF144829F0ECFF134829F089
:1060E000E9FF134829F0FAFF80CC08000AD7233BC8
:1060F00066D62342E8E80800495F07000024744997
:1061000000401C4600401C4400000000CECC4CBEA9
:10611000BC760800C876080048A109002CB7090021
:10612000609D0900CCB20900709D0900809D0900A6
:10613000A8B1090008B505F02FFC0E2008BD00BF6E
:1061400008B503690BB105F047FC0E2008BD00BF80
:1061500002280BD193070BD110B50D4B0C461168DB
:10616000994282B006D01E2002B010BD00207047B8
:106170001E2070479168A068019225F017FA019AD5
:106180000028F0D0217913799942ECD13E20EBE739
:10619000B4E20800806870470079400040F00100D8
:1061A000704700BF30B589B0154C009403AD084668
:1061B000019511461A4602231FF0E8FF00210C202A
:1061C0001EF06AFC0F4B036004460122039805A9E8
:1061D00023F092FC069B062B0AD1049A032A0BD8C3
:1061E00020460599D2B205F009FC204609B030BD21
:1061F0000548062129F066FF044829F05BFF00BF2F
:1062000050BE0800B4E20800FCBF0900F0BF09005E
:1062100010B588B004460122886805A923F06CFCFB
:10622000059920460C780B794A7903944C780294AE
:106230008C780194CC780094024929F01FFE08B0B4
:1062400010BD00BF60730800062801D00020704711
:1062500030B50E4B8D682B40062B83B00C4610D00A
:10626000686830B123795840400040F0010003B025
:1062700030BD01A9284628F0DBF901993CF00CFC5F
:10628000F0E728093CF03EFDEBE700BF0F0080FF80
:1062900031291DD8102918D91139202914D8DFE83F
:1062A00001F01E21131313131313131313131313DA
:1062B000131324111313131313131313131313139F
:1062C00013131B0022230370704721B9017070471C
:1062D0004129FBD070477047312303707047112369
:1062E00003707047122303707047212303707047B7
:1062F0002DE9F04F97B00DAB414C019304310923C8
:10630000013800941FF0D8FE3E490D9840F2FC423F
:106310001FF080FF40F2A2523B4906460E981FF044
:1063200079FF0F9BDAB213F0C00F089262D19DF88B
:1063300040800746404605F06BFB9DF84490484678
:1063400005F066FB129D002D57DB14989DF84CA0BC
:106350000E282BD00DF1280B0122594623F0CCFB3F
:106360000B9BAB4232D8BAF1000F2DD115980E28F5
:106370002FD028F085F902460021282009921EF02E
:106380008BFB099A3146214E0660CDE905B2089A89
:106390000092CDE9035ACDE901893B46002204462B
:1063A00005F020FC204617B0BDE8F08FBAF1000FD1
:1063B00011D0DDB916480DF1280B0122594623F002
:1063C0009BFB0B9B9D4201D39D42CFD0114829F0EE
:1063D00071FE0022D0E70DF1280B0D48012259462D
:1063E00023F08AFB0B9B9D42C0D2EFE7284627F0A3
:1063F0006DF8E0E7084829F05DFE084829F05AFEEC
:1064000060BE0800A4E908003CEA0800C0E40800F7
:106410006825090070A20900D0B60900889F09000C
:1064200043684BB110B5044621460448FFF704FB0E
:10643000002363600E2010BD0E207047A99003005A
:10644000F0B583B00546406801900E461F461446DD
:1064500002F086FE01983CF013FD40F201139E42CB
:1064600005D016233B604FF0FF3003B0F0BD14F0B1
:106470000100FAD0284605F07FFB003818BF012044
:1064800003B0F0BD70B52DED028B86B003AD234C8B
:1064900001950846009411461A4603231FF076FE24
:1064A0001F49039840F2DD221FF0B4FE0546049810
:1064B00025F08AFDB5EEC00AF1EE10FA26D4059E4D
:1064C000002E26DD00211C20B0EE408A1EF0E4FAEA
:1064D000144B03600446012130461EF0DDFA9FEDA7
:1064E000120AE06028EE008A0023BCEEC88AC4E9E4
:1064F00004630E486560A361214684ED028AFFF7BC
:1065000063FA204606B0BDEC028B70BD084829F046
:10651000D1FD084840F2CB2129F0D4FDA8BE0800E7
:10652000C0E40800E0E3080000007A44A9900300FA
:10653000C4B60900E4C1090010B50446406802F081
:106540000FFE204605F018FB400040F0010010BD92
:1065500070B50446406802F003FEEFF3108072B697
:10656000154B996829BB01229A60144A144ED2F83F
:10657000805035401D60C2F88060D2F884505D6064
:106580004FF0FF35C2F8845000B962B69868002217
:10659000C4E9052258B151B9EFF3108072B6074A29
:1065A0001C6814605C685460996000B962B60E2083
:1065B00070BD0121E8E700BFF454012000E100E0D4
:1065C000FC06FFBD70B582B00546406801901446D8
:1065D0000E4602F0C5FD01983CF052FC14B920466D
:1065E00002B070BD22463146284602B0BDE8704078
:1065F00005F064BA08B5014829F016FDD0BB0900C2
:10660000807D400040F00100704700BF8068002896
:1066100008BF0E20704700BF30B5848AADF5037DFA
:106620003CB9204602AD294626F006FF0DF5037D54
:1066300030BD4268D06800F0BBF8937901465BB981
:106640004FF4007302AD21466A46CDE900353FF0B4
:1066500003FF60B102F094FE02AD2A46204605F029
:1066600037FC294626F0E8FE0DF5037D30BDBDF868
:106670000000D8E78B688BB170B50C46054616460E
:10668000084929F0FBFBA1682846324600F046FE87
:1066900028460549BDE8704029F0F0BB034929F0C0
:1066A000EDBB00BF2075080024730800307508009A
:1066B00010B584B002AB51F8044B0193074B009323
:1066C000013802231FF0F8FC20469DF80C209DF8AD
:1066D000081005F0F5FA0E2004B010BD50CD0800EA
:1066E00010B5044684B00846012201A923F004FA3B
:1066F000A38A13B90E2004B010BD204601A905F0ED
:106700002BFB0E2004B010BD10B400230A4C1A4617
:1067100034F81310814203F1440306D00132052AF4
:10672000F6D100205DF8044B704702EB021204EB37
:10673000C2005DF8044B7047A805012008B5436806
:10674000132118883FF054FE0E2008BD30B587B0E5
:1067500005AB51F8044B01930F4B00930138012313
:106760001FF0AAFC6068039000F018F805990398E0
:1067700010F05AFD6568284600F010F86B68D3E900
:10678000020127F053F963680446586826F0B4FD07
:10679000204607B030BD00BF60CD080008B505F049
:1067A0005BFB00B108BD014829F022FC40BB090099
:1067B00018B143680BB1188870474FF6FF707047E7
:1067C00008B5406805F048FB002814BF3E201E2095
:1067D00008BD00BF38B544682046FFF7DFFF94F8D6
:1067E00074304BB10E4D04E0FDF746FF94F8743061
:1067F00013B16B6A002BF7D0B4F86C3007EE903A07
:10680000F8EEE77AB7EE047A67EE877A17EE900A29
:1068100020F0030040F00200A0F1FF4038BD00BFAF
:106820000C52012000B583B040680190FFF7B6FF1D
:10683000019805F019FB03B05DF804EB26F004BFE6
:10684000436833B193F85A30022B14BF1E203E2008
:1068500070471E20704700BF10B5002104460C2071
:106860001EF01AF9024AC0E90024E06510BD00BF1D
:10687000CCE5080030B585B003AB51F8044B01936B
:10688000224B0093013801231FF016FC6468204658
:10689000FFF784FF94F85A30012B0AD11C4D05E014
:1068A000FDF7EAFE94F85A30012B02D16B6A002BF7
:1068B000F6D094F85A30022B19D0012384F85A30BC
:1068C00014492088124D3FF085FD02F053FD94F8E5
:1068D0005A30012B06D008E0FDF7CEFE94F85A306E
:1068E000012B02D16B6A002BF6D06B6A13B10E201C
:1068F00005B030BD94F85B100029F8D0882902D08B
:10690000054829F0F9FB054829F0F6FBC0BE080050
:106910000C520120D86A090094AD090030AD09007D
:1069200070B504462DED028B084625F04DFB6568D9
:106930002846B0EE408AFFF731FFB7EE047AC8EE82
:10694000077A012385F8743005F16C06FCEEE77ACE
:1069500017EE903A9BB2A5F86C30A5F86E30314630
:1069600028883FF039FD0446FDF786FE112CF6D04D
:10697000204602F0FFFCBDEC028B0E2070BD00BF74
:106980002DE9F0478CB005AB4B4C01930431072344
:10699000013800941FF090FB4849059840F2DD2231
:1069A0001FF038FC464940F2A252064606981FF0F6
:1069B00031FC9DF81C800746404605F029F89DF8FB
:1069C0002090484605F024F8099D002D70DB0B98B7
:1069D0009DF828A00E282FD0012202A923F08CF8C0
:1069E000039BAB4257D8BAF1000F30D09D4252D131
:1069F000002118201EF050F8324B0360466000233F
:106A00000446876080F8168080F817908382039987
:106A1000029826F043FDB5F5FF7FE0603EDC25825D
:106A200084F812A0F3691BB12146304605F004F842
:106A300020460CB0BDE8F087BAF1000F22D1224801
:106A4000012202A923F058F8039B9D4223D3002181
:106A500018201EF021F81B4B0360466000230446FB
:106A6000876080F8168080F81790838203990298D7
:106A700026F014FDB5F5007FE060D0DD134A4FF439
:106A800000710EE085B91048012202A923F034F804
:106A9000039B9D42AAD20E4829F00CFB0D4A4FF4ED
:106AA000FF710D4829F00EFB284626F00FFDEBE79D
:106AB0000A4829F0FFFA00BFC8BE0800C0E4080079
:106AC0003CEA08007CE60800682509006C710800B3
:106AD00070A2090064710800949F0900889F090052
:106AE000406870478068002808BF0E20704700BFCC
:106AF00030B5848AADF5037D3CB9204602AD294608
:106B000026F09AFC0DF5037D30BD43685A68D068C5
:106B1000FFF74EFE937901465BB94FF4007302AD67
:106B200021466A46CDE900353FF096FC60B102F09F
:106B300027FC02AD2A46204605F0CAF9294626F070
:106B40007BFC0DF5037D30BDBDF80000D7E700BF2D
:106B50008B688BB170B50C4605461646084929F07E
:106B60008DF9A1682846324600F0D8FB2846054931
:106B7000BDE8704029F082B9034929F07FB900BF10
:106B800058750800247308006475080010B50446A1
:106B900084B00846012201A922F0AEFFA38A13B9EE
:106BA0000E2004B010BD204601A905F065F90E20A5
:106BB00004B010BD30B5130683B004460D4601D4B1
:106BC000022A06D02946204603B0BDE8304024F012
:106BD00009BF4FF41D7001923CF0A8F80146204611
:106BE00029F0E0F80549204629F0DCF8019A294609
:106BF000204603B0BDE8304024F0F4BE50730800D6
:106C000008B543681BB101460248FEF715FF0E2088
:106C100008BD00BFC9F2060008B54368DBB15A6879
:106C20000AB1927922B9588A400040F0010008BDAB
:106C30009A7D12F0060FF6D0438C4FF6FF729BB28E
:106C4000934208D0408C80B2FFF75EFD18B105F08A
:106C50000BF90028E8DA00F001F800BF08B5014898
:106C600029F028FA20B5090008B505F0E9F900284F
:106C700003DB400040F0010008BDFFF7EFFF00BF5D
:106C80002DE9F0438BB0344C009407AD08460195D4
:106C900011461A4603231FF079FA3049079840F24B
:106CA000DD221FF0B7FA089F002F50DD0546099836
:106CB0000E284AD025F0DEF9044600212C201DF0D4
:106CC000EBFE274B03606B6840F2FD1806469B798C
:106CD000A87DA04528BFA04600F0300200F00604C1
:106CE0009BB9BAB91746134614BBA146CDE9014872
:106CF00000243046CDF800903A4629460394F4F734
:106D0000A9FF30460BB0BDE8F083134622461C466F
:106D1000002AE7D008F1020307FB03F3013318460A
:106D2000002105931DF0B8FE059B0746002CDCD022
:106D30000021404605931DF0AFFE002181464046EC
:106D40001DF0AAFE059B0446D0E76C8AB5E705480E
:106D500040F2CB2129F0B6F968CD0800C0E4080064
:106D6000E0E70800E4C1090010B5436884B08BB1C6
:106D700004460222084601A922F0BEFEDDE9011206
:106D8000204605F0A1F9011E06DB480040F0010095
:106D900004B010BD3CF06EF80148494229F092F968
:106DA000B0BD090010B5174B8AB00C4602A9CDE959
:106DB000003101380223211D1FF07EF92468636829
:106DC000F3B10298012207A922F096FE039800234E
:106DD0000E28059312D0012204A922F08DFE0598F9
:106DE0000090DDE90712049B204605F0D3F920EA64
:106DF000E070400040F001000AB010BD1846EFE717
:106E00003CF038F800BF08002DE9F0412A4D2B4B2B
:106E10002B6004F01DFC08B9BDE8F081284BDFF8B9
:106E2000B4801B78002B3CD198F80030012B38D06F
:106E30002B6913B1204804F0CFFDEB6813B11E4855
:106E400004F0AAFD1F4C0023AB6104F52A774FF62E
:106E5000FF760E252088B0424FF0130101D03FF09D
:106E6000C7FAE5658834A742F4D145F04FFD1248D2
:106E7000002104F0FDFB4FF46A23134A1B68934280
:106E800005D14FF47122D2F8FC2F9A4201D000F0C4
:106E9000FDFB98F80030012BBED1BDE8F04145F074
:106EA000CDBA0A484368002BC2D0094B1B78002B8F
:106EB000BED005F0ADF8BBE7D446012038E20800AB
:106EC000AD5B0120A80501203130444288440120F7
:106ED000A75B0120C95B01202DE9F04F83B09DF82D
:106EE0003040CDE9004383B38B4619B30746924641
:106EF000002606F101081AF8066000240AEB0809CA
:106F00003D5D01343246494638193DB1AE4202D8A2
:106F10001EF0DEF990B12C44A345F1D8009B83B15B
:106F2000019B4644B342E4D8009B83F0010003B0C8
:106F3000BDE8F08F084603B0BDE8F08F009B002B42
:106F4000EED0009803B0BDE8F08F012003B0BDE89B
:106F5000F08F00BF8068704730B589B005AB51F83D
:106F6000045B0193104B0093013803231FF0A4F836
:106F70009DF81830B3B19DF81C4084F001040598C9
:106F800002A9012222F0B8FDEA68039BD2E90210AF
:106F9000029A0094FFF7A0FF002814BF3E201E2095
:106FA00009B030BD0124EAE710BF08000369D3E946
:106FB000020126F03BBD00BF8379002B14BF3E20A9
:106FC0001E207047C379002B14BF3E201E2070473F
:106FD0008068002808BF0E20704700BF30B587B01A
:106FE00004AD144C01950846009411461A4602233C
:106FF0001FF0CCF80498104940F2A2521FF00AF991
:107000009DF8142003920546002118201DF044FD30
:107010000A4B0360044600201CF0F4FF039A034669
:1070200029462046F4F7A4FE02F0A4F9204607B052
:1070300030BD00BF28BF08003CEA0800A4E90800F2
:107040008B688BB170B50C4605461646084928F08A
:1070500015FFA1682846324600F060F92846054928
:10706000BDE8704028F00ABF034928F007BF00BF01
:1070700088750800247308009475080008B5014855
:1070800028F0D2FF14B40900022808D1930704D1D4
:1070900010680B461A49884203D01E207047002012
:1070A00070479979012913D000B58BB0184602A911
:1070B000019205F003FA019A06A9104605F0FEF9BF
:1070C000029A069B9A420CD01E200BB05DF804FB7E
:1070D00091790129E8D1998893889942DDD13E20A0
:1070E0007047039A079B9A42EED1049A089B9A42F2
:1070F000EAD1059A099B9A42E6D13E20E5E700BF16
:107100003CEA080008B58B7823B10B8883808B7824
:10711000837108BD014828F0E1FF00BFB8AD090048
:10712000827940F20113012A14BF184621207047CA
:1071300000B58379012B85B009D0694605F0BEF909
:107140001021684626F0AAF905B05DF804FB014855
:1071500028F046FF549D09008088400040F001005F
:10716000704700BF70B50C468EB0114606464FF012
:10717000021220461D461EF073FF002108201DF05C
:107180008BFC066004462868C20739D483072AD1DD
:1071900003683F4A934233D03E4A0240062A26D033
:1071A0003D4A934223D0012206A922F091FC0028F7
:1071B00067D0079B102B67D1069B02AE18685968F1
:1071C0009A68DB6835460FC5BDF8142000238DF89A
:1071D00014308DF8153020463146A28005F058F95C
:1071E00020460EB070BD2B4B0340062BDBD101A90E
:1071F00027F01EFA019B242B0DD0284828F05AFFB7
:1072000024F038FFB0F5803F38D20123A08020461B
:10721000A3710EB070BD037A2D2BEED1437B2D2BC5
:10722000EBD1837C2D2BE8D1C37D2D2BE5D1421EE4
:1072300000F12305002612F8011F084648F0F0FA75
:1072400020B10EAB3344013603F8201C9542F2D135
:10725000202ED2D106AB0DF117010EAD187848F0F3
:10726000FDFA0246587848F0F9FA023340EA021073
:10727000AB4201F80109F1D102AEA5E7084828F0B8
:1072800019FF084828F016FF074828F013FF00BF31
:10729000245F09000F0080FFBC62090040AE0900B6
:1072A00058AE090030AE090084BD090010B588B0A1
:1072B00003AB51F8044B0193164B009301380223A2
:1072C0001EF0FAFE0222039805A922F015FCA2790D
:1072D000049B012A0CD0069903F11002914215D3A8
:1072E00005992046194405F0E9F80E2008B010BDB4
:1072F00006999A1C914209D3059AA188D154134446
:10730000A2880E20120A5A7008B010BD024828F058
:10731000D1FE00BF38BF080018BE09008A79012AD3
:107320000B463AD010B592B004460EA9184605F0A7
:10733000C5F89DF838209DF839100D929DF83A2037
:107340009DF845000090CDE90B2120469DF83C209A
:107350009DF83B409DF83D109DF844300193CDE9E8
:1073600009249DF83E209DF83F409DF84630CDE928
:1073700007219DF840209DF84110CDE905249DF896
:1073800042209DF843400294CDE903219DF8472017
:10739000044928F073FD12B010BD8A88024928F014
:1073A0006DBD00BFD0740800C0740800062801D06D
:1073B000002070478A79012A0B4615D000B585B0A8
:1073C0001846694605F07AF8ADF102030DF10E0199
:1073D000002033F8022F99421044FAD1400040F0C7
:1073E000010005B05DF804FB8888400040F0010012
:1073F000704700BF08B544F073F9BDE8084000F0DD
:1074000001B800BF2DE9F04F2DED028BDFF878A217
:1074100089B0002500AFAAF1080B05EB05130BEBB3
:10742000C3034FEA051893F87830002B40F0A08092
:1074300008EB05030BEBC30393F8793053B901351F
:10744000052D0AF1880AE8D12437BD46BDEC028B30
:10745000BDE8F08F1AF8069CB9F1000F00F0AC807F
:10746000BAF82E30FB60FA680121484616F05AFD42
:107470000446002800F0FE80C288502A05D15146FB
:1074800008301DF025FF00286AD00023BB6107F1FA
:10749000180320460122194608EE103A3FF006F87C
:1074A0001AF8069C002033F02FFD0446002834D043
:1074B0000AF14903BB6004E0204633F025FD044691
:1074C00058B36678012EF7D1237803F001034B45BA
:1074D000F2D1E388502BEFD1B9687B60062204F12A
:1074E00051001DF0F5FE7B6884461A4663465146FE
:1074F00004F10800C7F804C0002BDDD11DF0E8FE40
:107500007B680028D8D018EE101A32462046BB619E
:107510003EF0CCFF1AF8069CCEE7FB687B834FF069
:1075200000033B763AF8083CBB833B8B49F48079F7
:10753000502403F0FE0329F0FE0943EA090920461E
:10754000FC83A7F8189016F03FFD18EE101A0646B7
:1075500002223EF0ABFF2246514630464CF084F901
:10756000A8440BEBC8084FF0000388F8793066E7B1
:1075700045F0CCF9DAE91E23801A61EB0301B0F57E
:107580007A7F71F10003FFF453AF4FF00003FB82E9
:107590003AF8080C032307F1160200213EF058FFC9
:1075A0006C4668B108EB05030BEBC3034FF0000218
:1075B000A54683F878203BE7BAF81230FB6052E723
:1075C000FB8A3AF8080C0733DB08A4EBC3039D469B
:1075D00007F11602032369463EF03AFF6E46002883
:1075E000E0D11AF8069CBAF85020FA600221484609
:1075F00016F098FCFA680346002840D0F98AC28841
:107600008A4208D100F10801F86068461DF060FE6A
:10761000FB680028C6D018460023BB6107F1180399
:107620000122194608EE103A3EF040FF1AF8069C77
:10763000BAF850207A834FF000033B763A8BF88AF1
:10764000F88349F4007302F0FE0223F0FE031343B3
:107650003B833AF8083CBB8316F0B6FC18EE101AD0
:10766000814602223EF022FFFA8A314648464CF01B
:10767000FBF897E707F1180308EE103A12E707F155
:10768000180308EE103AD5E7B005012070B5104E8A
:1076900082B04FF46A240125200B357004F5805424
:1076A0003EF000FF08B93EF0E9FEB4F5722FF3D1C9
:1076B000084B019301A901224FF46A203EF0F6FE27
:1076C0000548012201A93EF0F1FE02B070BD00BFE5
:1076D000C15B012031304442FC1F0F001E3918BF2E
:1076E0000121490041F001011EF02CBF38B50C46C4
:1076F0002046114602221D461EF0B2FC0CB91E2087
:1077000038BD286825F06AFD0028F8D03E2038BD35
:10771000032A04D01E2907D0064928F043BB1E299E
:1077200005D0054928F03EBB044928F03BBB04497D
:1077300028F038BB64710800547108006C710800AF
:107740005C710800052807D01E3918BF01214900C7
:1077500041F0010129F0D2BC00207047136803B149
:107760007047406822F092BF00B583B08C46D0E9E4
:10777000010100931346624620F0F8F903B05DF86A
:1077800004FB00BF0023012200F000B82DE9F04700
:107790000C46096888B0054608461F46914624F005
:1077A000C3FC01228046084605A922F0A5F96068BD
:1077B000012202A922F0A0F99DF810100022402019
:1077C0001EF038FD012835D1DDE90561022D06EBFB
:1077D000010A14D9A2680E2A04D00346404622F0BA
:1077E00095F90644032D0AD0E2680E2A07D0DDE998
:1077F00005414046012322F089F904EB000AB24515
:1078000005D24FF0FF30C7B908B0BDE8F087039B41
:10781000029ACDF80090AAEB0601304616F0AEFBB6
:107820000028EED0059BC01A400040F0010008B0CF
:10783000BDE8F087024828F029FC024828F03AFC0D
:10784000DCAA0900C0BC090001231A46FFF79EBF4D
:1078500000234FF0FF32FFF799BF00BF01234FF025
:10786000FF32FFF793BF00BF70B588B00D460C2004
:107870000021164603931DF00FF9134B036004AB70
:107880000193124B039A0093314604230446284681
:107890001EF07CFC04984AF089FA054605984AF0E7
:1078A00085FA29790279069B914209D0002262600B
:1078B00029460246204604F00FFE204608B070BD5F
:1078C000034828F0F7FB00BFC4ED080000CB080018
:1078D000E4B6090008B5086804F0E4FE0E2008BD0F
:1078E00008B504F0DFFE0E2008BD00BF10B5044649
:1078F000807A01F047FC237A1BB9012323723E20D2
:1079000010BD1E2010BD00BF10B50446807A01F0E6
:1079100039FC002323720E2010BD00BF70B50C4649
:107920008EB054F8046B03920546B07A01F02AFC3D
:10793000307A01F0F7FC0AAB0193154B039A0093E0
:1079400021460423681E1EF0B7FB0B98022207A9EC
:1079500022F0D2F8DDE90C310898069006AA05A8B5
:10796000059333F07FFB069B5BB10798059ABDF842
:1079700028100244304604F0FDFE38B90E200EB047
:1079800070BD044840F2CA2128F09CFB28F054FB4B
:1079900008D0080018C2090070B50546807A01F0C9
:1079A000F1FB287A01F0BEFC00201CF02BFB082420
:1079B000064602E00134782C0ED0E1B2284604F0ED
:1079C00089FE0028F6D0610041F001013046013403
:1079D00025F06AFC782CF0D1304670BD70B50C46AD
:1079E0008EB054F8045B03920646A87A01F0CAFBF5
:1079F000287A01F097FC0AAB0193134B039A00938A
:107A000021460423701E1EF057FB0B98012207A984
:107A100022F072F8DDE90C310898069006AA05A854
:107A2000059333F01FFB0799059A069B01200090F0
:107A30000A442846BDF82810F4F7C2F910B90E2000
:107A40000EB070BD28F0F8FA70C1080070B50C4691
:107A500096B054F8045B03920646A87A01F092FBB4
:107A6000287A01F05FFC0FAB0193234B039A00933C
:107A7000701E072321461EF01FFB109801220CA93F
:107A800022F03AF8DDE912310D98089008AA07A80B
:107A9000079333F0E7FA1198022209A922F02CF893
:107AA000DDE914310A98069006AA05A8059333F07B
:107AB000D9FA069ECEB1059B099C0C9ABDF83C10E4
:107AC00003911C44079B1A44002300932846089BFB
:107AD000F4F776F970B9039933462246284604F044
:107AE00049FE38B90E2016B070BD044840F253412B
:107AF00028F0E8FA28F0A0FA30CF080018C20900F0
:107B000070B50C4688B054F8046B03920546707A41
:107B100001F03EFB307A01F00BFC04AB0193154BF6
:107B2000039A009321460423681E1EF0C5FA9DF8AF
:107B30001420012A12D89DF81830012B17D89DF86F
:107B40001C00A0F1080101290ED8009004993046CC
:107B500004F060FE28B10E2008B070BD064828F081
:107B6000A9FA052028F068FA044828F0A3FA044886
:107B700028F0A0FAE0D00800DCB60900FCB6090045
:107B8000F4B6090070B588B00D460C2000211646E9
:107B900003931CF081FF174B036004AB0193164B5A
:107BA000039A009331460423044628461EF0EEFA59
:107BB00004984AF0FBF8064605984AF0FFF8054697
:107BC00006984AF0FBF8034658B19DF81C206AB9A4
:107BD000626020462A46314604F05CFE204608B02A
:107BE00070BD002DF1D1054828F064FA044828F052
:107BF0001BFA00BFECEE080090C10800C0B50900F8
:107C000050B8090008B5086804F03EFF0E2008BD12
:107C100008B504F039FF0E2008BD00BF10B50446BA
:107C2000407A01F0B5FA63681B68D3F82435B3F1E4
:107C3000805F2ED012D9B3F1804F28D005D9B3F18F
:107C4000004F154818BF012010BDB3F1A05F18D038
:107C5000B3F1005F114818BF012010BDB3F1006FF0
:107C600013D005D9B3F1206F0D4818BF012010BD06
:107C7000B3F1007F07D0B3F1806F0A4818BF01202D
:107C800010BD094810BD094810BD094810BD09487C
:107C900010BD094810BD00BF0124F40001093D00DA
:107CA0000148E80121A107000190D00391D0030011
:107CB00041420F0001127A0081841E00037A1BB931
:107CC000012303723E2070471E20704710B5044602
:107CD000407A01F05DFA002323720E2010BD00BF30
:107CE00070B50C468EB054F8046B03920546707A5A
:107CF00001F04EFA307A01F01BFB0AAB0193144BF2
:107D0000039A009321460423681E1EF0D5F90A98B1
:107D1000022207A921F0F0FE0B98089B069005AA05
:107D20000C99059306A833F09DF9059A12B90E2017
:107D30000EB070BDDDE906109DF8343001443046C8
:107D400004F0D8FE0028F2D1052028F075F900BF14
:107D500068CF080070B50C468CB054F8046B0392E1
:107D60000546707A01F014FA307A01F0E1FA09ABB5
:107D70000193134B039A009321460323681E1EF0C0
:107D80009BF90998012206A921F0B6FE0A98079BE3
:107D9000059004AA0B99049305A833F063F9049A9B
:107DA00012B90E200CB070BDDDE905313046194422
:107DB00004F0EAFE0028F4D1052028F03DF900BFC8
:107DC00028D0080070B50C4694B054F8046B0392A8
:107DD0000546707A01F0DCF9307A01F0A9FA0EABB1
:107DE00001931E4B039A009321460623681E1EF042
:107DF00063F90E9801220BA921F07EFE10980C9BCE
:107E00001199079006AA07A8069333F02BF90F984B
:107E1000022208A921F070FE1298099B059004AA7D
:107E20001399049305A833F01DF9069B049A934215
:107E300011D113B90E2014B070BD0899059A0B9892
:107E40000A4407990144304604F064FE0028F1D149
:107E5000052028F0F1F8024828F02CF920CB080082
:107E600070A90900F8B50E461F4614462BF0CCF851
:107E7000054690F8240001F091F940F201139E426A
:107E800005D016233B604FF0FF321046F8BD14F0CA
:107E900001020AD16307F8D56B68187933F08AFFBD
:107EA0000028F2D142F00402EFE705F110003DF0A6
:107EB00001F9021E18BF0122ECE700BF2DE9F04FC7
:107EC0002DED028BA1B06E4C009414AD08460195C7
:107ED00011461A460C231EF059F9159849F06EFF09
:107EE0008146149849F06AFF0746002800F09F81F8
:107EF000DDF85CB0ABF10503042B00F2D181189ED4
:107F0000604B9E4200F098815F4B9E420CBF022660
:107F10000026199B013BDBB2012B00F2C7811A98A6
:107F200024F052F8B5EEC00AF1EE10FAB0EE408A35
:107F300000F1A081DFED557AB4EEE70AF1EE10FA18
:107F400000F398811C9849F039FF80461D9849F04C
:107F500035FF82461E9849F031FF9DF87C20049041
:107F60000121282003921CF0BFFD494901601B9BA1
:107F70000593BBF1080F99B2169DDDE90323044672
:107F800040F09181002B40F07781002A40F074810D
:107F9000426040480368D3F800351A0708D0836868
:107FA000D3F800351B0702D03B4828F083F808308F
:107FB0006060002F5DD0002900F06181022E00F08A
:107FC0006581B8F1000F00F045814FF0010C0023EE
:107FD0008DF84F30002F00F03A813B790D93B9F1C5
:107FE000000F00F0318199F804300E93BAF1000FC0
:107FF00000F027819AF804300F93B8F1000F00F0D9
:108000001D8198F80430B5F5966FCDE9103440F233
:108010002E8122494FF41662002302E001EBC302D5
:108020009268954203F1010301D9002AF6D101EBD0
:10803000C3035B6890F804B01293002E18BF0E269D
:108040008DF84E60164E8DF84DC00BEBCB0306EB52
:1080500083029B000321049392F820308DF84C108A
:108060000BFA01F103912BB30E4A0F490F4828F088
:108070005DF8B9F1000F9ED10D4828F01BF800BF44
:10808000B0C10800ECEF080010F008000000C84282
:1080900058F0080020030120A4BF090084DD080077
:1080A000205101200500AD0B64A509004C570900C3
:1080B00000AE09000DA9CDE90623F7F7A1F9016883
:1080C000079BC1F81031D1F810110C910C9901687F
:1080D000069AC1F82031D1F820110B910B99016853
:1080E000C1F82431D1F824110A910A990168C1F824
:1080F0004431D1F84411099109990168C1F8583106
:10810000D1F858310893089B03686A49C3F80413EF
:10811000694B01685360119B049AB35041F30732D5
:10812000002A9DF84C304FEA1131C0F2998002F1DB
:1081300060425B0102F56142DBB282F80033036802
:1081400043F3073100294FEA13320DDB4B099B0043
:1081500003F1604303F5614302F01F0101228A40ED
:10816000C3F880211A600368039A5A4406EB82061A
:1081700008210022C6E90622C3F800157261012217
:1081800086F82020B9F1000F0FD0BDF8141084F844
:10819000222004F110003CF04DFF002879D099F81E
:1081A000040084F8240001F093FA002F3BD03879C2
:1081B00084F8230001F08CFAB8F1000F29D098F868
:1081C000040084F8260001F083FABAF1000F26D0EB
:1081D0009AF8040084F8250001F07AFA9FED370A36
:1081E0006068A56028EE008A0023BCEEC88A84F887
:1081F000213084ED038A04F1200133F035FD304B4A
:10820000984202463ED1204621B0BDEC028BBDE82B
:10821000F08FFF2384F82630BAF1000FD8D1FF2366
:1082200084F82530DAE7FF2384F82330C4E7B9F176
:10823000000F7FF45DAE1FE701266AE64FF0FF33C3
:10824000E1E64FF0FF33D7E64FF0FF33CDE64FF0D6
:10825000FF33C3E6BAF1000C18BF4FF0010CB6E6CD
:10826000184A01F00F015B01DBB2535467E74FF48A
:108270009E23DFE649F03EFE134827F01BFF13481C
:1082800027F018FF1249134827F050FF124827F033
:1082900011FF606833F09AFD1049114827F03AFF4A
:1082A000104827F007FF104827F004FF0F4827F079
:1082B00001FF00BF1003420085F3070000007A446D
:1082C0000000AD0B14ED00E050B209005CB70900EE
:1082D00064A509004C570900E0B3090054B909002E
:1082E0004C560900B4A9090088B609006CC0090001
:1082F00008B5086804F084FC0E2008BD08B52AF013
:1083000083FE04F07DFC0E2008BD00BF10B52AF0EE
:108310007BFE044690F8240000F040FFA068400077
:1083200040F0010010BD00BF10B52AF06DFE0446FC
:1083300090F8240000F032FF04F110003CF0BAFE87
:10834000400040F0010010BD10B52AF05DFE04466B
:1083500090F8240000F022FFD4ED037A9FED077A15
:10836000F8EE677AC7EE877A17EE900A20F00300DE
:1083700040F00200A0F1FF4010BD00BF00007A44B1
:1083800010B52AF041FE044690F8240000F006FFE4
:1083900061680B6843F30732002A0FDB1B0B52099D
:1083A00011480121203203F01F0301FA03F340F8C2
:1083B0002230BFF34F8FBFF36F8F61680023C4E992
:1083C00006330B6843F30732002A4FEA133308DB06
:1083D0000548520903F01F03012101FA03F340F895
:1083E00022300E2010BD00BF00E100E038B50D4680
:1083F0002AF00AFE044690F8240000F0CFFE28463A
:1084000023F038FE6368A060B0F5966F1D6818D938
:108410000D4C4FF41662002300E08A68013390424D
:1084200004EBC30108D9002AF7D104EBC3035B684E
:10843000C5F824350E2038BD4B68C5F824350E200C
:1084400038BD4FF49E23F3E784DD080038B50D46B0
:108450002AF0DAFD044690F8240000F09FFE28463A
:1084600023F0B2FDB5EEC00AF1EE10FA10D4DFED44
:10847000097AB4EEE70AF1EE10FA09DCDFED067ACC
:1084800020EE270A0E20BCEEC00A84ED030A38BD98
:1084900049F030FD0000C84200007A4400B50B4BA3
:1084A00083B08B4214BF4FF4CD734FF4AD7340F2E1
:1084B000FB12CDE90023064940F2512340F2CE22BF
:1084C00027F0DCFC03B05DF804FB00BFECEF080014
:1084D0007C72080070B514460E462AF095FD0546DC
:1084E00090F8240000F05AFE0CB9204670BD2246D8
:1084F00031462846BDE8704004F0C0BB10B584B0DA
:10850000CDE9022101932AF07FFD044690F8240072
:1085100000F044FEDDE901320399204604B0BDE8D5
:10852000104004F035BC00BF30B50C4683B0114696
:10853000204606221D461DF093FD0CB32868C20795
:1085400011D5012C23D123F095FD01460190204641
:10855000F7F776FC019A04460021C0681CF07AFF08
:10856000204603B030BD830703D10A4B02689A420C
:10857000E7D00146012003B0BDE83040F7F730BB3B
:108580002146012003B0BDE83040F7F759BC02484E
:1085900027F07CFD245F0900C0C30900F7F786BB04
:1085A00010B5044682B0806801A926F041F8E3685E
:1085B000019A934207D2C05C4000013340F00100B1
:1085C000E36002B010BD002002B010BD32B9084611
:1085D00011B1194600F00AB80248704708B50248C0
:1085E00027F022FD6825090020A0090070B50A685F
:1085F000930790B00E46044625D111684D4B994221
:108600001ED04D4B1340062B21D04C4B99421ED00F
:10861000012C40F0868012F0010535D0521000F197
:10862000868011460CA801924AF096FE019A0E9897
:1086300000211CF00FFF3F480CA925F095F90246D8
:10864000104610B070BD3C4B1340062BE0D1A01E6D
:10865000012866D810460CA925F0EAFF3268364B8F
:108660001340062B054623D054680C9ED4B100213C
:1086700010201CF011FA2F4B03600246C0E902657E
:108680004460104610B070BD1046B22103AA21F01C
:10869000FDFF039B8BB103AA294628461FF0F4F87F
:1086A0000246CDE7284631463AF0F6F90446DEE7C1
:1086B00010093AF027FB0446D7E73068224605A99F
:1086C00021F006FA30BB306824F0C6FD0CADE0B1F5
:1086D000411028464AF02EFE306808A921F072FAAF
:1086E000044607E023F0C6FCFF281DD8C1B2284687
:1086F0004AF036FD204621F041FC0028F2D10D4819
:10870000294625F031F902469AE7102128464AF019
:1087100011FEE1E7DDE90512064825F005F90246FC
:108720008EE7074827F0B2FC064827F0C3FC00207C
:1087300027F0C0FC3C5A09000F0080FFBC62090012
:10874000C0C309003CA90900F0B585B0154606462E
:1087500023F0EAFC0C4607466946304625F068FFE0
:10876000042D12D1A307064603D1124B22689A4268
:108770000ED0009900232246384621F0C7F9305C1C
:10878000400040F0010005B0F0BD002005B0F0BD94
:10879000009801AA214627F02BFF40B1DDE9013204
:1087A0003846F118D21A25F025F905B0F0BD024877
:1087B00027F03AFC84620900709C09002DE9F0471B
:1087C0008F070C460646154610D001F00F03022B0A
:1087D00004D0B368002B5AD0BDE8F087D6074FEA23
:1087E000111150D5BDE8F0470AF0BCBF4968CBB2C3
:1087F0002D2B53D025D8062B3BD02C2BE9D1022A88
:1088000062D1E768002FE4D017F00308E1D17B685C
:10881000DAB28E2AB9465BD0312A74D0322AD8D146
:10882000012D00F09580022D00F09D80D9F80830D0
:10883000B06A1B09BDE8F04718226FF0010112F081
:108840009DBB2E2B13D1002AC3D1A168002937D09C
:108850008D0704D10A464968CBB2922B24D004F18B
:10886000080230460121BDE8F04700F083B89D2B97
:10887000AFD1002DADD104F108023046090ABDE8A0
:10888000F04700F077B8BDE8F0470BF0D7BB2146C2
:108890003046374ABDE8F0470BF022BCA268002AF8
:1088A00097D0002D95D15168090A022906D1D368C5
:1088B00023B1980702D11B79AC2B8AD008323046FD
:1088C000BDE8F04700F056B8A1680AF083FF98E7CA
:1088D0004FEA1329022D09F1FF390DD0B9F1000F2C
:1088E0000ADD07F1040A5AF8041F08F101083046AE
:1088F0000AF070FFC845F6D109F1020957F829902E
:1089000099F8042088E7022D0ED03046D9F80810D7
:108910000AF060FF012DB06A11D0BDE8F047562281
:108920006FF0020112F020BBB06A1FF01DFDB06AAB
:108930005622BDE8F0476FF0020112F015BB582235
:10894000022112F011FBB06ABDE8F0471FF08CBDA8
:10895000B06A1FF013FCD9F80810B06A0909BDE825
:10896000F0471FF0B1BBB06A1FF002FD5EE700BF29
:1089700004A909002DE9F04F814683B088460029FB
:1089800052D001399346171F0E0200244FF0FF3AD0
:1089900004E00134A045A6F580761BD057F8045FAB
:1089A000002DF6D0AB07F4D12B79222BF1D1BAF1FF
:1089B000FF3F44EA06034FF0310229D1D9F82800DD
:1089C0000191A246013412F023FBA0450199A6F5BE
:1089D0008076E3D1BAF1FF3F13D0002454450ABF9B
:1089E000DBF80030DBF800109968002248460134BB
:1089F000FFF7E4FEA0450BF1040BEFD803B0BDE890
:108A0000F08FD9F828004346302212F001FBE4E74A
:108A1000D9F80830002BF1D1084A2946484603B05E
:108A2000BDE8F04F0BF05CBB806A0B4630224FF084
:108A3000FF3103B0BDE8F04F12F0EABAC49E09005E
:108A40002DE9F04301F00F03022B83B00C4623D035
:108A5000054621B9AB682BB303B0BDE8F08311F034
:108A60000306F7D10B792C2B24D02D2BF2D1A4683F
:108A7000002CEFD063681B0A022B36D0002BEBD002
:108A8000271D57F8041F2846FFF7DAFF63680136F1
:108A9000B6EB132FF5D3DFE7090903B0BDE8F043C8
:108AA0000AF0E2B82D4A2146284603B0BDE8F0435B
:108AB0000BF016BB89680AF08DFEE768002FC9D05D
:108AC00017F00306C6D17B68DAB28E2A394615D074
:108AD000312A2AD0322ABDD18968A86A022209091E
:108AE00003B0BDE8F0431FF0D3BAE368002BC7D052
:108AF0009A07C5D11B79AC2BC2D1ABE71B0A03F196
:108B0000FF38B8F1000FC8BF07F1040907DD59F8B5
